:10000000C00A0020ED000000C1000000C100000097
:10001000C1000000C1000000C1000000000000009D
:10002000000000000000000000000000C10000000F
:10003000C100000000000000C1000000C10000007D
:10004000913A0000210800009D430000BD430000DC
:10005000C1000000C1000000C100000061110000EB
:10006000D90100002102000069020000B102000075
:10007000C1000000C1000000C1000000C10000007C
:10008000C1000000C1000000C1000000C10000006C
:10009000C1000000C1000000C1000000C10000005C
:1000A000C1000000C1000000C1000000C10000004C
:1000B000B93A0000C1430000C1000000C1000000C7
:1000C000094B5922162088211A6018601960A02354
:1000D000D805826882B00192019B01210B430193F4
:1000E000019A826002B070470001005008B50023F9
:1000F0000A4A0B499818884204D20A49CA5804335C
:100100000260F5E7084B094A934202D2002001C37E
:10011000F9E704F01BF901F059FE08BD00000020CA
:100120002C0000206CFE00002C000020BC060020EB
:1001300007B500230193032823D8134B1A686B4695
:100140005205520F03331A701A78002A02D103F0B5
:10015000C7FC0AE01A78012A02D1FA23DB010DE07C
:100160001A78022A03D103F0BFFC019007E01B7844
:10017000032B02D1054B1B6800E0054B019301984E
:1001800000E004480EBDC0461402005000000020EC
:1001900080B14F010197FFFFF8B5071C0E1C012825
:1001A00015D9002913D00D1C0124381C291C06F078
:1001B00057FE084B821E9A4203D8013C2406204376
:1001C00007E080230134AD195B009C42EDD1012092
:1001D0004042F8BDFDFFFF0013B50F4B01219A68A7
:1001E0000E4C0192019A0A430192019A9A60236887
:1001F0005B1823606368002B0CD0A368002B09D028
:100200002369013B2361002B04D1A06962699047F7
:10021000E368236113BDC046000001402C000020AC
:1002200013B50F4B01219A680E4C0192019A0A43B3
:100230000192019A9A60E3695B18E361236A002BDB
:100240000CD0636A002B09D0E36A013BE362002B08
:1002500004D1606B226B9047A36AE36213BDC04672
:10026000200001402C00002013B50F4B01219A689B
:100270000E4C0192019A0A430192019A9A60A36B73
:100280005B18A363E36B002B0CD0236C002B09D00D
:10029000A36C013BA364002B04D1206DE26C90475A
:1002A000636CA36413BDC046000011402C00002005
:1002B00013B50F4B01219A680E4C0192019A0A4323
:1002C0000192019A9A60636D5B186365A36D002BC0
:1002D0000CD0E36D002B09D0636E013B6366002BED
:1002E00004D1E06EA26E9047236E636613BDC046D4
:1002F000200011402C000020034B01221A675A678E
:100300009A67DA677047C0462C000020F0B585B0C8
:100310000C1C0092032800D9A1E0534B06F08CFD81
:10032000022C57801E6F012E00D09AE04F4A1568AC
:10033000002D00D095E04E48166081680391039F20
:1003400004210F430397039F311C8760494F3D6091
:10035000B86803900398014303910399281CB9607E
:100360001D609D605460FFF7E3FE211CFFF714FF42
:10037000431C4BD1404875E0586F012871D13B4A6E
:100380009568002D6DD13A4990608E680396039F61
:10039000082637430397039F8F60384F3D60B96845
:1003A0000391039901430391039EBE605D62DD6189
:1003B000D460FFF7BDFE211CFFF7EEFE411CD9D033
:1003C00003021B0A7B60009B000EDE0624E0996F8F
:1003D000012946D1254A1569002D42D124481161D1
:1003E00086680396039F102637430397039F876011
:1003F000234F3D60B868039003980143039103992C
:100400000220B9609D631D645461ACE7030200994A
:100410001B0A7B60000ECE0630433860281C21E0AA
:10042000D96F01291DD1114A9569002D19D11048A4
:10043000916186680396039F202637430397039FA5
:100440008760104F3D60B8680390039801430391A3
:1004500003990320B9605D65DD65D46183E70A48CF
:1004600000E00A4805B0F0BD2C000020AC000020E0
:1004700000020050000001400297FFFF20000140F1
:1004800000001140200011400197FFFF0397FFFF7C
:1004900073B50024032800D9C2E0624C06F0CCFCFE
:1004A00002316290256A002D00D0B8E05E48012636
:1004B0004660266A013626620195019C002C2EDCDE
:1004C000019D142465434519AD68002D15D1019D8A
:1004D000012665434519AE60019D65434519E960F4
:1004E000019D6543451929610199614341184A619C
:1004F000019A5443001983618FE0019C01340194F7
:10050000DBE7656A002D00D089E0474801260662D6
:10051000666A013666620195019C002C01DD0024AB
:100520007EE0019D1424654345196D6A002D15D1A7
:10053000019D0126654345196E62019D654345197C
:10054000A962019D65434519E9620199614341181A
:100550000A63019A5443001943635EE0019C01342D
:100560000194D9E7A56A002D59D12F480126C66309
:10057000A66A0136A6620195019C002CCFDC019D84
:100580001424654345192D6C002D15D1019D0126BC
:10059000654345192E64019D654345196964019DB4
:1005A00065434519A964019961434118CA64019AD8
:1005B00054430019036530E0019C01340194DBE7EA
:1005C000E56A002D2BD1184801268665E66A0136BA
:1005D000E662019502E0019C01340194019C002C2B
:1005E0009DDC019D142465434519ED6D002DF2D16C
:1005F000019D012665434519EE65019D6543451939
:100600002966019D65434519696601996143411851
:100610008A66019A54430019C366019C00E0034CAA
:10062000201C76BDAC0000202C0000200497FFFFAA
:1006300010B503282FD814246143174A174B5118BB
:1006400006F0FAFB020C162000208860196A0139B6
:1006500019621B6A83421ED153601CE0002048626D
:10066000596A013959625B6A834214D1136212E0FC
:1006700000200864996A013999629B6A83420AD111
:10068000D36308E00020C865D96A0139D962DB6A02
:10069000834200D1936510BD2C000020AC000020E7
:1006A00007B5032834D8802292051A4B06F0C4FB04
:1006B000020D18251849086801900198024301921B
:1006C000019A0A608022520014E0144908680190DF
:1006D000019802430192019A0A608022920009E087
:1006E0000F4908680190019802430192019A0A603B
:1006F0008022D2001A6000200BE00A4908680190AD
:10070000019802430192019A0A6080221201F1E7E6
:1007100005480EBD00E100E000000140200001405E
:1007200000001140200011400197FFFF07B503288A
:1007300033D81B4A1B4B06F07FFB020D18251A49C4
:1007400008680190019802400192019A0A60802293
:10075000520014E015490868019001980240019286
:10076000019A0A608022920009E01149086801900C
:10077000019802400192019A0A608022D200DA6751
:1007800000200BE00B49086801900198024001929B
:10079000019A0A6080221201F1E707480EBDC046A7
:1007A000FFFFFFDF04E100E0000001402000014006
:1007B00000001140200011400197FFFF07B50328FA
:1007C00015D88023DB0506F037FB02040610094A22
:1007D00002E0094A00E0094A1168002001910199EC
:1007E0000B430193019B136002E0054AF4E70548BF
:1007F0000EBDC04600000140200001400000114035
:10080000200011400197FFFF014B18687047C04658
:100810002C000020014B00221A6070472C000020A1
:1008200007B5084B08211A680192019A0A43019200
:10083000019A1A60044B1B6B002B01D000209847D3
:1008400007BDC04600400040AC00002007B50928A5
:1008500040D8214B1A68019206F0EEFA05080B14F5
:100860001E2225282B33019A802117E0019A80212E
:1008700021E0019A40210A430192019A1A60022262
:10088000164B1BE0019A40218A430192019A1A609B
:10089000134B0222DA6712E0019A10210A430BE09F
:1008A000019A102107E0019A0121F7E7019A02213C
:1008B000F4E7019A02218A430192019A1A6000200A
:1008C00009E0072211400A0201980649014011433C
:1008D0000191F2E704480EBD0040004000E100E055
:1008E00004E100E0FFF8FFFF0597FFFF37B51C4B61
:1008F0000F25DA680192019C0122AC431443019454
:10090000019CDC60DD680195019C1025AC430194DD
:10091000019CDC60DD680195019C20252C4301943D
:10092000019CDC605860996019690191019802434B
:100930000192019A1A61BFF36F8F18690124084D63
:100940002040FAD129684023194207D02868019035
:10095000019A044813430193019C2C603EBDC0469C
:1009600000C000508188FFFF13B51D4B0F24DA68CB
:100970000192019AA2430192019ADA60DC68019423
:10098000019A1024A2430192019ADA60DC68019472
:10099000019A2024A2430192019ADA605860002053
:1009A00098601C6901200194019A02430192019C04
:1009B0001C61BFF36F8F1869094AC407FBD4106824
:1009C0004023184008D01168019101980343019316
:1009D000019B0448136001E094680C6016BDC0469A
:1009E00000C000508188FFFF1C4B82B0D968019184
:1009F000019A0F218A4302210A430192019ADA6087
:100A0000D9680191019A10218A430192019ADA6012
:100A1000D9680191019A20210A430192019A01218A
:100A2000DA60586018690190019A0A4301920198AE
:100A30001861BFF36F8F18690121084A0840FAD185
:100A400011684023194207D01068019001990448A9
:100A50000B430193019B136002B0704700C000502C
:100A60008188FFFF0A4B82B05A68042101920198E5
:100A700008430190019A01215A60064B18680190C1
:100A8000019A0A4301920198186002B07047C0466B
:100A90000002005000C00050054B82B01A680121CE
:100AA0000192019888430190019A1A6002B0704740
:100AB00000C0005073B5FFF7A7FE0500FFF7AAFEC0
:100AC000022D00D8DBE10221D04B1A681C000A423B
:100AD00000D1D9E01A68D20617D5CD4B01391A7862
:100AE0008A431A70092D03D81A785218D2B21A7094
:100AF000C84A11781A784A401A701B78DB0700D56B
:100B00002DE11022236893435FE01A68920600D417
:100B10009DE004211A680A420DD140201A680A4358
:100B20001A60196881431960092D00D9A7E11A6874
:100B300002431A60A3E180211A688A431A60092DD2
:100B400002D81B680B4323604022236821685B089E
:100B500013400A40934200D091E104222368AD4E35
:100B6000934323602368AC4D1B0630D52B78317836
:100B7000AA4ADBB2C9B2D1542B783178A848DBB28B
:100B8000C9B2C1540023180029788B4204D8D15C23
:100B900001334840DBB2F7E7002800D0DFE0012254
:100BA00023680221134323609E4B0332DA679E4B76
:100BB0009E4A18700300FFF76BFC802223685205E1
:100BC0001343236022689A4B1340236057E12B782C
:100BD000DBB2002B02D0012B06D01FE03F2233787E
:100BE0009343802B00D1BAE08021924B49011A68CF
:100BF0000A4213D11A680A431A608F4B18888F4B28
:100C0000DB6801939847002803D022688C4B13407F
:100C100003E0802223681202134323602B7832788A
:100C20007E49DBB2D2B2CA542B7832787C49DBB22F
:100C3000D2B2CA5420222368934323602B78013315
:100C4000DBB22B702B78102B00D988E017E1714AAA
:100C500013785B00DBB21370092D03D813780133CE
:100C6000DBB21370774A13780133DBB21370137859
:100C7000072B05D9202123680B4323600023137021
:100C8000102223681343A0E78026186876023040BC
:100C90006C4A62D0AB1F032B04D821686A4B0B400F
:100CA0002360E5E02368DB060FD5684B1968490827
:100CB00019600A2D04D98020196880020143196047
:100CC000102123688B43236012E0614B19684908A7
:100CD00019600A2D04D98020196880020143196027
:100CE000102123680B43236013780133DBB21370A8
:100CF0001378122B33D81378122B00D0BFE080204A
:100D0000524B53491A68800252081A600A6802421C
:100D100002D11A6802431A6008681A6842401A60D1
:100D20001A684C4B9A4200D0A9E04B4B18680A68ED
:100D300090420FD1012223680221134323603A4BD2
:100D40001C321A700023394A1800FFF7A1FB2268F1
:100D5000424B39E70A681A6001E0042D15D8236870
:100D60009B0704D501213E4B3E4A1B78D154226893
:100D70003D4B134023600023324A1370264A137000
:100D8000334A1360314A136079E00A2D70D97D2D02
:100D900008D91A241968314319601968A1431960E8
:100DA00010706CE01378122BD9D923685B0706D535
:100DB00023680B4323602168234B0B4023600421ED
:100DC00023680B43236023689B0758D52368491881
:100DD0000B4323602168254B21480B4000212360F1
:100DE0000D4B117019700378632B03D91D4B0170E3
:100DF000197044E00F4A1168802212010A403ED166
:100E000001331849DBB20370CA5438E0840600206D
:100E100070060020250500208D050020BA03002063
:100E2000FD04002004E100E0F40500208D440000F2
:100E30000FFFFEFF94060020A8030020D0FC000056
:100E4000FF7FFFFF8E060020FFFFFEFF6C060020E5
:100E5000FC050020FFFF03002C05002001FFFEEF32
:100E6000E00000200006002000FFFEFFCBFFFEFF99
:100E7000082D00D973E713780133DBB2137073BD0B
:100E8000F7B58022A14E92033368A14D134333601E
:100E90002B8837009F4CDB042BD5002204212271C4
:100EA000627963880A43013362719B4A9BB2638013
:100EB00093420DD8994AD05C06F068FE984906F036
:100EC00097F9984B011CDB689748019398474CE0D1
:100ED000964A934206D1FC21924B8905DB689248E1
:100EE000019398476288924B9A423ED900236380CF
:100EF0003BE0042263799C46134236D0277963880D
:100F00007A1CD2B22271002A23D1591E894889B293
:100F1000844D814205D801339BB2638027717F4A9B
:100F20005FE0628063460422FC2193436371EB68B7
:100F300089057D48019398476379002B00D0E3E051
:100F40006B6979480193984732687B4B1340336053
:100F5000DAE0002B00D1D7E001336F4A9BB2638007
:100F6000934200D9D0E06D4AC2E02B8801269B0451
:100F70001DD50022637922711E4363886F4A0133B5
:100F80009BB24332D05C6380667106F0FFFD64491A
:100F900006F02EF9634B011CDB6863480193984708
:100FA0006288674B9A4200D8AEE0664B5AE062799D
:100FB0001100314039D021796388481CC0B22071BA
:100FC000002825D15A1E92B201925F4A554D94468F
:100FD000019A62450ED80133584A9BB26380217151
:100FE0004332D05C06F0D2FD4D4906F001F9EB68C2
:100FF000011C58E0FC21EB68608089054A48019398
:1010000098476379B343637100D07DE06B695DE01D
:10101000002B79D001334A4A9BB2934200D9494B05
:101020006380464B6288433362E02B885B041BD5A8
:101030002171022163880A4301336271434A9BB2E2
:101040006380934252D9424A934206D1FC21354BE8
:101050008905DB6834480193984762883D4B9A4282
:1010600052D9002363804FE002239C461A424BD0A2
:1010700026796388711CC9B2217100292ED1581EAE
:10108000354D80B2A84211D8344A01339BB2283280
:101090006380D05C267106F079FD214906F0A8F83E
:1010A000204B011CDB6801931F482CE063466180E4
:1010B000FC219A431B4B8905DB681B480193627135
:1010C00098476379002B1FD1164B5B690193164833
:1010D00098473A68184B13403B6015E0002B13D03B
:1010E00001331A4A9BB2638093420DD81B4A2832BF
:1010F000D05C06F04BFD0A4906F07AF8094B011C5A
:10110000DB68094801939847F7BDC0468406002074
:1011100042050020E000002042280000A8960000C0
:1011200000007F43B8FC00000602000043280000D6
:101130004FC9000041280000FFFFDFFFA8BE0000EC
:10114000C7050000AC050000E3250000B61500004F
:10115000B715000092200000B5150000A8E40000BB
:10116000042210B5024B1A60024B1B69984710BD50
:1011700044001440E800002013B51024064B074A31
:1011800019681088064B214201D01B6900E05B6999
:1011900001939847F2E7C04690050020B401002073
:1011A000B8FC0000044B4118884203D0027801309B
:1011B0001A60F9E77047C04600000540F0B5070027
:1011C00085B00C00002803D00300103B012B0AD887
:1011D000AE4B1A7F520706D50F21AD4A11701A7F08
:1011E0000E390A431A77FF2F0DD15F25FE2C00D050
:1011F0003D005922A74B1A60433A1A6072321A60B6
:10120000FFF730FCF9E0192F08D1A34B1A78002A18
:101210000ED1192C0CD89D4A947609E01D2F09D1C6
:101220009E4B1A78002A03D1192C01D8974A94773B
:10123000FF2227E108229A4B5B789343E52B32D1BA
:10124000984D8C3BEC55934C2360433B23607233A9
:101250002360FFF707FC002F04D1FA204002FFF7BC
:10126000C3FB15E0FB439B0712D1EA19531E197803
:10127000EB5D09041B06C918931E1B78033A1B0279
:10128000C9181378C918FA235B02F818FFF72EFB68
:10129000854A864B11680B401360FFF7FDFB002366
:1012A00002202360F0E03B001E3B784E012B01D969
:1012B000062F04D1B37E0220002B00D1E4E0072FDB
:1012C00005D1B07EC0B2002801D13070DCE0B37E21
:1012D0000137FDB2002B0BD00A2D09D800D1002513
:1012E0000A232822B07E58436B4B2D18EDB21A709A
:1012F000B37F002B0BD00A2C09D800D100240A237D
:10130000B27F53432822E418644BE4B21A70735D31
:1013100001209C4200D1B7E0AC2D1FD13300320038
:10132000AC331C70A93218781178884202D2127836
:10133000D2B21A7032003300AC32AA331078197866
:10134000884202D91B78DBB213703300AC331B78B0
:10135000574ADBB213706422564B1A7059224D4B18
:101360001A60433A1A6072321A60FFF77BFBF82367
:10137000DB01EF18BF0002A93800FFF7F5FA029968
:10138000FF220B001340934202D1994366182BE0D1
:10139000FF2C01D1745530E008009043464A90423A
:1013A00006D12340A6189C421ED02602434B15E0CE
:1013B000424A0B0C1804904206D1090A21408C4283
:1013C00009D12602130009E0090EFF2908D12340A4
:1013D00026069C4208D1FF2326041B06F61803E0CC
:1013E00021408C4209D1260631003800FFF77EFAF1
:1013F00031003800FFF77AFA38E0244A6BB25455CE
:101400000192002B19DBF8204002FFF7EDFA0026CD
:10141000019B9B5D013BFF3B0093F823DB01F71829
:10142000BF0000993800FFF761FA013600993800D3
:10143000FFF75CFA802EEBD118E0F9204002FFF7AD
:10144000D3FA8026019B9B5D013BFF3B0093F82371
:10145000DB01F718BF0000993800FFF747FA0136A3
:1014600000993800FFF742FAFF2EEBD10021144813
:10147000FFF73CFAFFF710FB0022064B1A60034B04
:101480005C55F93301201A7005B0F0BDD803002077
:10149000AD010020000100508F060020B4030020A1
:1014A000BA0300209905002084060020FFFFF7FF03
:1014B000FC0400209805002000FFFFFF0000FFFF54
:1014C000E4F301008021104B09011A68F0B50A43CA
:1014D0001A6000211A000D4D0D4E0E4F6B5C280056
:1014E0009C46735C34009C4502D013683B401360FB
:1014F00001311029F2D10023E25CD2B2C25401338F
:10150000102BF9D1F0BDC046840600203105002023
:10151000BA030020FFF7FFFF70B500240A4B21003B
:101520001C800A4B1C800A4B9D680A4B1888A847F0
:10153000094B21001888A847084A094B11680B403D
:101540001360084B1C6070BD88060020AC060020AC
:10155000D0FC0000B6010020C80100208406002055
:10156000FFFFEFFFB003002070B52E4C2E49637FC4
:101570002E4DDB0603D54B784233E35C19E0A379AB
:10158000012B2AD94B780E2B15D8A279A0784B784D
:10159000121AD2B2013B53439BB22B8028880D21F3
:1015A00080B205F05DFC80B22880A3782A88D31829
:1015B0009BB22B801FE06279A0794B78121AD2B2CD
:1015C0000E3B53439BB22B8028880E2180B205F03E
:1015D00047FC80B22880A379E8E76279A37848784D
:1015E000D21AD3B258431C2105F0C4FCA678F6B237
:1015F0008619B0B2288031340D4A237812685B080E
:1016000013400C4A1B0707D080212B8849045B0834
:101610002B8013680B4302E01168074B0B401360EB
:1016200070BDC046D8030020BA030020AC060020DD
:101630005005002084060020FFFFFFFE194A10B568
:1016400013689B032DD4184B1B685B0429D5174BDB
:101650001B7D1268DBB2520510D5E02B0CD003D8ED
:10166000FF21802B1AD01CE0F82B03D0FC21FE2B8D
:1016700014D016E0F02111E0C0210FE0F02B0CD0C7
:1016800003D88021C02B09D00BE0FC2B03D0FE2116
:10169000FF2B03D005E0F82100E0E0211320FFF745
:1016A0008DFD10BD8406002028050020D8030020F1
:1016B0008022F8B5234B9200196806000A401C00EE
:1016C000214D002A2ED1802101206F7F490307423E
:1016D00008D0002E08D01E680E421DD01B685B0586
:1016E00020D509E0002E0ED080221E68D2000E42C6
:1016F00005D01B681A4015D1144B1A8020E02368CE
:101700001A4322600CE01A680A4205D01B685B0588
:1017100008D50E4B1E8013E022680D4B134023604A
:10172000FFF78CFFE87CC0B2002809D00020EB7CDA
:101730005BB2834204DA80222368D20053402360E4
:10174000F8BDC04684060020D8030020AC06002067
:10175000FFFBFFFF5922094B10B51A60433A1A608C
:1017600072321A60FFF77EF9F82000214002FFF77D
:10177000BDF8FFF791F902F071F910BD00010050BA
:10178000F7B501251B4B1C4C0133D97F1B4F4A1C5D
:10179000DA771B4B2940A6681888002904D0290055
:1017A000B0473888002102E0B04729003888B047A8
:1017B000144B154FDB680021388801939847134E6E
:1017C000A46801213088A047114D01212888A04735
:1017D0000022104B1A601A68092AFCD9FE21019BCD
:1017E00038888905984730880021A047288800213B
:1017F000A047F7BDE8000020D0FC0000C801002091
:10180000B6010020B8FC0000A4010020B4010020B3
:10181000CC020020DC040020002803D0C0460138A0
:1018200080B2F9E770470000F7B58E4B0233DA7FDC
:101830000132DA778C4BDB6801938C4B1888019B63
:1018400098478B4D002814D12B002E000F27894A72
:101850003D333E361C78337811683B400B431360B0
:1018600033781168BB431B010B431360824B188014
:101870001AE0814B00241A882B00B1331B781B021D
:101880009A4211DA2B002F000F207A4A3D333E375F
:101890001C783B78116803400B4313603B78116858
:1018A00083431B010B431360744B1888019B9847BB
:1018B000704B002815D12A002F000F263F321278D6
:1018C000403714433A78196832400A431A603A782C
:1018D0001968B24312010A431A60694AA4B210801F
:1018E0001AE0674A11882A00B23212781202914235
:1018F00012DA2A002E000F203F32127840361443AD
:101900003278196802400A431A60327819688243B3
:1019100012010A43A4B21A601A68D20708D52A1D18
:10192000D17F2A0094321278120252181443A4B2C2
:101930001A68920708D56A1DD17F2A00953212785D
:10194000120252181443A4B21A68520708D5AA1DED
:10195000D17F2A0096321278120252181443A4B290
:101960001A68120708D5EA1DD17F2A00973212782B
:10197000120252181443A4B21A68D20509D52A00DB
:101980000832D17F2A00983212781202521814437A
:10199000A4B21A68920509D52A00283211782A00C3
:1019A00099321278120252181443A4B21A685205DE
:1019B00009D52A00293211782A009A3212781202A7
:1019C00052181443A4B21A68120509D52A002A3203
:1019D00011782A009B321278120252181443A4B2D2
:1019E0001A68D20409D52A002B3211782A009C32B9
:1019F0001278120252181443A4B21A68920409D53C
:101A00002A002C3211782A009D32127812025218C4
:101A10001443A4B21A68520409D52A002D32117851
:101A20002A009E321278120252181443A4B21A6885
:101A3000120409D52A002E3211782A009F3212781A
:101A4000120252181443A4B2FF22120214421FD0F1
:101A5000802208215200224214D0FF321440A4B246
:101A600016E0C046E8000020D0FC0000B2010020D3
:101A7000D803002050050020B80300209E0300205A
:101A80004405002001395200C9B292B20029E2D1C6
:101A90001A68D20305D52A00B43212789200144392
:101AA000A4B21A68920305D52A00B53212789200C2
:101AB0001443A4B21A68520305D52A00B63212782C
:101AC00092001443A4B21A68120305D52A00B73253
:101AD000127892001443A4B21A68D20205D52A00E3
:101AE000B832127892001443A4B21A68920205D553
:101AF0002A00B932127892001443A4B21A68520232
:101B000005D52A00BA32127892001443A4B21A689A
:101B1000120205D52A00BB32127892001443A4B2F7
:101B20001A68D20105D52A00BC32127892001443FB
:101B3000A4B21A68920105D52A00BD32127892002B
:101B40001443A4B21A68520105D52A00BE32127895
:101B500092001443A4B21A68120105D52A00BF32BC
:101B6000127892001443A4B21A68D20005D52A0054
:101B7000C032127892001443A4B21A68920005D5BC
:101B80002A00C132127892001443A4B21A6852009B
:101B900004D5C2352A7892001443A4B21A68824B45
:101BA000002A05DA1A00C332127892001443A4B254
:101BB0001900A73108787D4A002811D018000D7847
:101BC000A43011680078090A414079480D4202D0DA
:101BD0001900AA3101E01900A9310978C9B20170D0
:101BE0001900A8310978002904D11900A731097812
:101BF00000292AD0C02021008025800001406D00EE
:101C0000A94202D11900A9311BE08025AD00A942EB
:101C100015D0814219D11900AA310E7865490D7885
:101C20000800AE4205D11900A9310978604DC9B24A
:101C300029701900A9310D7801788D4205D119005C
:101C4000AA3109785A48C9B201705B481168156811
:101C50000088002820D011685848C90608D50168B6
:101C6000490501D5991C00E0D91CC97F0C43A4B2D9
:101C70000168490209D5597F490706D50168490518
:101C800008D5991CC97F0C43A4B2802500210120EE
:101C9000ED004BE0D91CF5E7F0260F202D11354063
:101CA0000840290001431800AD30007801421BD1E3
:101CB0001068424DC00608D52868400501D5981C1B
:101CC00000E0D81CC07F0443A4B2286840020BD5B2
:101CD000587F400708D52868400501D5981C00E0CA
:101CE000D81CC07F0443A4B21800AD300078014274
:101CF000CBD01900AE31097818000C431900AF3071
:101D00000078B03184430978A4B24C40BDE72B4F32
:101D10003F682F4203D107008F40BC43A4B2022783
:101D20009E5D3E4208D1013108290ED00E003536A5
:101D30009F5D0742F3D0EAE7204E36682E42F2D08C
:101D400006008E40B443A4B2EDE719008331097850
:101D5000490602D51168490708D41900833109786A
:101D600049B2002909DA1168090706D5190083313B
:101D700008783F2101400C43A4B21149C6330988B9
:101D80004842414149420C400E490C8010240E4902
:101D90000868204308601B7812681B021A4202D0B0
:101DA0000B68A3430B60F7BDD8030020500500204B
:101DB000FC040020B80600208806002084060020CD
:101DC0008C06002042050020940600201F21F0B55B
:101DD000E24A0124536893B08B4307390B435360A5
:101DE000A023DB059A6912391092109ADC4E224327
:101DF0001092109ADB4D9A61DB4ADC4814609A69B4
:101E00001092109A8A431092109A9A61336828802F
:101E1000019398477368210028880293984728887F
:101E20000025B6680021B047D14F019B3D802800B6
:101E300098472100029B3888984729003888B04786
:101E4000CC4FCD48019B388098472100029B3888B1
:101E5000984729003888B047C84FC948019B388047
:101E600098472100029B3888984729003888B04756
:101E70008120C44F80003880019B98472100029B3D
:101E80003888984729003888B047BF4FBF48019B22
:101E9000388098472100029B388898472900388865
:101EA000B047BB4F20003C80019B98472100029B1C
:101EB0003888984729003888B0470520B54F019BDE
:101EC000388098472100029B388898472900388835
:101ED000B0470420B04F019B388098472100029BF7
:101EE0003888984729003888B0478120AB4F400098
:101EF0003880019B98472100029B38889847290029
:101F00003888B0470420A64FFF303880019B98479F
:101F10002100029B3888984729003888B04707205D
:101F2000A04F019B388098472100029B3888984732
:101F300029003888B0479C4F9C48019B38809847BF
:101F40002100029B3888984729003888B047984F6D
:101F50009848019B388098472100029B3888984711
:101F600029003888B047C120934E80003080019B03
:101F7000984703213088029B9847904E9048019BD8
:101F8000308098470321029B308898470620019BA8
:101F9000FF30984706202900029BFF309847822097
:101FA000019B4000984782202900029B40009847EF
:101FB0008020019B4000984780202900029B400020
:101FC000984701237F4A5B4213807F4A7F491380F1
:101FD00059227F4B0D601A60433A1A6072321A60C0
:101FE0007C4B1A6A109210987B4A02401092109A09
:101FF0001A621A681092109A144310941C00109AD6
:102000001A60E368DB07FCD5C8230C220120150009
:102010001D43054202D152085B08F8E7023A50021C
:102020009A1EC0231B02134303430B60236A1093C1
:102030000B681098DB05DA0D430A5B021343F822A4
:102040001093109B92012362236A10930B681098DF
:102050001A40624B03401343C0221093109B12029C
:102060002362236A10930B6810991A405C4B0B4053
:1020700013431093109B5B492362236A1093109AB9
:10208000594B13401093109B2362236A1093109BAB
:102090000B401093109B23620391E3684D4A5B074A
:1020A000FBD5072113691093109B8B4305390B4314
:1020B0001093109B1361D3681B0603D5D3687E3140
:1020C0000B43D36002F00AF90122A36800211343F5
:1020D000E022A360454CD20023680800134323602C
:1020E000FEF7B4FB00210220FEF7B0FB402223687C
:1020F0001343236000243E4B1C60FEF7B3FCF82022
:1021000010A94002FEF730FC109B5B3300D0B7E013
:10211000FF2680343604F723DB01E518AD0010A953
:102120002800FEF721FC2700FF21109B803F1A0E9C
:102130009446100609062F4A88425DD119003140A5
:10214000B14207D1FF21180009020840884202D09D
:102150001B0A00E01B0CDBB2D35552E00003005019
:10216000D0FC0000B601002000E100E00603000002
:10217000C8010020A401002002020000B4010020D8
:1021800003020000CC020020A6030020050200008C
:10219000D0020020B0010020A4030020A2030020F0
:1021A000B8010020BA010020C60100200103000090
:1021B000A003002006020000B20100209E030020C0
:1021C00005030000B803002044050020B0030020F0
:1021D0000001005000020050FFFFF7FFFFC1FFFFAA
:1021E000FF3FFFFFFFFFFEFFFFFFFBFF0040004040
:1021F00028050020D8030020694663460B74097C3B
:10220000D15580239B00E81810A9FEF7ADFBFF27EE
:10221000109B0500190E0806A24A3F06B8420FD1CE
:1022200019003140B14207D1FF21180009020840CE
:10223000884202D01B0A00E01B0CDBB2135501E000
:10224000C9B21155802301345B009C4200D062E783
:10225000FA24954E640210A92000FEF785FB934AEC
:10226000109B9349A2188B541A0A32701A0C1B0E39
:10227000B370904B0434727004369C42EBD125E06D
:10228000F8204002FEF7B0FBF9204002FEF7ACFB5D
:10229000894F844EE35D3355F823315DDB01E5184A
:1022A000AD000139FF392800FEF720FB2300803301
:1022B000FA5C0134F254F15C802301399B00E81888
:1022C000FF39FEF713FB0500802CE1D1754C7B4AEA
:1022D0002300F9331B78DBB21370FEF7DDFB23001C
:1022E000002D04D1022076490A6802430A601A00D0
:1022F000A9321178272901D8282111701A00AA3291
:102300001178FA2901D9FA21117019001A00AC319B
:10231000A9320C781078844202D21278D2B20A70B4
:1023200019001A00AC31AA320C781078844202D914
:102330001278D2B20A701A00AC3212786149D2B265
:102340000A7061490A701A00AB321178C82901D9A4
:10235000C82111701A00A6321178632901D96321AE
:1023600011701A7DD2B2F02A11D006D8C02A0ED030
:10237000E02A12D0802A15D10FE0FC2A07D002D81B
:10238000F82A0AD00EE0FE2A07D0FF2A0AD18020C0
:102390004E49C0000A68024303E04C494C4A0868B1
:1023A00002400A609A1CD27F002A03D1DA1CD27F35
:1023B000002A04D00021474A1170033151702321B3
:1023C0002024022543485A5C002A05D0424A8A1834
:1023D000520084540132855401312F29F3D1202435
:1023E00002253C4885315A5C002A05D03B4A8A18B0
:1023F00052008454013285540131C429F3D11A00AA
:1024000031321278920704D5324A643991705739C3
:10241000D1701A0031321278520704D560212D4A4A
:102420001171573951711A0031321278120704D5DF
:102430006021284A91715739D1711A0031321278CE
:10244000D20604D56021234A1172573951721A00FD
:1024500031321278920604D560211E4A91715639A4
:10246000D1711A0031321278520604D56021194A0E
:1024700011725639517211200222942140241027E2
:102480008446585C102804D11248551C8454664672
:102490002EE0585C202823D10E48551C8454475503
:1024A00027E0C046D80300209A050020000CFEFF5C
:1024B0009905002014F4010087FA0000F3050020BC
:1024C00028050020B8060020FC0400208406002017
:1024D000FFFBFFFF55050020DEFFFF7F59FFFF7F59
:1024E000585CC0B2402804D10F26E44DA854501CBB
:1024F0002E54023201311C2AC3D1A02380210C208A
:10250000DB05DA6849050F920F9ADD4C0A430F92FA
:102510000F9ADC4EDA60DA6803270F920F99DA4AD5
:102520000A400F920F9ADA60D84A51690F910F99B9
:1025300081430F910F99516191690F910F9921403A
:10254000B0242403214380240F910F9964059161E5
:1025500091680F910F9921430F910F999160CC4988
:102560000C6A0F9401240F9D25430F950F9D0D625A
:102570000D6A0F950F9D35400F950F9DC54E0D624D
:102580000D6A0F950F9D85430F95FF250F980862E3
:10259000486A0F900F98A84320430F900F98EF3D83
:1025A0004862596BBC480F910F9921430F910F99C5
:1025B0005963596B0F910F9901400F910F9959630E
:1025C000B64908680F900F98B8430F900F980860AD
:1025D000586B0F900F9828430F900F98B04D586389
:1025E000586B0F900F9828400F900F985863086809
:1025F0000F900F9DAB4828400F900F980860586BC4
:102600000F9020200F9D05430F950F9D5D635D6B1F
:102610000F950F9D35400F950F9D5D630D680F95CC
:102620000F9EA14D35400F950F9D0D609F4D296860
:10263000214329609E4D9F492E68314039432960CE
:102640009D4D9E492E683140C02636013143296098
:102650008025D9686D020F910F9929430F910F9929
:10266000D960D968039E0F910F9931400F910F994E
:102670000226D96093680F930F9B1D430F950F9B04
:1026800093608F4B99680F9104210F9D0D430F9517
:102690000F9D9D609D680F950F9D35430F950F9D74
:1026A000EE369D609D680F950F9DB5430F950F9D6C
:1026B000844E9D60DD680F950F9D85430F950F98A3
:1026C000D860D8680F900F9807430F970F98D8607D
:1026D000D8680F900F9888430F900F98D860D868EB
:1026E0000F900F9888430F907F200F99D960196A37
:1026F0000F910F9981430F910F99196253690F93AD
:102700000F99714B0B400F930F9B5361956901F02B
:10271000E7F98022336892050F930F9B2D05134331
:1027200080220F930F9B5205336033682D0F0F9358
:102730000F9B291913430F930F9B644D336033682C
:102740000F9304F08DFB624904F08AFB0F9A023864
:1027500083B2100C000418430F900F9B3360FDF7F9
:10276000CBFD22005B490020FDF7D0FD0020FEF7E5
:1027700025F80020FDF794FF2200C8212000FDF776
:10278000C5FD2000FEF71AF82000FDF789FF2100A3
:102790000023514A2000FDF77BFEC2229200A95877
:1027A0004E4B4F4E0B40C02109020B43AB503368D8
:1027B000039398474B4F73682100388805939847D7
:1027C000B3684949388804939847F368474938887B
:1027D0000693984733693888079398477369388810
:1027E00008939847424E40493088049B98472100FF
:1027F0003088059B98473D493088069B984730882C
:10280000079B98473088089B98473A4E21003088AC
:10281000059B984730883449049B98473349308852
:10282000069B98473088079B98473088089B9847B5
:10283000314E2100059B30889847304B34885A7AB6
:102840000393104B09930E4B0C93134B0B93144BA8
:102850000D93104B0A93002A56D0039B587AC0B2AE
:1028600006F0E2FD264A274B06F010F802000B00A6
:1028700005F0CAF906F06EFE011C46E05505002081
:10288000FFFF00FFFFFBFFFFFFFFFFEF0002005015
:1028900000000E40FFDFFFFFFFFEFFFF4040005043
:1028A000FFEFFFFFFFFCFFFFFFF3FFFF2805002006
:1028B0003C000050FCFCFFFF30000050F3F3FFFF32
:1028C0000000054024000540FFFFFFFC00E100E0A0
:1028D00090D0030048E80100D1570000FF00FFFF3F
:1028E000B8FC0000B40100206F12833A0AD7233CE1
:1028F000A6030020CC020020A4010020D803002061
:10290000FA9CBB5D2F4D013FE3492000049B984793
:10291000FE21E24C89052088069B98472088079B6A
:102920009847DF4CDF48019B208098472088002192
:10293000029B98472088DC4C0321A36801939847A9
:102940002368DA4801939847FA210122C90002203E
:10295000FDF7DCFC0220FDF731FF0220FDF7A0FEB1
:102960000023D34A01210220FDF792FDC2229200EA
:10297000AB58D0490B408021C9030B43AB50CE4B21
:102980001A00A7321278002A03D1A8331B78002B33
:102990001FD0CA4BCA481978C9B204F0EBFA012219
:1029A00001000320FDF7B2FC0320FDF707FF032021
:1029B000FDF776FE0023C34A01210320FDF768FDE1
:1029C000C222C0219200AB5809061B021B0A0B430E
:1029D000AB50BD4CBD492088049B984720880121FD
:1029E000059B9847FC2120888905069B98472088ED
:1029F000079B98472088089B98470422B449802069
:102A00000B6C00240F930F9B000613430F930F9B37
:102A10000B64B049B04B19618023C1212B60890040
:102A20006B581B021B0A0343AC486B50AC49046053
:102A30000B6813430B60AB4B196811431960AA492B
:102A40000C80802419686405214319600F21A74B6D
:102A50001970994B190031310978049049B2002955
:102A600002DB197F91431977002301930293E0223F
:102A70009F4BD2011B889B4D9E4C13420FD080224E
:102A80002B689203134205D18F4B18889A4B1B6910
:102A900005939847802223681201134302E02268BD
:102AA000964B13408E4E236033685B0500D489E05B
:102AB000402733683B4217D000207F4C6178637811
:102AC000C9B20133DBB26370A077A076FEF776FB64
:102AD000617F637FC9B20133DBB21C206377FEF7ED
:102AE0006DFB3368BB43336080277D4E33683B42C8
:102AF00021D00023704C1020A377A376617C637CE7
:102B0000C9B20133DBB26374FEF758FBA17CA37C2E
:102B1000C9B20133DBB21120A374FEF74FFB617F12
:102B2000637FC9B20133DBB21C206377FEF746FB3B
:102B30003368BB433360039AF820F9321178137875
:102B4000C9B20133DBB21370FEF738FB039AF920E8
:102B5000FA3211781378C9B20133DBB21370FEF781
:102B60002DFB039AFA20FB3211781378C9B2013396
:102B7000DBB21370FEF722FB039AFB20FC321178C4
:102B80001378C9B20133DBB21370FEF717FB039A57
:102B9000FC20FD3211781378C9B20133DBB2137017
:102BA000FEF70CFB039AFD20FE3211781378C9B2B0
:102BB0000133DBB21370FEF701FB494A0999136830
:102BC0000B401360464C23689B040BD5FE21FF206D
:102BD000FEF7F4FAFF210800FEF7F0FA23680A9ADC
:102BE0001340236001262B68334200D13FE7802247
:102BF0002C68120514401ED12B68414F13432B60E3
:102C00004048414D3B682880059398477B683100D8
:102C10002888069398472100BF682888B8473B4C0E
:102C20003B48059B2080984703212088069B9847B6
:102C300020883100B84780222A4D12042B682D4984
:102C400013432B602A68334B134020222B600B6800
:102C500093430B600021304B19702B681B0700D584
:102C600043E215494B7F134200D03EE22B4B2C48E8
:102C70001A68D2B2865C4A782A68920156D40A0051
:102C80002F32127896424DD14E7880212A68C9049D
:102C9000F6B20A4349E0C0467B690A38A401002025
:102CA000A803002002030000E0FC0000B50A0000B9
:102CB0005D5F0000FFFF00FFD8030020B806002082
:102CC000A0860100396D0000A00300207B698A38CE
:102CD00000001440810E0000E800002000010050B8
:102CE000280500208406002088060020AD01002071
:102CF0004205002094060020B8FC0000FFF7FFFF0B
:102D0000D0FC000006040000C40100209C03002049
:102D100007040000FFFFBFFFAF0600202C050020C6
:102D200087FB00002968AD4A0A402A60AC4A527805
:102D300096420CD02A68920309D4502E01D000F09C
:102D40004FFEA84A1268520701D400F049FE2968D4
:102D5000A54A0A402A602A6892031FD42A685201B1
:102D60001CD4802019681024A04A8000C90506D50B
:102D70001168214311601B68034206D00AE0116804
:102D8000A14311601B68034204D080222B6892018A
:102D9000134302E02B680A9A13402B60944B954A28
:102DA0001B685B010CD51168904BC90504D58020C8
:102DB00019684001014302E019680D98014019604B
:102DC00013688B4C9B0A13605523116810681940D7
:102DD00040080340994200D1DCE080212B68C90102
:102DE0000B432B601368DBB2272B01D1183B1BE090
:102DF000322B01D1023B17E0362B01D1063313E011
:102E0000372B01D108330FE0CD2B01D102330BE07A
:102E1000784AD82B01D1183306E0DC2B01D12033BE
:102E200002E0DD2B01D12233136023685B0131D432
:102E3000704B0822196889070CD51968114229D1ED
:102E40001B689B0626D58027654BFF005B7FDB0751
:102E500015D50BE0196811421CD01B689B0619D4CC
:102E600080275F4BFF005B7FDB0708D423683B4272
:102E700010D1FEF751FB23681F43276008E0236849
:102E80003B4207D0FEF748FB2368099A13402360B2
:102E9000FEF7D4FB0220574B554A1C680821044218
:102EA00038D01868084279D080241F68E4044F485D
:102EB000BF0616D5176880221B68274208D0134228
:102EC00003D08022036812011EE002684A4B15E01D
:102ED000134203D00368194301605FE003688B432A
:102EE00016E0126880211B68224209D00B4203D0F1
:102EF00080220368520007E003680B9A134007E042
:102F000001220B4202D00368134301E0036893439C
:102F1000036043E01C6820270C421DD11968394228
:102F20003CD080241768E4048021304A1B68274283
:102F300008D00B4203D081311368FF3125E01168BE
:102F40002E4B1CE00B4203D013681843106025E0A1
:102F500013688343136021E0196839421ED080242E
:102F60001168E4048020214A1B68214209D00342F1
:102F700003D080211368C90007E0136809990B404A
:102F8000E8E70421034202D013680B43E2E7136829
:102F90008B43DFE722681A4B13402360144C2368ED
:102FA0005B0104D523689B0301D400F013FD0123CA
:102FB000104A11680B401168490701D502210B43E3
:102FC0001268D20601D5042213430A4A054F12683B
:102FD000520617D50822134360E0C046FFFFFFFBEF
:102FE000D803002028050020FFFFFFFD500500202A
:102FF000840600202C050020FFF7FFFFFFFDFFFFE8
:10300000FFBFFFFF012B47D1502E06D13B685B0766
:1030100003D5029B0133DBB20293019B012B29D024
:1030200023689B031DD5CB4B1A78002A19D1963201
:103030001A7080222168D202C74B11420DD0187835
:1030400031000138C0B2FEF7B9F8002801D1FEF70F
:1030500081FB2268C14B134002E01E7023681343BA
:10306000236080222B68D20053402B60FEF7E6FAE3
:10307000FEF752FA01230193029B802B01D800F046
:10308000A9FC80222B689202134304222B603B6828
:1030900093433B6000F09EFC012B04D980213A68E9
:1030A000C9010A433A6004213A688A433A602268B7
:1030B000920301D500F091FCA94A002B10D0013BEE
:1030C000DBB221685B00DBB2890401D4013BDBB2D7
:1030D000A4494B709BB21380FEF746FA002300E030
:1030E00013800193029300F075FC2A689E4B1340F5
:1030F0002B609E4B1E782B68F6B2DB0500D41FE1D7
:103100000320FDF713FB0F21964B1A781C008A430E
:10311000702A00D011E12A68120500D49DE31A78C4
:1031200092077BD15A78C72A78D85978C9B24A1CF5
:10313000192A08DC152A0CDA0A2A0AD007DB0D390D
:10314000022904D805E0422A03D05F2A01D00020DA
:1031500000E001205A78C72A01D900F041FC00287C
:1031600001D000F03DFC0C2219780A40082A04D056
:103170000C2A45D0042A4ED13AE01F219A788A437E
:10318000E02A48D10725DF3AA1782940884204DAAD
:1031900052000130D2B2C0B2F6E79978744CC90639
:1031A00017D59978090704D559780131615C114325
:1031B00003E059780131615C91435878F934C0B229
:1031C000FDF7FCFF0021F920FDF7F8FF0023237035
:1031D0000BE059780131615C0A4099780823194065
:1031E00001D0002A01D10A4315D1FEF7C9FA12E035
:1031F0009A785B785E490133CB5C9A420BD1F4E755
:1032000058789978C0B2C9B2FDF7D8FF0028ECD140
:10321000FEF7A0FAE9E7574B1B8819E319785A78AB
:1032200003230B401B029B18059301339FB2E0233D
:103230009B009F4204D9504BFB18012B00D8CFE3D1
:103240004E4D4F4C6B682088032106939847AB681E
:10325000012120880693984701F0ECF86420FEF7DE
:10326000DBFA0F233F4903240A781340454A7033A1
:1032700013704B78DBB253708B78DBB29370002203
:10328000414B1A703220FEF7C7FA082601252800A4
:1032900001F0DCF81920FEF7BFFA6D0001F0CAF862
:1032A000013E1920FEF7B8FAEDB2002EEFD1364AF2
:1032B000013C1378E4B20133DBB21370002CE1D18E
:1032C0002F4B01211888069B98476420FEF7A4FA2B
:1032D0006B460A251C776A46FA262C4B127F1A7019
:1032E0001920FEF799FA264B1888244BDB680693C1
:1032F0009847041E18D1059B254A9B189BB20C2B9E
:103300000FD8184A1378DB431B070AD1380091788D
:103310006330C9B2C0B2FDF751FF2100F920FDF7BB
:103320004DFFFEF72DFA03E0013EF6B2002ED7D195
:10333000013DEDB2002DCED152E30320FDF7B0F9EF
:10334000084A1378002B25D180222B689200134362
:103350002B6054E068060020D0030020FFFFFBFF35
:10336000AC060020BA030020FFFFFDFF8D05002002
:10337000D8030020420500207EFCFFFFD0FC0000A7
:103380009C0300200400002090060020F40500208B
:103390007BFCFFFF2968C24B0B402B60C14B597F60
:1033A000107889061AD5597C884211D15078997CB9
:1033B00088420DD10221535C481EDBB20131135407
:1033C0001029F8D1B84A1378013BDBB2137011E031
:1033D000DA7C002A00D103E3B44A06E05978884237
:1033E00008D0D97C002900D1FAE21278DB7C9A421D
:1033F00000D0F5E2AD4B5B78E42B00D1F0E2AC49B4
:103400000B78002B0ED0A74A137F5B070AD50B78E9
:10341000013BDBB20B700B78002B03D10121137F32
:103420008B431377802204212B6892041343A14A13
:103430002B6013689D4C8B4313602B680B990B40DA
:103440001F212B6063788B43602B00D126E208D8C4
:10345000202B00D186E0402B00D11FE2002B0FD0A3
:10346000BEE2A02B00D17CE203D8802B00D1F7E193
:10347000B6E2C02B00D193E2E02B00D14EE1AFE2E7
:10348000032E00D9ACE26378DB0615D503236278FE
:103490001340022B01D1A37801E0A378803B814A3D
:1034A000DBB2D17C8B4200D19AE2D374D17C132061
:1034B000C9B2FDF783FE93E20F2366781E40012E0A
:1034C0003AD0002E05D09E4200D089E2FEF758F98E
:1034D00086E2FEF721F8784B5F69784B1888B84789
:1034E000774B1888B847774B1888B847764B310028
:1034F0009F68764B1888B847754B31001888B847D5
:10350000744B31001888B847734B31001888B8479E
:10351000724B31001888B84780222B685200134341
:103520002B6023780196002B00D059E26C4BFD3ABA
:103530001A700023019353E25A4C637F0E2B06D07E
:103540000E236377617F1D20C9B2FDF737FEE37C50
:10355000002B04D000211320E174FDF72FFE00F0B2
:103560008AFA3DE280211368C9010B4313605C4B6A
:103570001A78032A01D100221A704A4DEB7C2F00E1
:10358000002B04D0EA7C23789A4200D028E2554BE5
:103590001A68D20700D523E21B689B0700D51FE2FB
:1035A0007F26A078B043FEF783F8002800D017E20A
:1035B000A3781E40A67009D0A378013BDBB2A370AC
:1035C000A378002B05D1FDF7A7FF2DE0464B1E8009
:1035D0002AE0A3783E2B00D909E2AA79AB78A0783B
:1035E000AD78D21AEDB2D3B258437E2103F0C2FCBB
:1035F0006D083D4B281880B2188031373B4A3B7824
:1036000012685B0813403A49374A1B0700D1F7E1BB
:103610008020138840045B0813800B6803430B6011
:1036200013885B009BB2138063783C2B00D0D7E1FA
:1036300000222E4B1A601C4A10780438032800D947
:10364000C8E1E27819681207520F0A431A60E2785B
:1036500003F0F2FB02081550D20700D4BAE11A6851
:103660001021B5E1D20703D510211A680A431A6068
:103670001E4923790A68DB0213430B60AAE1D207D3
:1036800003D510211A680A431A60184B2279196869
:10369000D2020A431A6062791968D20498E1C046DE
:1036A000FFFDFFFFD80300208D050020BA03002096
:1036B000AD01002028050020B8FC0000B401002066
:1036C000CC020020A6030020D0FC0000D002002085
:1036D000B0010020A4030020A2030020B8010020B4
:1036E0002405002094060020AC0600205005002090
:1036F00084060020D20703D510211A680A431A60F5
:1037000022791968D2020A431A6062791968D204D0
:103710000A431A60A2791968D20659E12B681B0581
:1037200000D49AE0A3781E2B59D9A3782A2B56D817
:10373000A278B54BE1789A181F3A11700122A1784E
:10374000B2481F398A4001880A43B14992B20280C7
:103750008A4244D11A783E2A01D0FDF70DFD5A78ED
:10376000002AFAD19A78002AF7D1DA78342AF4D1EB
:103770001A79022A14D15A79062A11D19A79002A83
:103780000ED1DA79002A0BD11A7A302A08D15A7A66
:10379000052A05D19A7A202A02D1DB7A162BDCD0B1
:1037A0005923049A1360049A433B1360049A7233BA
:1037B0001360FDF757F9FF204002FDF715F9954911
:1037C0009548FDF793F80321944A13680B4310932F
:1037D0001360FDF761F9924A924B1A60FEE7924B33
:1037E0001B88002B02D00022884B1A8008216278A7
:1037F0008E4B8A438E4DE42A1AD1A278E92A0CD145
:10380000E278AA2A04D180211A6809030A4302E057
:103810001968884A0A401A60E2E0A078E178C0B2EC
:10382000C9B2FDF7CBFC002811D1FDF793FF0EE0E4
:103830001B681B0300D4D3E063788B43E52B00D0D7
:10384000CEE0A078E178C0B2C9B2FDF7B7FC2B8812
:103850000133794A9BB21380C2E0FDF733FEBFE02B
:10386000042E00D9BCE0754BD87C2278904200D160
:10387000B6E05A7F724B920708D51A688A431A60DD
:1038800060781A68014011431960A3E00F2219689B
:103890009143196060781968024099E080211368AB
:1038A000C9010B431360674B1A78032A01D1002228
:1038B0001A70624DEB7C002B04D02278EB7C9A428C
:1038C00000D08DE00127604B1A683A4200D087E0B3
:1038D0001B689B0700D583E0042E00D980E02023DD
:1038E00060781840FDF7E4FE002879D11F23627844
:1038F0001340637063781B0702D14B4B188038006C
:103900000F2366781E40012E02D1FDF705FE300020
:103910006B7F9B070DD410216278494B0A4202D07D
:103920001A680A4301E01A688A431A6063785B00E8
:1039300008E063785B00DBB2637063789B0603D5B5
:1039400063780133DBB263701F23627813406370C6
:103950006378033BDBB26370002841D1FDF704FEBE
:103960003EE0042E36D8354BDA7C23789A4237D0A5
:103970006278334B1968D20608D5344A0A400F21C1
:103980001A60627818680A40120207E0304A0A405A
:103990000F211A60627818680A401203121818E0A2
:1039A000264BDA7C23789A421AD06278244BDE2A9E
:1039B00007D11A680C990A401A60A2781968120493
:1039C00006E01A681202120A1A60A2781968120632
:1039D0000A431A60FDF728FF02E0002301930293D7
:1039E000124A1C4B11680B401360FFF740F86B79CB
:1039F000AA79A078AD799B1AEDB23F38DBB2F3E536
:103A00000868154B03400AE671060020AC0300204D
:103A1000FF0F0000A5AA55A5FCFF010000C0005043
:103A20000400FA050CED00E0AC060020840600203E
:103A300042050020FFFFF7FF8A060020D803002080
:103A4000500500202405002094060020FFF0FFFF11
:103A5000FF0FFFFFFCFFFEFFFFFFFFFEA023D805C7
:103A6000826882B00192019B02210B430193019A6B
:103A7000826002B07047A023D805826882B00192AC
:103A8000019B01210B430193019A826002B07047B0
:103A900007B5A023D805826910210192019B0B4331
:103AA0000193019A826103480368002B00D0984774
:103AB00007BDC0460C01002007B5074B40211A681E
:103AC0000192019808430190019A1A60034B5868CB
:103AD000002800D0804707BD000200500C010020E4
:103AE00000487047001BB70030B5144B85B06A46DC
:103AF00023CB23C21868124910600D6A6C46280354
:103B000001D5104A00E0104A0D6A0D4B0020ED036C
:103B100011D4186A1D6AC1051B6AC80DA904C90E13
:103B20001D04023050430231AD0F03F099F9AA0091
:103B3000A15803F095F905B030BDC046A8FC0000BF
:103B40000002005000805101001BB7006A4B37B5DE
:103B50001968F0221004694C084318602568C023D6
:103B60009903294321602068654A664B0240226020
:103B70009C6880210194019D480305430195019AA9
:103B800080219A609C6889030194019D0D430195F1
:103B9000019A9A609C6880220194019DD4032C4371
:103BA0000194019D9D609A6880250192019C2A04E0
:103BB00022430192019CA025EA059C60D4680194EF
:103BC000019D284301900198D060D4684E4801942B
:103BD000019D28400190019CD460D5680195019811
:103BE0000143019101994948D160D4680194019D34
:103BF000284001900199464DD1605A690192019C7B
:103C0000254001950198586159690191019A9400E4
:103C1000A5080195019830245861D9690191019A4C
:103C2000C021A2430192019DDD61D8690190019AF2
:103C30008A430192019CDC61364B08249D68019502
:103C4000019820430190019A80209A6099680001B0
:103C50000191019D05430195019A9A60996880221E
:103C60000191019D11030D430195019D9D609A688D
:103C70000192019D8022120515430195019D9D60D1
:103C8000254B9D680195019D2C430194019C9C60EE
:103C90009D680195019C20430190019898609D6862
:103CA0000195019C21430191019999609868C02177
:103CB0000190019D19482A430192019A8D009A6052
:103CC000174B184A1C682040284318601C68C02005
:103CD000010122400A431A601D68134CC022900162
:103CE0002C4004431C601968104DC0240D40220272
:103CF00015431D6000203EBD080200500C0000501E
:103D0000FFFFCFFF00020050FFFFEFFFFFFFDFFFCD
:103D1000FFFFFFCF0000044000001440FCFCFFFF49
:103D200038000050F3F3FFFFCFCFFFFF3F3FFFFF0F
:103D30000E4B00B5C018FF21072814D803F07CF8FB
:103D4000120406080A0C0E1001210CE002210AE000
:103D5000032108E0042106E0052104E0062102E039
:103D6000072100E00021081C00BDC04600FEFFFF47
:103D700007B5FFF7DDFF072318400138062805D8EF
:103D800003F05AF806080A0C13191F00124B06E03C
:103D9000114B0BE0104B0FE00F4B13E00F4B9968EA
:103DA00001200191019A824311E00C4B9A68019223
:103DB00001980B4A0AE0094B98680A4A0190019859
:103DC00004E0064B9968084A01910198024001926B
:103DD000019A00209A600EBD0000044000001440CB
:103DE000FFFEFFFFFFFFFEFFFFFFFFFE07B5FFF730
:103DF0009FFF072318400138062805D803F01CF858
:103E00000F1B27333E4A5600374801218268019232
:103E1000019B0B430193019A0023826051E03248D9
:103E2000802182680192019B4A001A430192019B02
:103E30008360012345E02C48802283680193019927
:103E400053020B43019301990223816039E0264814
:103E500080238268019201995A040A4301920199D0
:103E6000032381602DE02148012183680193019A99
:103E70000A430192019B8360042322E01B488023B4
:103E80008268019201995A000A430192019905231F
:103E9000816016E01548802281680191019B5102E2
:103EA00019430191019B836006230AE00F48802398
:103EB0008268019201995A040A43019201990723E9
:103EC000816004200121034206D0094A043B1068A6
:103ED00099400143116005E0064A994010680B1CA7
:103EE0000343136000200EBD000004400000144096
:103EF0007C0014407C00044070B5061C0D1C081C9E
:103F0000FE21890503F048F90124002841D1301C25
:103F1000FFF70EFFFF283CD00024072839D802F015
:103F20008BFF0406080A0C17222D1B4C06E01A4EC4
:103F30000FE0194C18E0184E21E0184CE06803F02F
:103F400025FE291C03F01EFB03F03AF920611FE057
:103F5000124EB06903F01AFE291C03F013FB03F0A4
:103F60002FF9F06114E00D4C606A03F00FFE291C7C
:103F700003F008FB03F024F9A06209E0074E306B60
:103F800003F004FE291C03F0FDFA03F019F9706335
:103F90000024201C70BDC0460000044000001440F6
:103FA000F7B50C1CFFF7C4FE6F49071C201C03F07B
:103FB000E9FA03F005F98023051C590501208D421B
:103FC00000D9D0E0694A95422DD9290C281C8EB21F
:103FD00002F046FF80246302984201D90136B6B24E
:103FE000802041008E4221D92E0A290E301CCCB2ED
:103FF00002F036FF80256A02904201D90134E4B212
:1040000000250120011C2B18A940DDB2A142F8DDDA
:104010006A1E9040C4B20020102C00D9A3E03502E3
:104020008026760003E00226041C00E00124311CF7
:10403000281C02F015FF211C02F012FF83B207209A
:104040000740013E87420AD80125BD40C0210D42EC
:1040500012D13022154206D10C20054201D1444D27
:1040600002E0434D09E0434D2968FF220191019888
:1040700016409043021C07E03E4D2968F6B20191BC
:1040800032023D48019E064016430196019E601E85
:104090002E600F2812D802F0CFFE080A110C111161
:1040A000110E1111111111111110042406E0002438
:1040B00004E0012402E0022400E00324013B781E16
:1040C0009BB2062806D8072702F0B6FE1113151773
:1040D00023313F00264E072570682C40019001993E
:1040E000A9430C430194019C7460F3603AE0204DB5
:1040F00010E01F4D1CE01E4E28E01E493C404A685F
:1041000001920198B84304430194019C4C60CB6038
:1041100028E0184D696827400191019A70203F01FD
:1041200082433A430192019E6E60AB611AE0114DE9
:10413000696827400191019C104A3F0214403C43AA
:104140000194019868606B620CE00A4E7568274024
:10415000019539030A4C019F27400F430197019AAB
:10416000726033630020FEBD001B374BFFFF010070
:104170000000044000001440FF00FFFFFFF8FFFFB5
:10418000FF8FFFFF13B50C1CFFF7D2FD012307289B
:1041900047D802F051FE0406141C1E272B37224B71
:1041A00018E0214B996801910198002C1CD08022C5
:1041B000D2000243019201989860002331E01A4B2B
:1041C000986801900198002C16D1184A24E0164BEB
:1041D00019E0174B98680190019A0420002CE8D14F
:1041E00082431AE0124BDDE7124A15E0104B9A6841
:1041F00001920198002C02D08024E202D9E70B4AF8
:104200000240D7E70A4B996801910198002C02D02F
:104210008024E204CDE7084A0240019201999960A6
:10422000231C181C16BDC04600000440FFFFFBFF06
:1042300000001440FFFBFFFFFFFFFFFB030A054ADE
:1042400099008B181A68C0B2012181408A4300206E
:104250001A60704730000050030A0D4A10B59C01E7
:10426000A318C0B21C6842000320904084431C6025
:10427000022903D0032906D0012907D11C689140E7
:104280002143196002E0196808431860002010BD3E
:1042900000400050094AC3B2000A80018018012280
:1042A000002904D101689A4091430B1C03E0016886
:1042B0009A40131C0B4303600120704708400050D4
:1042C000030A054A99018B181968C0B2C140081C3D
:1042D000012210407047C0461040005070B5174C86
:1042E000174D23695807460F042E02D8012E04D01B
:1042F00000E00326B300E85818E0226A1104880F92
:104300008642B641226A7342C61A120301D50D4B8A
:1043100000E00D4B216A226AC805C00D9104C90E48
:1043200002305843023102F09BFDF040A46922079D
:10433000110F013102F094FD286170BD00020050A0
:104340001800002000805101001BB70070470000DA
:10435000094B0A4882B000930190009B009A0849DB
:10436000106808431860019B019A04211068884373
:104370001860002002B07047DC400050D840005068
:104380000400040000207047024B04221860024819
:10439000026070471401002000E100E008B5044B02
:1043A00004481A6A01681A620348884708BDC04673
:1043B000C0400050140100200203000070470000BC
:1043C00010B5194C236BDA070CD5184A116800296F
:1043D00001D050688847164807220368012193439B
:1043E0000B430360206B82070CD5104A1369002B26
:1043F00001D0906898470E480721026802238A433B
:104400001A430260246B62070CD508484269002AEF
:1044100001D0C0689047064B07211C6804208C43DC
:1044200004431C6010BDC04600000E40180100206F
:1044300030000E40034B10B51888034B00219B68D9
:10444000984710BDC4010020D0FC000070B50500E5
:10445000094B01219C68094B1888A047084B094A61
:104460001B78DBB2D15C084B29401888002900D0AA
:104470000121A04770BDC046D0FC0000C40100204F
:1044800090060020040000209C030020F0B5C14CE1
:1044900085B023780133DBB22370207801384128BE
:1044A00001D900F02DFF02F0D1FC42006B00B400F6
:1044B000C3002B0743032B072B072B07BD03C503A3
:1044C0002B072C062B0761062B072B072B072B0727
:1044D0002B072B072B072B072B0770062B072B0708
:1044E0002B072B07B706E806D306E806D506E8062D
:1044F000D706E806D906E806DB06E806DD06E80684
:10450000DF06C9062B072B072B072B07D106E8066A
:10451000D306E806D506E806D706E806D906E80673
:10452000DB06E806DD06E806DF06E306EB0600220A
:10453000994B9A481A709A4B1A700178994B0F2927
:1045400004D91C689849214019600270974A127872
:10455000002A03D11968944A0A4003E080211A68AE
:1045600049050A431A60924B1B78012B01D800F0D1
:10457000C7FE00238F4A13808F4A138000F0C0FECD
:104580000F218A4B1A788A43702A04D18549864ABA
:10459000086802400A608948027F52B2002A01DBA3
:1045A00000F0AEFE1A78FF2A01D000F0A9FE5A787A
:1045B000FB2A01D000F0A4FE9A78002A01D000F076
:1045C0009FFEDA78002A01D000F09AFE1A79002ABC
:1045D00001D000F095FE5A79002A01D000F090FE3B
:1045E0009C79E4B2002C01D000F08AFEF0237449DB
:1045F0000A689A430300FE330A601C700300FD330F
:104600001C700300FC331C700300FB331C7000F0B3
:1046100077FE6A4B5B7F1B0704D4624A624B1168CA
:104620000B4013600F22674B1A705A7000F068FE3F
:104630005E49624A08780B00FF2800D0FEE1107F37
:1046400040B2002800DB9FE04978C9B2FD2900D9BB
:10465000C0E0FC2900D3F2E07F2900D190E0FB29E3
:1046600000D091E099783E2900D08DE0504909783A
:10467000890700D188E05449D8780D7A0E00854228
:1046800000D02BE2487A1979884200D026E2B17A2C
:1046900000915F79B94200D020E2F67A01969E79C6
:1046A000019FB74200D019E2062780213C4EC90085
:1046B0003770464F3E680E4380213E60404E4900B1
:1046C00037680F433760DF79002F16D11B7ADBB2D2
:1046D000002B12D1326810398A433260374A1100F8
:1046E000FE310B701100FD310B701100FB32FC31FB
:1046F0000B7013702E4A1370F0E12C4EF379002BDF
:104700000DD0F379DBB25374337A2026DBB2937485
:10471000537F334353772A4A6036136809E0337A6C
:104720002026DBB25370537FB3435377244AB61924
:10473000136833431360264EAB093C33F25C214BC4
:1047400000991A703F221540755D5D708508755D92
:1047500000019D700D0940191040305C8900D8702F
:104760000198800909181140715C197101990A407A
:104770008021B25C89005A71114A13680B4307E02B
:104780009A783E2A00D129E1064A1168064B0B406F
:104790001360A3E1F4050020E80400208D0500204B
:1047A0003005002084060020FFFFFFEFFD040020FD
:1047B0002405002088060020AC060020D803002035
:1047C00028050020120000209905002094060020F2
:1047D000ECFC0000C448C5490578012D2AD00D68BD
:1047E0002D0402D55D78ED0705D40D682D0421D484
:1047F0005D78ED071ED4007802281BD19E78DF7803
:104800003606B44618793E045D79000266443618CF
:10481000B748B84F76190660387A0506787A0004EA
:104820002818BD7A2D024019FD7A4019B24D286032
:10483000864204D20A68B14B13400B604EE1B04887
:10484000A9490568AD052AD516009D78FA36EDB25E
:1048500035701600DD78FB36EDB2357016001D7927
:10486000FC36EDB2357016005D79FD36EDB235706F
:1048700016009D79FE36EDB23570DD79A14EEDB2B0
:1048800035701600F936357006689F4D3540802624
:1048900005600568F6003543056001250D701500BB
:1048A000FA352E789D78AE421CD11500FB35DE78A6
:1048B0002D78AE4216D11500FC351E792D78AE420A
:1048C00010D11500FD355E792D78AE420AD1150064
:1048D000FE359E792D78AE4204D18A4DDE792D7851
:1048E000AE4204D00D78012DAED0022203E00A784A
:1048F000002A01D101320A7008787C4A012800D1CF
:1049000043E70978022900D93FE71168090402D575
:104910005978C90707D41168090400D535E75978D3
:10492000C90700D531E706218020784AC000117000
:104930007749784E0A683700024380200A60704940
:1049400040000A68FA3702430A603F786948BC466B
:10495000057A9F78AA093832BC4521D1DF78BC4658
:104960003700FB373F78BC451AD11F79BC4637006A
:10497000FC373F78BC4513D15F79BC463700FD3723
:104980003F78BC450CD19F793300FE331B789F42A2
:1049900006D120260B6833430B6004231A43D2B29E
:1049A0005D495E4B8A5C1A703F2215404D5D5D701B
:1049B000457AAE088E5D2D019E70877A3E09AD194D
:1049C00015404D5DDD70C67AB800B509401910403C
:1049D0003240085C8A5C18715A717FE0454AD97888
:1049E000107A884200D0CFE61979507A884200D0F8
:1049F000CAE65979907A884200D0C5E69979D27A88
:104A00008A4200D0C0E6464A11781000072902D930
:104A10000021444D07E0022280213C4BC9001A705E
:104A20003B4A1368AAE60278073A914256DACA1D51
:104A30009A5CD2B26A540131C9B2F4E70025202051
:104A400032490D70567F3040A8421CD01E78507CF1
:104A5000864204D02E4B1B689B0527D43EE0587835
:104A6000927C9042F6D102222E4E0A702A002C4DE2
:104A7000287802388242EDDA901C185CC0B2B0543B
:104A80000132D2B2F4E71D7852789542E2D1022287
:104A90000A700200224D234E287801388242D9DA6A
:104AA000571CD85DC0B2B054FAB2F5E71E4B1B8854
:104AB000002B13D00B78022B10D101331B4A0B7043
:104AC000137815489B09C31814491B7F0B703F23AB
:104AD00012781340C35C4B709A238B702378013398
:104AE000DBB2237000F00CFC2405002084060020BB
:104AF000C001002099050020A8010020FFFFFFEF62
:104B000028050020F3050020FFFDFFFF30050020F1
:104B100094060020D8030020ECFC000012000020C6
:104B20008D050020E804002088060020B006002043
:104B3000B74B1888B74BDB6800939847002804D020
:104B4000B54AB64B11680B401360B54B1A68D205D5
:104B500017D51968B34A0A401A602D2203AB1A70A0
:104B60000C325A70AC4B1B68DB0000D4C8E3AE4B70
:104B70001B7FDB0700D4C3E3022103A8FCF712FB71
:104B8000BEE3AA4B1B78FF2B00D1B9E38022A24CD5
:104B900052012368A44903A8134219D02268A44BE8
:104BA00013402360CB7C002B0ED14B7F9B0607D597
:104BB0009C2303704A7C5D3B13409E4AD35C2AE0F1
:104BC000A3230370093326E0A6230370503B22E0A1
:104BD000236813432360CB7C002B0ED14B7F9B06B5
:104BE00005D580228B7C92009B188D7C0AE0802268
:104BF0004B7892009B184D7804E08022CB7C920089
:104C0000CD7C9B18C23AFF3A2A409B09894D9BB242
:104C1000EB5C0370AB5C43702368DB0000D46FE394
:104C20000B7FA6E77C4B1B68DB0500D468E30422FE
:104C3000814BA8E27C4A784E137F9B0700D4E7E1C2
:104C40003368DB0000D45BE310210320744C7B4D00
:104C5000236800958B43236023682B402360784BA7
:104C600019788143EC2908D11978053081438020D7
:104C7000197021680001014321601878E038072885
:104C800000D93DE302F0E2F82B003C033C033C0377
:104C900012000E0008000A00002100E0012101318D
:104CA000C9B200E000210131C9B200E00021507F0B
:104CB000644F80060BD53878052803D91025206865
:104CC0002843206038780138C0B2387008E038785E
:104CD000042805D9102720683843206000E000210F
:104CE00010202768074000D197E1107F40B20028CC
:104CF00000DB8DE1534806780190092E1CD94B4EFC
:104D00005148377A737A3F02FF18504BBFB29C4626
:104D100089003300FF2F00D19AE002D8002F17D06E
:104D20006BE180267600B74200D1D4E00222FF3248
:104D3000974200D128E160E13C4D0120AC46654638
:104D40001E5CC71DF6B20130EE550828F7D1D6E734
:104D5000206800051CD5B07AF67A0130F6B21654F8
:104D6000987A1E7B0230F6B21654987A5E7B033036
:104D7000F6B21654987A9E7B0430F6B2165480260A
:104D800020687601304320602068009D0540256042
:104D90003F25987A274C0130105C80092030091893
:104DA000C9B22948615C0170997A0131515C29408E
:104DB000615C4170997A0231515C8908615C817053
:104DC000997A0231515C9E7A0F010336965D310962
:104DD00079182940615CC170997A0331515C9E7ADF
:104DE0008F000436965DB10979182940615C017124
:104DF0009B7A0433D35C1D40635D4371019B1A7839
:104E0000124B082A01D8042200E006221A705BE047
:104E1000A8030020D0FC000084060020FFFFFFEF65
:104E200028050020FFFEFFFFD8030020FD0400201E
:104E3000FFEFFFFFECFC000000E100E0FFF7FFFFE9
:104E4000E80400208D05002012000020300500201D
:104E5000B77A502F3FD8B37ADC4ADD4CD3185B7851
:104E60009B092033C918C9B2635C3F210370B37A30
:104E7000D3185B780B40E35C4370B37AD3189B780C
:104E80009B08E35C8370B37AB77AD3189B781D01D3
:104E9000D319DB781B09EB180B40E35CC370B37AC2
:104EA000B77AD318DB789D00D3191B799B09EB18CF
:104EB0000B40E35C0371B37AD21813791940635C39
:104EC00043716246062313708021C24AC9001368E9
:104ED0000B43136014E29E7A1E2E55D820680005FD
:104EE0001CD5987ADE7AC830F6B21654987A1E7BB2
:104EF000C930F6B21654987A5E7BCA30F6B21654B0
:104F0000987A9E7BCB30F6B21654802620687601C4
:104F1000304320602068009D054025603F25987A39
:104F2000AB4CC830105C800920300918C9B2AA48BF
:104F3000615C0170997AC831515C2940615C4170B3
:104F4000997AC931515C8908615C8170997AC9315B
:104F5000515C9E7A0F01CA36965D31097918294055
:104F6000615CC170997ACA31515C9E7A8F00CB36F0
:104F7000965DB10979182940615C01719B7ACB3348
:104F8000D35C1D40635D9BE79A7A1E2A35D89A7AD6
:104F9000924CD2B2A25C8E4D920920328918C9B2CD
:104FA0006A5C3F2102709A7AD2B2A25C0A40AA5C83
:104FB00042709A7A0132A25C9208AA5C82709A7A54
:104FC0000132A25C9E7A17010236A65D3209BA1838
:104FD0000A40AA5CC2709A7A0232A25C9E7A97005A
:104FE0000336A65DB209BA180A40AA5C02719B7A20
:104FF0000333E35C19406B5C62E72031744BC9B248
:105000005B5C0370AC2343708370C370037157E71C
:105010003268734B1340336072E1022171480170B2
:105020001C786D496A48E4070ED56F4A9278C72A02
:1050300007D85A78654CA25C92090A705B78E25CEA
:1050400055E00F704F7055E01C78E02C47D13F279A
:10505000654A664BD47801341C5DA4090C70D47881
:1050600001341C5D3C404C700C78045D0C704C7835
:10507000045D4C70D47802341C5DA4088C70D47824
:1050800002341C5DD6782401A446302465460336DC
:105090009E5D2C403609A419CC708C78045D8C7010
:1050A000CC78045DCC70D47803341C5DD678A40031
:1050B000A4463C24654604369E5D2C40B609A419DE
:1050C0000C71D27804329B5C464A1F404F710B79B9
:1050D000C35C0B714B79C35C4B710623F3E65C78C0
:1050E0000134145DA4090C705B780133D25C3F235A
:1050F00013404B700B78C35C0B704B78C35C4B70E8
:10510000FEE03B4C3B4B2088DE68B0473A4D220026
:10511000002803D02968324B0B402B602B682D4CA4
:10512000DB000DD52F4B1978002909D019782A48B2
:10513000C9B2FCF737F82268304B1340236007E010
:105140001088B047002803D02A68254B13402B60F5
:1051500023685B0500D4D3E08022236892001343C8
:1051600023602268264B13402360C9E0254B1A6850
:10517000D20400D4C4E080211A6889010A431A606D
:105180001968214A0A401A60BAE000210800FBF7BA
:105190004FFA04221D4B1A60174A13681B0200D4F1
:1051A000AEE0802310685B00184000D0A8E0184BE8
:1051B0001B78012B00D9A3E013681B0100D49FE0EA
:1051C0000300144A0521FBF763F999E099050020D3
:1051D000ECFC000094060020120000205505002081
:1051E000FFFFFFEF30050020FD040020D803002062
:1051F000A8030020D0FC000084060020FFFDFFFF74
:10520000FFFBFFFF28050020FFEFFFFF00E100E0AC
:10521000240500208D4400003A4B1B681B0136D545
:10522000394A13780133DBB21370012213402ED1B7
:10523000364A11780B2909D9137007E0FFF7FAF8FD
:10524000324A13780133DBB2137059E001200CE0CD
:1052500002200AE0042008E0082006E0102004E014
:10526000202002E0402000E08020FFF7EFF847E038
:10527000264A13780133DBB21370FFF7DBF83FE007
:10528000234B01211888234B9B6800939847224B9E
:105290001A6880235B00134003D11A4A1268120770
:1052A00000D41D231D4923700A681D4BD2B25A70C9
:1052B0000A681C48120AD2B2DA700A68120CD2B21A
:1052C0005A710A681900120EDA71028892B2002A25
:1052D00010D003885B080133DBB24B724B7A5BB2B0
:1052E000002B01DA7F234B720F4B1B885B08DBB26C
:1052F000CB7201E05A72DA7200210800FBF798F9CC
:1053000005B0F0BD8406002030010020900600208A
:105310009C030020D0FC00009406002050050020D3
:105320000400002088060020AC060020F0B516001E
:1053300085B01D000AAB040018880BAB1B7835360E
:1053400001935E4B9E5DF7B2160084369E5DF6B209
:10535000029616008C369E5DF6B2B4467EB2002EE2
:1053600000DAA8E0564E3688314200D1A3E00A2682
:10537000029971430291F9062BD5029BAB4225D8C5
:10538000019B0821002B11D04E4B0F4207D01B6907
:10539000200001939847002D00D08CE077E05B69F6
:1053A000200001939847002D75D084E0464B39408A
:1053B0009B68019305D0012120009847002D72D0F1
:1053C00079E020009847002D75D16EE0002D52D075
:1053D00071E0B9061CD50199002915D03B4A7033FC
:1053E00012681E7802F0D2FBF6B2071C300002F001
:1053F000CDFB011C381C01F0FBFE324D011CEB689B
:1054000020000193984756E07332C0B2985452E09E
:105410007B0650D563465E43029BAB4203D05B00E4
:105420009B19AB4225DC019B0822002B10D0254B99
:10543000174206D01B69200003939847002D1FD107
:1054400025E05B69200003939847002D23D017E0E7
:105450001D4B9B680393174205D0012120009847FC
:10546000002D0DD11FE0019920009847002D1CD080
:1054700006E0002D04D1019A0823002A05D110E08E
:10548000029B9E19AE4216D1F5E71F4203D00D4B89
:1054900020005B6902E020000A4B1B6901939847DA
:1054A00009E01F4201D0002100E00121064B20004D
:1054B0009B680193984705B0F0BDC046D803002013
:1054C00042050020B8FC0000D0FC0000840600204B
:1054D000F7B51D00464B0E00040019001000723194
:1054E000353009787B321F5C3E30185C9A5CFFB225
:1054F000D2B201927AB23140C0B2002A77DB3D4A83
:105500001288324094467A0727D56246002A51D144
:10551000002906D071331978374B1B88994200D285
:105520000198002D59D002F031FB03F0BFFF00229B
:10553000324B02F095FE02000B000020304903F0D0
:105540001FFC04F007F82F4D011CEB6820000193AD
:1055500098472B692000019332E06246002A29D047
:10556000002906D071331978234B1B88994200D249
:105570000198002D15D002F009FB03F097FF0022DF
:105580001E4B02F06DFE0B0002001D49002003F0CF
:10559000F7FB03F0DFFF1B4B011CDB6820000193CE
:1055A000984750231F4222D1002D16D0154B2000C2
:1055B0001B6904E0002D05D02000124B5B690193AC
:1055C000984714E0104B29009B68200001939847EE
:1055D0000E4A1378B343137009E00B4B01219B680B
:1055E000200001939847094A13781E431670F7BDAF
:1055F000D8030020420500208806002000E06F400C
:105600000000F03FB8FC0000D0FC000026050020A0
:10561000F0B552B285B0050001911E00002A00DBF2
:10562000BEE06B469F885F4B1B88002B22D0002476
:105630007F0803D00134A4B2082CF9D1023CA4B2F3
:10564000002E05D0584B28005B690293984705E06F
:10565000564B31009B68280002939847544A554B9B
:10566000116864000B4013600022534B5A700233E0
:105670007A1CE252514A138803929BB2002B05D048
:105680004B4B1B689B0000D48AE000237F0803D0AB
:1056900001339BB2082BF9D1023B9BB2484A5B0015
:1056A00002931288019B444F1A4267D0404C454BED
:1056B0002268520501D5A23300E0A33318780A23EB
:1056C0005843029BBA1CD35A002B23D10121029BC1
:1056D0002800D152002E04D0334B1B690293984707
:1056E00003E0324B9B68029398477B78002B57D19D
:1056F000344B01991A00A03212780A4250D0C021CE
:105700002268C9050A4322606A461279A1337A7079
:105710001B7830E098420ED901339DB2029B0A21DA
:10572000D55201F09DFB80B2854239D12268264BCB
:105730001340236034E0984232D1029B0130D052B2
:10574000002E05D0184B28005B690293984705E0AE
:10575000164B31009B682800029398477B78019A8A
:1057600013421DD02268194B1340236000237B7025
:10577000039B1B885B08039A138011E0002E05D061
:10578000094B28005B690193984705E0074B3100FE
:105790009B682800019398470023029A0237BB5266
:1057A00005B0F0BDAC060020B8FC0000D0FC000045
:1057B00084060020FFFFFF9F3001002088060020A4
:1057C00042050020D8030020FFFFFFBFFFFFFFDFDF
:1057D000F0B5534C87B02368DB0505D50023514A4B
:1057E00005211800FAF754FE4F4D504A2B6801333B
:1057F0002B601378002B03D01378013BDBB21370BE
:10580000002213004A49885C002801D00133DBB232
:105810000132642AF7D1474A1370474B1A78002A9D
:105820000FD01A78FF2A0CD01A78002A03D01A78E1
:10583000013AD2B21A701B78DBB2002B01D13F4A79
:1058400093763F4B1A78002A0FD01A78FF2A0CD093
:105850001A78002A03D01A78013AD2B21A701B784B
:10586000DBB2002B01D1354A9377364A364913888B
:105870008B4203D8138801339BB21380334A1388B9
:105880008B4203D8138801339BB21380304EB37B15
:105890000133DBB25F2B01D8B37306E00023802213
:1058A000B37323689200134323602A4C2368DB05FB
:1058B00000D538E3284B1B78012B00D933E32B6844
:1058C000DBB2002B05D1254B254A1B8801339BB247
:1058D0001380244A13680133136023689B0349D55E
:1058E000214E0021F3680393204B1888039B9847AF
:1058F0001F4F039B3888002198471C4A2368108853
:105900005B0303D52B689B0605D502E02B681B06BD
:1059100001D5746900E03469A0473888A04702E3E4
:10592000940600208D4400009005002068060020A9
:1059300000060020B00600208F060020D8030020BB
:10594000B4030020B8030020FDFF00004405002040
:10595000300100208406002024050020420500209C
:105960008A060020B0030020B8FC0000B40100202B
:10597000CC02002032692368CA495340CA4A5B05F9
:1059800005D50B8801339BB2138023683361C74B65
:1059900071331B78002B07D0C54B1B88002B03D01D
:1059A0000B8801339BB2138010880B8898423AD041
:1059B0000B889BB21380BF4B00221888012319006B
:1059C000FFF786FDBC4B0221188801231A00FFF760
:1059D0007FFDBA4B0222188804210123FFF778FDCE
:1059E000B74B0622188840210023FFF771FDB54B05
:1059F0000322188808210023FFF76AFDB24B042216
:105A0000188810210023FFF763FDB04B052218888A
:105A100020210023FFF75CFDAD4B07221888802171
:105A20000023FFF755FD738B0A2401339BB20393C8
:105A30006B469B89B08A7383B38BF18A01339BB227
:105A400004936B461B8A328BB383F38B358C013303
:105A50009BB205936B469B8A0130F383738C0131B3
:105A600001339BB273849C46B38C01320135013300
:105A70008E4F80B289B292B2ADB29BB2B082F18247
:105A800032833584B38470373F786743874CBD4297
:105A900001DD00253584683425780A246C43A04252
:105AA00002DD00248B48848280480A250400693482
:105AB00024786C43A14202DD00248649CC82010097
:105AC0006A310C780A216143824C8A4201DD00224E
:105AD000228302006B3211780A224A4303999142D1
:105AE00001DD0022628302006C3211780A224A43EF
:105AF0000499914201DD0022A28302006D321178E7
:105B00000A224A430599914201DD0022E283020004
:105B10006E3211780A224A43944501DD00226284E4
:105B200002006F3211780A224A43934201DD0023BA
:105B3000A384030035331A7820231A4222D10200AD
:105B4000363212781A421DD10200373212781A42C8
:105B500018D10200383212781A4213D102003932B9
:105B600012781A420ED102003A3212781A4209D142
:105B700002003B3212781A4204D102003C32127801
:105B80001A4214D0E31DDB7F002B02D0238C023B92
:105B90002384228C022A02D80021E31DD977703099
:105BA0000378013B934202DC0122E31DDA770126F0
:105BB0000025404AA38A10880196228C3100009269
:105BC0000022FFF7B3FB3C4AE38A10880196228C3F
:105BD000022100923200FFF7A9FB384A238B10887C
:105BE0000196228C042100920222FFF79FFB344A87
:105BF000638C10880195228C402100920622FFF7C9
:105C000095FB304A638B10880195228C0821009205
:105C10000322FFF78BFB2C4AA38B10880195228C63
:105C2000102100920422FFF781FB284AE38B1088A1
:105C30000195228C202100920522FFF777FB244F4B
:105C4000A38C38880195228C802100920722FFF7CF
:105C50006DFB164C0421230037331A78174BD2B250
:105C600018883300FFF7D4FC230038331A78154B1B
:105C7000D2B2188808212B00FFF7CAFC2300393361
:105C80001A78114BD2B2188810212B00FFF7C0FCF4
:105C900023003A331A780D4BD2B2188820212B00FA
:105CA0001AE0C046420500208A060020D8030020E2
:105CB00088060020B4010020CC020020A6030020AA
:105CC000A2030020D0020020B0010020A403002085
:105CD000B801002030010020FFF79AFC23003B337D
:105CE0001A78924BD2B2188840212B00FFF790FC13
:105CF00023003C331A783888D2B22B008021FFF77A
:105D000087FC8B4B1A882300AA4200D0A4E0220013
:105D100061321278AA4204D1220062321278AA4279
:105D200047D00125834A84481268039202682A42B8
:105D30003FD1026892073CD48021804A89051468CB
:105D40000C4036D11F00613739788C460F216646EA
:105D50003140039E31400CD0016865330D437849D2
:105D600005600C851B7877482A3103800C703B78DE
:105D700013E0704C26681C0062342778360A3E42D5
:105D800017D006686533354305606D486D4D018554
:105D90001B782A302B80017023785BB2002B04DA49
:105DA00080211368C9000B4302E01168664B0B4069
:105DB0001360664B1A0063321278002A04D11A006D
:105DC00064321278002A47D05A4A5B48126803921C
:105DD0000268D20740D4022502682A423CD18021C1
:105DE000564A890514680C4036D11F00633739784C
:105DF0008C460F2166463140039E31400CD001682D
:105E000065330D434E4905600C851B784D482A319A
:105E100003800C703B7813E0464C26681C00643409
:105E20002778360A3E4217D0066865333543056049
:105E30004348444D01851B782A302B80017023781C
:105E40005BB2002B04DA80211368C9000B4302E027
:105E500011683D4B0B401360374C2368DB072DD591
:105E60003A4B603319783A4BCDB21888394BDB681E
:105E700003939847324B002804D0E92169431A8DD7
:105E800091420ED21A0000212B322A3311701A7857
:105E9000322A04D901222368934323600EE00132A1
:105EA0000BE0190001322B311A850A780132D2B287
:105EB0000A700A2A02D900222A331A7023689B0723
:105EC0002FD5224B60331A78234BD5B21888214B3B
:105ED000DB68039398471A4B002804D0E9226A43F1
:105EE000198D8A420FD21A0000212B322A331170E9
:105EF0001A78322A04D9022223689343236010E0DF
:105F000001321A700DE018002B3002780132D2B243
:105F100002700A2A03D91A0000202A3210700131B7
:105F20001985FBF781FC07B0F0BDC046A203002035
:105F300088060020500500209406002084060020DA
:105F400030010020AC060020FFFBFFFFD80300203B
:105F5000B2010020D0FC00009E030020B54AF0B53D
:105F60001100B54C2C312368B44F013323600B78FA
:105F700087B001330B703B881600002B03D03B88A1
:105F8000013B9BB23B80AE4B1A88002A03D01A8893
:105F9000013A92B21A808022AA49520008680191FF
:105FA000024001D000F0BEFE0425A749086828423F
:105FB0001CD0A6480280326B002A11D10868A84381
:105FC000086008686D19284210D00868A843086066
:105FD0009F48073D417F694041779E490A7005E02F
:105FE0009D490988002901D1013A3263974D9A48A9
:105FF00029880288914200D192E01021974A1170BD
:10600000934A9049313212780968D2B2890054D447
:106010009349D208096800928C460C2162461140CF
:10602000009A114202D02A8892B20280874A8021C7
:10603000128884489446884AC9031588844A0068AF
:10604000AC4529D9D278084201D0520800E0D2B23A
:10605000844909688A4230D87D4A7F499578088802
:10606000854206D9413215780888854201D91278CF
:106070000A80794976480A88013292B20A80827889
:106080000D885208AA4203D98278520801320A8048
:106090000021744A116010E01279084201D05208C0
:1060A00000E0D2B26F490868824206D86A48028886
:1060B000013A92B2028000220A601A88664B002AD6
:1060C00003D0002261491A800A801D88ADB2002DDC
:1060D00006D080215B4A490313680B4313601FE01D
:1060E000614B29009B680093604B1888009B984780
:1060F0005F4B29001888009B9847FE215D4B89055E
:1061000018885D4BDB68009398474E4A5B4B1168DB
:106110000B4013605A4B1D605A4B1D605A4B1D605B
:1061200033002C331A78322A64D98021454A490039
:10613000106801405ED11970454B5448DD7A002D3E
:1061400055D0DD7A00950578AC46009DAC454ED91A
:1061500004205D7F28401ED080251068ED03284371
:1061600010603A4A0F25118032003432117032002B
:1061700035321170587B3A4A2840103010605B7BF2
:106180001068AB431B011B1803201360FAF750FA89
:106190000A233B802EE02025DB7E2B420FD03300EC
:1061A00036331B78042B0AD88021284B49031880EA
:1061B000136819431160244A13682B431360244B5E
:1061C000DB7E5B0616D5330036331B78042B11D9E2
:1061D000002280211D4B49031A801A4A13680B4381
:1061E00020211360184A13680B43136002E0037800
:1061F0000133037020680138172801D900F0FDFB36
:1062000000F024FE4600FB03FB034D007B009800DA
:1062100098009800C50016021F021F021F024F02BD
:106220000402B502B502B502B502B502B502B50267
:10623000B502E60230010020DC040020AE0100209F
:106240008C0600208406002094060020AC06002066
:10625000D803002046050020880600209A0300206D
:1062600050050020B0030020D0FC0000B601002043
:10627000C8010020A4010020B8FC0000FFFFEFFFD0
:1062800048050020F805002020050020AF0600206A
:10629000C74B1B88312B00D9B4E3042323600124AE
:1062A000C44B31331B78234211D0FE21C24B8905E8
:1062B0001888C24BDB6800939847FF21C04A536A95
:1062C0000593059B8B4323430593059B5362340041
:1062D000002336342370BB4B1B685B0200D491E370
:1062E000B94B1888B94BDB6800939847002800D158
:1062F00088E323780133237084E3B24B1B685B028D
:106300000CD5B14B1888B14BDB6800939847002837
:1063100004D0320036321378013313700121A54BBB
:1063200031331B780B4200D16CE30720A84A136875
:10633000834382E19F4B31331B78DB0700D49CE120
:106340009F4A136B9E49DB07FBD5A248A24C0388EA
:106350009BB25A1C92B202800A685B001205120DB1
:106360001A530388632B01D9002303800720984A1E
:106370001368834306380343136080220B6A1201BB
:106380000593059B13430593059B0B6275E1894BB0
:106390001A00313212780093D30703D5884B1B6B58
:1063A000DB07FBD58B48038802889BB292B2511C55
:1063B00089B20180824952000C6887492405240D66
:1063C000545202883387632A01D9002202805A007E
:1063D0008F5A002230001400009D3A300270A6351A
:1063E0002878013090420CDB002B02D0013B9BB29D
:1063F00000E063235800085A01323F18D2B201244A
:10640000EEE7002C03D0338733003A331A700323AE
:106410005F43009B7F10A5331A78002A01D01B78B8
:106420005F436E4A1188138802334B43DF1B009B86
:1064300032331B7801927B43D90FCB1868495B102C
:106440000B601388132B05D8142310880A681B1AB5
:1064500053430B60634C624D23682821FB18236073
:10646000009B3333187823682A685843029200F05F
:1064700081FD029B0395C3182B6022685A4B9A42F8
:1064800000DD23602368002B01DA00232360574DD1
:10649000009B2868524C34331B78381A22685843C2
:1064A0000A21029200F066FD029BC31823602F6050
:1064B00022684F4B9A4200DD23602368002B01DAEB
:1064C00000232360019B3F4C1B88002B51D080236D
:1064D0002768DB001F4080232168DB053B4A454DD0
:1064E0001940002F0AD09768002902D0288800217F
:1064F00014E0414B1888B847288812E000290BD0D7
:106500009368390002933C4B1888029B984728886F
:106510000121029B984706E097682888B847364BC8
:1065200018880121B847009B234F31331B78234D36
:10653000DB0708D5039B186801F0E0FA02F0B6FF0C
:1065400000222E4B06E0019B188880B202F06CFFFF
:1065500000222B4B01F084FE0B0002002949002091
:1065600002F00EFC02F0F6FFEB68011C0093388885
:10657000984723685B020CD5134B1888134BDB68D4
:1065800000939847002804D0320036321378013344
:106590001370FF220A4B5B6A0593059B9343DF3A16
:1065A00013430593059A064B5A620022164BDCE012
:1065B000AC060020D8030020A4010020B8FC000095
:1065C00000000E4084060020A8030020D0FC00003C
:1065D00030000E40CE020020D202002088060020AB
:1065E000B406002048050020400D030020050020CF
:1065F000FFFF0000B6010020C8010020E0FFEF40CF
:1066000000E06F400000F03F94050020B54B1B6890
:106610005B0200D4F6E1B44B1888B44BDB680093FE
:106620009847002804D032003632137801331370B3
:106630000721AF4A13688B4306390B431360AD4AF9
:10664000BCE0AC490B6BAB4ADB07FBD55369AA48EE
:106650001B0501681B0D5B1803600720A4490B682C
:106660008343063803430B608021136A09010593B5
:10667000059B0B430593059B13629A4B1B685B02BA
:1066800000D4BFE1984B1888984BDB68009398477B
:10669000002800D1B6E1320036321378013313708E
:1066A000B0E1944A136B934DDB07FBD56B699249BC
:1066B0001B050A681B0D9B180B6033003B331878D1
:1066C000421C1A700F230A6803405B00F3189210F3
:1066D0009A87A02100238C461A00180037008749AA
:1066E0003C37DF5B303109780097674601317943E9
:1066F000009F8F4201DD013292B2142A08D98049ED
:10670000804F0880804908808049086080490F8058
:106710000233202BE2D1734B1A688023DB03134032
:1067200017D0714B1888714BDB680093984700288D
:1067300004D032003632137801331370FF226B6AB3
:106740000593059B9343EF3A13430593059B6B62B7
:1067500009E0704A1168704A914204DC6A4A128862
:10676000632A00D8236000226C4B1A604AE15D4B1B
:106770001B685B0200D445E15B4B18885B4BDB6810
:1067800000939847002804D0320036321378013342
:10679000137058490B6B574ADB07FBD53000236851
:1067A0001169103B09055C305B00090D1952072087
:1067B0004F490B688343063803430B608021136AFB
:1067C00009010593059B0B430593059B136219E192
:1067D000444B1B685B0200D405E13200343213786D
:1067E000312B01D801331370330034331B78322B33
:1067F0000CD1424B5A7F04231340434A01D010234B
:106800005B4213803300332234331A700022444B2E
:10681000364D1A70344B1888EB680093984700285F
:1068200004D032003632137801331370314A136BBF
:10683000DB07FCD531002F4A23681269103B120593
:106840005B005C31120D5A522C4B1B7BDBB2002BD0
:1068500000D0B4E00A88488890421BD2310001334E
:106860005E31881E008884460888844504D301333D
:10687000DBB20231092BF4D13100013B5C31488A93
:106880005B005B5A1218D21A92B209E0023382B24C
:10689000102B05D0C81840889042F7D2101CF5E79D
:1068A0003B88002B0DD1154BC73319780A234B4376
:1068B000FA2189005B189A4203DD320035321378E1
:1068C00030E03200703213780A2B2BD93200353287
:1068D0001378002B01D0013B13703300002270337A
:1068E0001A7021E084060020A8030020D0FC0000DC
:1068F00030000E4000000E4094050020D803002018
:106900008806002010270000AC060020500500205B
:106910008C060020B40600204FC30000CC030020EA
:10692000AF06002001331370330035331B78032B7F
:1069300057D980220024FE21019BD2001B68C24E41
:106940005340019A89051360C04B1C80C04B1C80CA
:10695000C04B1888F36800939847BF4B1888736939
:1069600000939847BD4BAD6818882100A847BC4BE1
:1069700021001888A847BB4B21001888A847BA4BAC
:1069800021001888A847B94B21001888A847802102
:10699000B74AC90113680B431360FAF74FFE04228C
:1069A000B44B2100DA672000F9F742FE21000120F4
:1069B000F9F73EFE21000220F9F73AFEFEE7AE4B62
:1069C0001A68D2020DD4320036321278012A03D965
:1069D0001968AA4A0A4003E080211A68C9000A43DC
:1069E0001A6000232360A64B1A68A64B9A4209DC62
:1069F000964B1B88B32B05D802E023681E2B01D9C8
:106A000000232360A04B1B78012B00D98AE19F4D06
:106A10002B7801950133DBB22B701F232A781340AA
:106A20002B702B78002B33D1994C23781B0706D57C
:106A30008A4B01211888974B9B68009398472378CD
:106A4000DB0606D5864B01211888924B9B68009384
:106A5000984723789B0606D5824B012118888D4BD9
:106A60009B680093984723785B0606D57E4B0121EF
:106A70001888884B9B680093984723785BB2002B5B
:106A800006DA7A4B01211888824B9B68009398475D
:106A900076250427804A280011007231535D097859
:106AA0007538C0B2DBB214000F420BD01100713147
:106AB00009788C46664909888C4503D22B00083337
:106AC000D35CDBB2019A7F001278FFB2DB089342FD
:106AD00014D202386F4B614A03280AD800F0ACF98F
:106AE000020406085E4A04E05E4A02E05E4A00E0F4
:106AF0005E4A9B68108800210093984701357B2DE2
:106B0000C8D1664D2B68DB0600D40BE15A4B1B68DD
:106B10005B0555D52300C4331A78002A45D01A786E
:106B2000520602D51B789B063FD55D4B1888594B02
:106B3000DB68009398475B4900282FD10B885A4A9D
:106B4000002B03D113780133DBB213702300B3336E
:106B50001878137898421ED100223C4B20001A80EE
:106B60002B68043213432B600F23C4300278134088
:106B70004E4A5343013333630278D20601D59B005A
:106B800033632300C4331B785BB2002B03DB082282
:106B90002B6813432B60FA239B000B800B88002B80
:106BA00003D00B88013B9BB20B802300C5331A78BE
:106BB000002A00D1B6E01A78520600D58AE08CE0AF
:106BC0002300C4331A78002A00D17BE01A785206D9
:106BD00002D41B789B0675D5314B18882D4BDB688A
:106BE000009398472F49002865D10B882E4A002B27
:106BF00003D113780133DBB213702300B333187859
:106C00001378984254D10022104B20001A802B6830
:106C1000043213432B600F23C43002781340234AFD
:106C20005343013333630278D20601D59B003363AB
:106C30002300C4331B785BB2002B3CDB08222B689B
:106C400013432B6037E0C046B8FC0000AC060020C0
:106C500088060020A4010020A6030020D002002006
:106C6000B0010020A4030020A2030020B8010020EE
:106C70002805002004E100E084060020FFFBFFFF60
:106C8000B40600205FEA000024050020540500201F
:106C900026050020D0FC0000D80300209406002028
:106CA000B2010020B6030020460500201027000096
:106CB000FA239B000B800B88002B03D00B88013B31
:106CC0009BB20B802300C5331A78002A2AD01A7889
:106CD000520602D41B789B0624D5134B1888134BFD
:106CE000DB680093984700281CD10422104B210038
:106CF00018802B68C53113432B600F230A7813408B
:106D00000C4A5343013333630A78D20601D59B0002
:106D10003363C53423785BB2002B03DB08222B6876
:106D200013432B6007B0F0BD9E030020D0FC000091
:106D3000AC06002010270000F7B5354B1B78012B5F
:106D400064D8344D344C2A782378344F9A4202D197
:106D50003B78002B5AD03B78002B03D03B78013B8B
:106D6000DBB23B7001202E4A2E4E13780092013385
:106D7000DBB2137011782C4B01402C4A3BD01288A7
:106D80009B680100100001939847DC23227853434D
:106D900073602A7823789A4238D0009B1B780A2B9C
:106DA00034D90026224BAB330193019B1B789E42C2
:106DB0001DD82A7823789A4203D923780133DBB28D
:106DC000237022782B789A4203D92378013BDBB2D7
:106DD000237022782B789A4206D164233B70217865
:106DE000AB20C9B2FAF7EAF90136F6B2DDE70123C2
:106DF000009A13700AE09B68108800939847DC2380
:106E000022785B4253430B4A9B187360F7BDC04620
:106E100024050020FC040020B8060020980500206E
:106E2000AE06002020001140D0FC0000BA01002076
:106E3000D8030020E8DF050002B471464908490084
:106E4000095C49008E4402BC7047C04603B47146D9
:106E5000490840004900095A49008E4403BC704764
:106E6000002243088B4274D303098B425FD3030A89
:106E70008B4244D3030B8B4228D3030C8B420DD39C
:106E8000FF22090212BA030C8B4202D3121209022A
:106E900065D0030B8B4219D300E0090AC30B8B4268
:106EA00001D3CB03C01A5241830B8B4201D38B0316
:106EB000C01A5241430B8B4201D34B03C01A5241BB
:106EC000030B8B4201D30B03C01A5241C30A8B42FE
:106ED00001D3CB02C01A5241830A8B4201D38B02E9
:106EE000C01A5241430A8B4201D34B02C01A52418D
:106EF000030A8B4201D30B02C01A5241CDD2C309FF
:106F00008B4201D3CB01C01A524183098B4201D37A
:106F10008B01C01A524143098B4201D34B01C01A65
:106F2000524103098B4201D30B01C01A5241C308DD
:106F30008B4201D3CB00C01A524183088B4201D34C
:106F40008B00C01A524143088B4201D34B00C01A38
:106F50005241411A00D20146524110467047FFE7A4
:106F600001B5002000F0F0F802BDC0460029F7D0BE
:106F700076E7704703460B437FD4002243088B42D9
:106F800074D303098B425FD3030A8B4244D3030BB0
:106F90008B4228D3030C8B420DD3FF22090212BA75
:106FA000030C8B4202D31212090265D0030B8B42F1
:106FB00019D300E0090AC30B8B4201D3CB03C01ADB
:106FC0005241830B8B4201D38B03C01A5241430BB6
:106FD0008B4201D34B03C01A5241030B8B4201D3A6
:106FE0000B03C01A5241C30A8B4201D3CB02C01A11
:106FF0005241830A8B4201D38B02C01A5241430A89
:107000008B4201D34B02C01A5241030A8B4201D377
:107010000B02C01A5241CDD2C3098B4201D3CB011E
:10702000C01A524183098B4201D38B01C01A5241CD
:1070300043098B4201D34B01C01A524103098B42D1
:1070400001D30B01C01A5241C3088B4201D3CB00BC
:10705000C01A524183088B4201D38B00C01A52419F
:1070600043088B4201D34B00C01A5241411A00D24F
:1070700001465241104670475DE0CA0F00D04942B8
:10708000031000D34042534000229C4603098B4228
:107090002DD3030A8B4212D3FC22890112BA030AB0
:1070A0008B420CD3890192118B4208D38901921132
:1070B0008B4204D389013AD0921100E08909C309B7
:1070C0008B4201D3CB01C01A524183098B4201D3B9
:1070D0008B01C01A524143098B4201D34B01C01AA4
:1070E000524103098B4201D30B01C01A5241C3081C
:1070F0008B4201D3CB00C01A524183088B4201D38B
:107100008B00C01A5241D9D243088B4201D34B00A5
:10711000C01A5241411A00D20146634652415B10E7
:10712000104601D34042002B00D5494270476346C8
:107130005B1000D3404201B5002000F005F802BD0D
:107140000029F8D016E770477047C0468446081CEF
:107150006146FFE71FB500F0D1F9002801D40021F6
:10716000C8421FBD10B500F05DF94042013010BDAE
:1071700010B500F0C3F9002801DB002010BD01208C
:1071800010BDC04610B500F0B9F9002801DD00209F
:1071900010BD012010BDC04610B500F06BF90028ED
:1071A00001DC002010BD012010BDC04610B500F06C
:1071B00061F9002801DA002010BD012010BDC04691
:1071C0009E2110B5C905041CFFF7F0FF002803D16C
:1071D000201C00F071FC10BD9E21201CC90500F090
:1071E000E5FA00F069FC80231B069C466044F2E748
:1071F000F0B5564644465F464D46F0B4440246005C
:10720000C70F83B08846650A360EBA463DD0FF2EBA
:1072100022D00023EC00802599469B46ED042543AF
:107220007F3E43465C025800DB0F640A000E98461E
:1072300036D0FF2830D080230021E400DB041C433B
:107240007F38301A0190484642460843724E80000B
:1072500030587A4013008746002D44D108239946C0
:10726000063B9B46DDE70122FF2000241A40640212
:10727000C305640AD2071C431443200003B03CBC7E
:1072800090469946A246AB46F0BD002D20D104237E
:107290009946033B9B46C4E7002C17D1022102E02C
:1072A000002C0AD10121321A01924A4643460A4370
:1072B0005A48920082587B409746200002F0D6F947
:1072C000431F76309C4040420021BAE70321B8E7D3
:1072D000280002F0CBF9431F9D4000237630464240
:1072E00099469B469DE70C239946093B9B4698E7A8
:1072F00080240022E403FF20B9E70024C2468B4625
:107300005A465346022AAED0032A7DD0012A31D1F3
:10731000012200201A400024A9E70122101A1B288C
:1073200056DD1A4000200024A1E78023DB031D4224
:107330004BD18023DB032B435C02640A3A00FF201D
:1073400095E76D016001854230D2019A0024013A2F
:1073500001921B220127290064006D00002901DB36
:10736000A84201D82D1A3C43013A002AF3D16A1EE3
:1073700095412C4301987F300028CEDD620704D070
:107380000F222240042A00D00434220103D5244ACB
:10739000019814408030FE2800DD64E70122A4013A
:1073A000640AC0B21A4062E72C00A9E72D1A1A221B
:1073B0000124CFE76B02BCD500248023DB031C43F0
:1073C0006402640A4246FF2051E71C42B3D1F4E74D
:1073D00021002022C140101A8440621E94410C43B7
:1073E000620704D00F222240042A00D00434620134
:1073F00004D5012201201A40002438E70122A4010B
:10740000640A1A40002032E78023DB031C43640235
:10741000640A5246FF202AE72CFD00006CFD0000A4
:10742000FFFFFFF7430270B542004C005D0AC30F37
:107430004802120E460A240EC90FFF2A0FD0FF2C55
:1074400011D00120A24200D070BDB542FCD18B42C8
:107450000DD0002AF8D12800431E9841F4E70120FE
:10746000002DF1D1EBE70120002EEDD1E9E700205E
:10747000EAE7C0464302F0B542005D0AC30F480286
:10748000440A4800120E000EC90FFF2A1FD0FF2821
:1074900022D0002A09D16E426E4100280FD1002C63
:1074A0000DD10020002D09D005E0002801D1002CCD
:1074B00001D08B4213D0584201231843F0BD002E57
:1074C000F7D048424141012049420843F6E7002DE8
:1074D000DDD002204042F1E7002CDAD0F9E7824209
:1074E000E9DC04DBA542E6D80020A542E6D25842FA
:1074F000434101205B421843E0E7C0464302F0B538
:1075000042004C005E0AC30F4802120E450A240EC8
:10751000C90FFF2A17D0FF2C19D0002A0BD17042B7
:107520007041002C17D0002807D04842414101206B
:1075300049420843F0BD002C13D08B4214D058426E
:1075400001231843F6E70220002EF3D1E3E70220DF
:10755000002DEFD1E1E7002DE5D10020002EE9D08C
:10756000EDE7002DE9D1EAE7A242E8DC04DBAE4218
:10757000E5D80020AE42DDD25842434101205B42B3
:107580001843D7E7F0B557464E4645464300E0B4AA
:1075900046028846760A1F0EC40F002F47D0FF2FE1
:1075A00025D0002380259A469946F600ED042E4307
:1075B0007F3F434642465D02D20F5B006D0A1B0EC1
:1075C000904640D0FF2B39D080220020ED00D2041D
:1075D00015437F3BFB1842465746591C62408C4678
:1075E00007430F2F5CD86F49BF00C9598F46002E43
:1075F00045D108239A46063B9946DAE742460228D7
:107600002DD0032800D1C3E0012800D0A2E000253E
:1076100000260240D4B27602ED05760A2E43E40736
:10762000264330001CBC90469946A246F0BD002E71
:107630001AD104239A46033B9946BAE72A00511E01
:107640008A41901CC6E70120002DC3D0280002F01B
:107650000DF8431F76309D4043420020BAE70124D5
:10766000FF2514400026D6E7300001F0FFFF431F3E
:107670009E400023763047429A46994699E70C236C
:107680009A46093B994694E780260024F603FF2595
:10769000C1E735004846B2E7350022004846AEE76C
:1076A0002904090C0800370C3604360C2C0C7943DD
:1076B000704367437443060C64183619B14203D90A
:1076C00080214902884647440004000C310409180F
:1076D0008D01681E8541890E2943350CED19AD01D8
:1076E0000D43290104D5012369081D4063460D435C
:1076F00019007F31002925DD680704D00F202840BC
:10770000042800D00435280103D5274980330D40D3
:107710001900FE29A3DC0124AD016E0A1440CDB28C
:1077200079E78020C003064207D0054205D12843EF
:107730004602760A4446FF256DE706437602760A3E
:10774000FF2568E70124611A1B2905DD1440002587
:10775000002660E76346CBE72E002023CE40591A6F
:107760008D406B1E9D412E43730704D00F23334081
:10777000042B00D00436730104D5012401251440E4
:10778000002648E70124B601760A1440002542E7A6
:1077900080260124F6032E437602760A1440FF2544
:1077A00039E7C046ACFD0000FFFFFFF7F8B54A021D
:1077B0004E0043024400240EC50F9B09360EC90F2C
:1077C0009209FF2E00D183E001204140A01BA94275
:1077D0005CD0002800DC95E0002E1CD1002A00D0EF
:1077E00081E05A0704D00F221A40042A00D0043343
:1077F0005A013BD50134FF2C00D191E001209B01BF
:107800005B0AE4B205405B02E4055B0AED07234333
:107810002B431800F8BDFF2CE3D08021C9040A4394
:107820001B2800DD90E016002021C640081A824087
:10783000511E8A4132439B1A5A0115D59B019E095C
:10784000300001F013FF0538864084426CDC041BD5
:10785000330020200134E340041BA640721E9641F1
:1078600000243343BDE70D005A07BCD1DF080123D4
:107870001D40FF2C33D1002F00D190E08022D20395
:1078800013003B435B025B0AFF24BCE700284FDD8B
:10789000002E2ED0FF2CA4D08025ED042A431B28D7
:1078A00000DD97E016002025C640281A8240501EB1
:1078B000824132439B185A01D5D50134FF2C6DD03B
:1078C00001227B481A405B08034013430D0088E700
:1078D000002A00D07AE777E7031EC5D100257B0296
:1078E0005B0AE4B28FE701380028A4D0FF2C97D1BF
:1078F00077E7002A00D174E701380028DAD0FF2C9E
:10790000CDD16EE7002821D1601CC0B2012858DD1E
:1079100080279E1AFF0437402FD0D61A0D008FE71C
:1079200001231D4000236EE7624B241A334058E7C1
:10793000002851D1601CC6B2012E33DDFF282DD0A6
:107940009B185B0804004CE7012274E7002C1AD056
:10795000FF2E1FD08024E404404223431B2800DD77
:1079600096E01D002024C540201A8340581E834104
:107970002B43D31A34000D005EE7002E00D05FE7E2
:1079800000250024ABE7002B44D0C0430028F0D0F2
:10799000FF2EE3D11300FF240D0022E70D00FF248A
:1079A000002330E7002C5DD1002B7DD0002A00D1D0
:1079B00017E79B185A0100D456E73E4A04001340CB
:1079C0000FE7002C1ED1002B2FD1002A65D0130009
:1079D0000D0006E701226DE7002C1FD1002B59D0C6
:1079E000C04300280BD0FF2E4FD01B285EDC1D00AB
:1079F0002024C540201A8340581E83412B439B18E6
:107A0000340058E7002B1CD1002A49D013000D0088
:107A1000FF24E6E6130034000D00E2E6FF2E34D02A
:107A20008024E40440422343DFE7002A00D1D8E663
:107A30008027981AFF04074000D14DE7D31A0D00A4
:107A4000CFE6FF24002A00D1CBE68020DB08C0036C
:107A5000034204D0D208024201D113000D00DB0022
:107A6000FF24BEE6002B10D0FF24002A00D1B8E688
:107A70008020DB08C003034203D0D208024200D1B9
:107A80001300DB000D00FF24ABE61300FF24A8E683
:107A900001236EE713003400A3E6002700251EE74C
:107AA00080270025FF03E9E613009AE60123A6E7F5
:107AB000FFFFFF7DFFFFFFFB4302590A4300C20F98
:107AC0001B0E00207E2B0EDD9D2B0DDC8020000484
:107AD0000143952B0BDC9620C31AD9400B0058426A
:107AE000002A00D118007047034BD018FBE7963BE3
:107AF00099400B00F3E7C046FFFFFF7F70B50028F9
:107B000030D0C317C5185D40C40F280001F0AEFD8A
:107B10009E231B1A962B0DDC9622D21A95406A02E0
:107B2000520AD8B25202C005520AE4070243224365
:107B3000100070BD992B19DC9922D21A9540124A77
:107B40002A40690704D00F210D40042D00D00432D3
:107B5000510103D50C4B1A409F231B1A9201520A64
:107B6000D8B2DFE7002400200022DBE705222E0048
:107B7000121AB921D6402A00C91A8A40551EAA41B4
:107B800035001543DBE7C046FFFFFFFB70B5041E61
:107B900028D001F06BFD9E231B1A962B0ADC96223F
:107BA000D21A94406202520AD8B25202520AC00556
:107BB000104370BD992B18DC9922D21A9440114AB7
:107BC0002240610704D00F210C40042C00D0043265
:107BD000510103D50B4B1A409F231B1A9201520AE5
:107BE000D8B2E2E700200022DFE705222500121AC2
:107BF000B921D5402200C91A8A40541EA2412C0046
:107C00001443DCE7FFFFFFFBF8B556465F464D46E1
:107C10004446F0B40F00FD0FAA4609037C002E0075
:107C20005F00450F490A7F0D2943C5001803BC4674
:107C3000400A570F640DDB0F3843D2009A4500D13C
:107C4000AAE06646A61B002E00DCFFE06346002B80
:107C500039D10300134300D0D9E06B0709D00F23BB
:107C60002B40042B05D02B1DAB42AD416D42491971
:107C70001D000B0200D482E0CA4B01349C4200D1AB
:107C8000FEE00A005646C84BED081A40500764054E
:107C900052020543120B640D002112030B0D1B054C
:107CA0006405120B1A436308C04CF60714401C43CA
:107CB000640064083443280021003CBC9046994687
:107CC000A246AB46F8BDB74B9C42C6D080231B04EE
:107CD0001843382E00DDEBE01F2E00DD1EE12023CF
:107CE0009B1B9C4603006746BB40984613004746D3
:107CF000F3403B436746BA40571EBA411343020064
:107D0000F240EB1A9D42B6411D008A1A7642911B41
:107D10000B0231D54A02560A002E00D1B4E03000E1
:107D200001F0A4FC0300083B1F2B00DDB5E020227E
:107D30002900D21AD1409E400A009D4032439C4205
:107D400000DDB1E01C1B631C1F2B00DDD5E02021F2
:107D500014002800C91A8C40D8408D400443DA40F2
:107D6000681E854111002543002476E741463143D2
:107D700000D134E2310045466B0700D06FE756462C
:107D80004807ED08C9080543864B9C4235D00A03D5
:107D90006405120B640D7FE76346E31A9B46002BD4
:107DA00000DC8BE06746002F3CD07E4FBC4200D108
:107DB00053E780273F0438435B46382B00DCF7E06D
:107DC0000243501E82410020D2B253194218AB42E6
:107DD00089411D00494289180B02CDD5714B0134F0
:107DE0009C4200D13DE101206F4A6B080A402840C7
:107DF0001843D507054351082FE72B000B4300D14B
:107E0000CBE180231B030B431A03120B44E7013E13
:107E1000002E6DD1AE1AB5429B41091A5B42C91AB8
:107E2000350075E70700174300D116E701235B42D1
:107E30009C46E3445B46002B00D0E0E0AA18AA422F
:107E40009B4109185B4259181500C5E7002E75D1F2
:107E5000661C7605760D012E00DCF3E0AE1AB04606
:107E60004545BF410E1A7F42F61B370200D48FE012
:107E7000551BAA42B641411A76428E1B9A464BE7E1
:107E800056460022002507E7280001F0EFFB2030CE
:107E90000300083B1F2B00DC49E72A0028388240FA
:107EA00000259C4200DC4DE73F49E41A1140D4E62E
:107EB0000243501E8241D3B2002222E7002B00D0A1
:107EC000F3E0631C9C465B055B0D012B00DC9FE02F
:107ED000344B9C4500D1C3E0AA180918AA4280413E
:107EE00040424118CD075208154349086446B4E69C
:107EF0002C4B9C4200D0ECE6AFE611001F3CE14069
:107F00000C00202B00D17FE04021CB1A9A40154372
:107F10006A1E95410021254300242DE73300070008
:107F2000203BDF403B00202E70D04027BE1BB040DE
:107F30000243501E824113430022E2E6002C4FD040
:107F4000184CA44500D1ABE08024240476422143A0
:107F5000382E00DDDFE01F2E00DD43E12027BC1BB3
:107F6000A1460C004F46BC40A0462C004746F440BA
:107F70003C434F46BD406F1EBD41F1402C43151B95
:107F8000AA429241411A5242891A64469A46BFE671
:107F900041464546314300D0BEE600260024002578
:107FA000F2E6C046FF070000FFFF7FFFFFFF0F80E4
:107FB0001F2B59DC2027FF1ABC46070063469F4051
:107FC0005B46B9461700DF40B8464F4643461F435D
:107FD00063469A40531E9A415B463A43D840F4E6C2
:107FE0000C002C435CD0F643002E55D1551BAA4201
:107FF000A441411A6442091B9A46644688E6964F9A
:10800000BC4200D0D8E628E6002280E700208FE7B7
:108010000B002B43002C00D0C2E0002B00D101E16B
:108020000300134300D118E6AB18AB42B641091860
:10803000764271180A0200D409E1884A1D001140F5
:1080400064460AE6002C5BD10E002E4300D08AE085
:108050000100114300D1C2E0010015009A46FCE581
:108060006446002100258FE620235B429C46DC44C9
:1080700063460700DF405B46BC46202B00D1ACE0E6
:1080800040235F46DB1B98400243501E82416346FB
:1080900013431A00002098E66F4CA44500D057E720
:1080A0000100150064469A46D7E5002C39D10C0032
:1080B0002C436ED0DB43002B1AD0674CA44568D00C
:1080C000382B00DDA4E01F2B00DDAEE020240F00E4
:1080D000E41AA740B9462F00DF40B846A3464F46F2
:1080E000444627435C46A5406C1EA541D9403D430C
:1080F000AD1895429B4109185B42591864466BE6DE
:108100000C002C4315D1010011437BD00100150058
:108110009A46514CA1E50D43691E8D410021ECB2F8
:108120002DE74D4CA44534D0802424045B422143E8
:10813000C6E7040014434ED0ED084C072C438025BD
:10814000C9082D03294208D0C6082E4205D1D208FD
:10815000410711430C009A463100620FC900E50047
:1081600011433D4C79E50600164300D175E5AE1A82
:10817000B0464545BF410E1A7F42F61B370200D478
:10818000F4E5551BAA42B641411A7642891B9A462C
:1081900063E50100150064465FE5002200257BE5EC
:1081A000002B3BD00300134315D0ED084B072B43A6
:1081B0008025C9082D03294207D0C4082C4204D1C8
:1081C00041070B002100D2081343C9005A0F114385
:1081D000DD00214C41E5204C3FE5002054E700261E
:1081E0000025D1E534000F00203CE7403C00202E64
:1081F0002BD04027BE1BB1400D43691E8D4100218D
:108200002C43BCE6802100260903134C0025BBE566
:108210000D43691E8D410021EDB269E70100150093
:108220000D4C1AE50100150017E51C000F00203C5D
:10823000E7403C00202B0CD04027FB1A99400D430F
:10824000691E8D410021254352E70021D4E71D001E
:1082500092E50021F3E7C046FF070000FFFF7FFF24
:10826000F0B556464D4644465F46F0B41D000E0339
:108270004C00CB0F87B0070092468146360B640D49
:1082800098466AD06D4B9C4235D08022430F120431
:108290001343F6001E43C3009946694B00279C46D2
:1082A0000023644402932B0368001B0BED0F51461F
:1082B0009B46400D009500D178E0604B98426CD011
:1082C0005B46DA004B0F802109040B4313439B46A6
:1082D0005346D9005A4B9C46002360444246201A1C
:1082E0006A40924601901F430F2F00D9B0E05548D5
:1082F000BF00C0598746374300D088E00023994625
:108300000233082700260293CDE74346B346494689
:108310000093029B009A9246022B00D0BFE10021FD
:1083200053460122002689461A40444B0021360359
:108330000C0D2405360B2643434C1B0526401E43DB
:108340007600D207760816434846310007B03CBC99
:1083500090469946A246AB46F0BD330003434FD04A
:10836000002E00D1BCE1300001F080F903000B3B8E
:108370001C2B00DDADE11D220100D31A08393A00A3
:108380008F408E40DA40B9461643304B00279C465A
:10839000002360444442029385E753465A46134300
:1083A0002CD1002300219B46023397E70B4320D0BA
:1083B0005B46002B00D19EE1584601F057F90300BF
:1083C0000B3B1C2B00DD8FE102005946083A91401F
:1083D0008B461D21CB1A5146D9400B0059460B4301
:1083E00051469B469140194B9C46604440420023B5
:1083F00074E7002300219B4601336FE703236DE7F9
:108400000023994601330427002602934BE70323F8
:108410000C27029347E70122D51A382D00DCB0E182
:1084200053461A4000210023002689467EE7002398
:108430008026994600223603004B77E7FF070000AD
:1084400001FCFFFFECFD0000FFFF0F80F3030000C5
:108450005E4500D972E100D16DE1019B4D46013BC3
:1084600001930023340002935B461E020B0E1E4351
:108470000B020393330C994633041B0C494620002E
:108480000093FEF7EDFC009B37004343060049468E
:1084900020009846FEF76AFD2C0C09040C43A04509
:1084A00009D9E419731EA74200D95CE1A04500D8A0
:1084B00059E1023EE4194346E41A49462000FEF71A
:1084C000CFFC0300009A80465343494620009B4658
:1084D000FEF74CFD2A040904120C0A4393450DD9FA
:1084E0004346D219013B974200D93AE1934500D85F
:1084F00037E102235B429C46D219E0445B46D21A24
:108500004346360433439B460399180C0B0C1D005D
:10851000059309045B46090C0C001B041B0C444327
:10852000049159436B4368431B190D0CEB189C4293
:1085300003D980246402A44660441C0C09041B0473
:10854000090C20185D18824200D2DEE000D1D7E08D
:10855000161A029B9C465D1BAC459B415B42F61A7A
:10856000B74200D106E149463000FEF779FC009B96
:1085700004004343494630009846FEF7F7FC2E0CB2
:1085800009040E43B04509D9F619631EB74200D954
:10859000F3E0B04500D8F0E0023CF6194346F31A88
:1085A000494618000293FEF75BFC009B060043431C
:1085B000494602989846FEF7D9FC2D0409042D0C73
:1085C0000D43A84509D9ED19731EAF4200D9D6E075
:1085D000A84500D8D3E0023EED192404210043460B
:1085E0003143049E059A3000ED1A0B040C0C1B0C51
:1085F00058436643534354439A19030C9B189E42B5
:1086000003D980225202944664441A0C00041B04CD
:10861000000C14191B18A54250D34DD00123194347
:10862000964A019B94466344002B00DCF3E64A071C
:1086300009D00F220A40042A05D00A1D8A42894126
:1086400049428B4411005A46D20108D55A468C4BF8
:108650001A4093468022D2009446019B6344894A83
:10866000934200DD5BE65A46C908500708435602AC
:10867000514601225B058146360B5B0D0A4055E6EB
:1086800080231B031E4211D05A461A420ED15E4669
:108690001E433603360B2A0089467B4B46E6032BE6
:1086A00000D1E1E0012BBBD11A40BBE61E433603EB
:1086B000360B4246744B39E6002BB1D07D194A1E69
:1086C000AF4252D91100A542A8D1039A9A42A5D12E
:1086D000A6E703003E00283B9E400023994654E64F
:1086E00000F0C4FF203041E603005246283B9A4088
:1086F0000021934677E6504600F0B8FF20305EE652
:10870000029B0026AB4200D323E7039E0299B446A6
:1087100061448846B045B6415B467642F619B218C8
:10872000013B0291974213D290424FD800D18EE084
:10873000161A9B460DE7894500D28EE674084B4613
:10874000F60735005B081D434B46DB0702938BE6BB
:108750009742EDD10399029CA142E5D93E1A9B466E
:10876000F7E69846CAE61E00A5E6AC423ED874D0AD
:10877000110053E70121494252E71C000EE71E0099
:108780002BE71F2D3CDC20230A0058465B1B98403A
:10879000EA4099400243481E81415E461143EE4043
:1087A0004B0709D00F230B40042B05D00B00191DDC
:1087B00099429B415B42F61833023CD55346012255
:1087C00000211A40002601238946AFE502235B42BF
:1087D0009C46039CE344A446029B63449846A04500
:1087E000B6417642F6190293B218B1E603988A1E92
:1087F00041008142B6417642F619AD19039161E715
:108800001F225242D31A5A46DA401300202D29D093
:1088100040225846551BA8400143481E814107206D
:108820000B4318400026002809D00F2200261A40CA
:108830001900042ABBD10B0070077602360BDB0847
:1088400003439946012253461A4000236EE50299DC
:108850008D42BBD89B4600267BE603989842C5D341
:10886000110032E70020D7E780265B4636031E431F
:108870003603360B009A8946034B57E5FF03000089
:10888000FFFFFFFEFE070000FF070000F0B55F4698
:1088900056464D464446F0B40D0399464E002B0B08
:1088A00087B00700924680469B46760DCC0F002E7F
:1088B00069D06D4B9E4235D05B468022DD001204AC
:1088C000430F13432B439B46C3009846674B002737
:1088D0009C460023664401934A4615035000D20F7C
:1088E00053462D0B400D914600D176E05E4A9042F2
:1088F0006CD080225B0F120413435C4AED00944657
:108900001D4353460022DB00604449463618701C64
:108910006140029017430F2F00D9AFE05448BF00C9
:10892000C759BF465B461F4300D088E000239B46E3
:108930009846023308270193CEE74946022A6AD0B7
:10894000032A00D109E2012A00D0BBE11140002234
:10895000002300259046CCB200212D030A0D1205FC
:108960002D0B1543434A1B0515401D436D00E407BD
:108970006D0825434046290007B03CBC9046994607
:10898000A246AB46F0BD034352D05B46002B00D15C
:108990008AE1584600F06AFE03000B3B1C2B00DD09
:1089A0007BE11D22D31A3A0001005D46DA40083906
:1089B0008D4013008F402B439B46B8462E4B00271B
:1089C0009C46002360444642019385E752462A4371
:1089D0002CD100250023022297E752462A4321D0BA
:1089E000002D00D154E1280000F040FE03000B3BB5
:1089F0001C2B00DD46E11D21CB1A51460200D94057
:108A00005346083A954093400D431B4A94466044B0
:108A10004042002279E7012400220C40124B00253D
:108A2000904699E70025002301226EE703226CE7B8
:108A300000239B4698460133042701934CE7032308
:108A40000C27019348E700238025984600242D0336
:108A5000054B81E75D464346019A6FE75D46434615
:108A60002100019A6AE7C046FF07000001FCFFFFF2
:108A70002CFE0000FFFF0F80F30300004246120CA3
:108A800091461A0C9446424617044A461B041B0C96
:108A90005A43604690464A4642431000039262465B
:108AA0001C003F0C7A437C4342440192220C9246C4
:108AB000019A5244904506D9824680204002804661
:108AC000C24450460390100C049048462404240CE1
:108AD0001204121905922A0C2D042D0C68432C0047
:108AE000824648467C4350438146200C804657438B
:108AF00057444744BA4503D9802040028046C144C8
:108B0000380C3F04B84648442404240C01900498CF
:108B1000A044404404905846000C81465846040442
:108B2000200C8246070048465F434C46434360465C
:108B300060436446834650464443380C8446E418F8
:108B40006444A34203D980235B029C46E344484625
:108B50003F04230C3F0C2404E419574668436F4339
:108B600084464D46504655434243380C8146624444
:108B70004A445B44944503D98020400284466544BE
:108B800003983F04834604983F0C8446E344C3455E
:108B900080414042824610048446019867448446DE
:108BA0006744A344BC46A345A4419946D4446442C7
:108BB0008742BF41D4458041E144A04699459B414D
:108BC0007F424042C8440743120CBA18A045A44152
:108BD0005F423B0064422343D71843467D19DB0DB7
:108BE0006D021D435B465A02059B1A43531E9A4170
:108BF0005B46DB0D1A4343465B021343EA0107D58C
:108C000001225C0813402343EA07029E13436D08C8
:108C1000574AB218002A4BDD580709D00F201840D8
:108C2000042805D0181D98429B415B42ED180300B3
:108C3000E80104D54F4A15408022D200B2184E48B0
:108C4000824200DDE7E60124DB08680718436D0275
:108C5000530580462D0B5B0D0C407DE68022594666
:108C60001203114208D0154206D115432D03984630
:108C70002D0B4C46414B6FE65D4615432D032D0BE6
:108C80003E4B69E603005546283B9D400023BCE669
:108C9000504600F0EBFC2030A8E60300283B9F4044
:108CA0000023BB46984689E600F0E0FC203073E6DE
:108CB0000124A61A382E07DD00220C4000230025CF
:108CC000904649E6029EA3E71F2E20DC20222C00BE
:108CD0001800921BF040944093400443581E834177
:108CE0001C43F540630709D00F232340042B05D014
:108CF00023001C1D9C4292415242AD182B021FD5ED
:108D0000012400220C4001230025904624E61F2068
:108D10002C004042821AD440202E1CD04022961BA8
:108D2000B5402B43581E834107202343184000259C
:108D3000002809D00F2200251A401C00042AD8D18F
:108D4000230068076D022D0B0124DB0803439846BE
:108D50000C40002300E60025E3E7802201241203F3
:108D600015432D0398462D0B0C40044BF4E5C046EB
:108D7000FF030000FFFFFFFEFE070000FF070000EB
:108D8000F0B557464E464546E0B40E001100F20FCE
:108D90009246C500420F180337037400400A4E0F75
:108DA0007F0A3043CF4E17435A00640D520DDB0F3C
:108DB000C900B24200D1E5E001267340A61AB446CC
:108DC000534500D1AFE0002E00DC0DE1002A3AD17E
:108DD00003000B4300D0E4E06B0709D00F232B40C6
:108DE000042B05D02B1DAB42AD416D427F191D00F8
:108DF0003B0200D488E0BB4B01349C4200D110E11F
:108E00003A00B94B51461A4001235007ED0852026F
:108E100064050543120B640D0B400021280012036A
:108E20000D0D120B64052D0515436208AF4CDB07D1
:108E30002C401443640064081C4321001CBC904671
:108E40009946A246F0BDA74B9C42C5D080231B0487
:108E500018436346382B00DDFDE01F2B00DD30E1B9
:108E6000624620239B1A02009A40664690460A00FA
:108E70009940F24046464B1E9941324311436346A6
:108E80000200DA40691A8D429B410D00BA1A5B421A
:108E9000D71A3B0235D57A02530A98464346002B2F
:108EA00000D1C4E0404600F0E1FB0300083B1F2B6B
:108EB00000DDC5E020222900D21A4746D1409F405C
:108EC0000A009D403A439C4200DDC0E01C1B631C2D
:108ED0001F2B00DDE4E0202114002800C91AD8402F
:108EE0008C408D400443DA40681E854117002543BD
:108EF000002471E7424663461A4300D14CE26746BC
:108F000045466B0700D069E7012351467807ED0815
:108F1000FA080B40054373498C4238D012036405AC
:108F2000120B640D79E7002E00DC9AE0002A47D08E
:108F30006C4A944200D14FE78022120410436246EB
:108F4000382A00DC08E10143481E81410022C9B2F1
:108F50004919D219A942BF410D007F42BF183A02F8
:108F600000D442E15F4A0134944200D14EE1012035
:108F70005D4A69083A4028400843D5070543570829
:108F80009A4629E706000E4300D017E714E72900A8
:108F9000114300D1F9E1802109030A431203120BA6
:108FA0003BE701235B429846C4446346002B72D1E1
:108FB000691A8D429B413F1A5B42FF1A0D0068E718
:108FC00002000A4300D107E7012252429046C444FE
:108FD0006246002A00D0E6E06918A942B6413F186F
:108FE0007642F7190D00BAE7002E00D080E0621C2F
:108FF0005205520D012A00DCF9E06A1A91464D45EE
:10900000B6413A1A7642921B9046120200D499E079
:109010004D1BA9428941C71B49427A1A90469A467C
:109020003CE752460123002513400022F5E62800C4
:1090300000F01CFB20300300083B1F2B00DC39E74D
:109040002A002838824000259C4200DC3EE7264F5B
:10905000E41A1740C0E60143481E81410022C9B20C
:1090600010E7002E00D0F1E0621C94465205520D2C
:10907000012A00DCA0E01B4A944500D1C5E0691834
:10908000A94292413F185242D2194908D5070D43CF
:1090900057086446A0E6134B9C4200D0D9E69BE6F5
:1090A00011001F3CE1400C00202B00D180E040214A
:1090B000CB1A9A4015436A1E954100272543002488
:1090C0001FE763460200203BDA406346202B71D045
:1090D000402366469B1B98400143481E8141114333
:1090E0000022CFE6FF070000FFFF7FFFFFFF0F809A
:1090F000002C48D0CA4CA24200D1A2E07442A14642
:109100008024240427434C46382C00DDDBE01F2C50
:1091100000DD44E14E462024A41B3E00A640A246AA
:10912000B0464C462E00E640B446464664462643CA
:109130005446A5406C1EA54134002C434D46EF40DB
:109140000D1B28E04A4643464D461A4300D0A5E68B
:10915000002300240025DEE61F2A5ADC6646202272
:10916000921B060096409146B04662460E00D640DD
:10917000424616434A4691404A1E914102006046CB
:109180003143C240E4E63C002C435AD0F443A146AC
:10919000002C52D14D1BA9428941C71B49427F1A5D
:1091A00014009A4675E69E4A944200D0C7E613E63C
:1091B00000227FE700208FE7002C00D0C8E03B00B2
:1091C0002B4300D10FE103000B4300D104E66918E3
:1091D000A9429B413F185B42DF193B0200D41AE1D0
:1091E000904B0D001F406446F6E59A4689E63A002A
:1091F0002A43002C5CD1002A75D102000A4300D119
:10920000CAE007000D009A46E6E564460022002504
:1092100081E662460600203AD6406246B046202AE1
:1092200000D1B7E040226646921B9040014342467F
:10923000481E8141114300228AE6794CA24200D0A7
:1092400061E707000D0014009A46C5E5002C41D1E6
:109250003C002C4378D0F443A146002C20D0704C25
:10926000A24271D04C46382C00DDB2E01F2C00DD4C
:10927000BCE02026341BA2463C005646B4404E4675
:10928000A0462C00F440A446444666463443A44617
:109290005446A54064466E1EB54125434C46E74002
:1092A0006D188D4289413F184942CF19140056E686
:1092B000002A2FD102000A4300D184E007000D00EC
:1092C0009A46574C88E53D436F1EBD41ECB20027DE
:1092D0000D1B60E7524CA24236D074428026360401
:1092E000A1463743BEE702000A4300D174E56A1A7B
:1092F00090464545B6413A1A7642921B9446120270
:1093000000D4F7E54D1BA9428941C71B49427F1A8A
:109310009A4661E502000A433AD0ED087C072C43E7
:109320008025FA082D032A4208D0C7082F4205D10C
:1093300045072C003A009A46C9080C43670FD20033
:10934000E5001743364C47E507000D00140043E5E0
:109350003A002A4343D002000A4319D0ED087C07A3
:109360002C438025FA082D032A4207D0C6082E4236
:1093700004D147073C003200C9080C43D700620FF4
:10938000E50017439A46264C26E50022002544E5D1
:10939000234C21E5002049E700230025BBE54C468E
:1093A0003E00203CE6404C46B446202C31D04024C0
:1093B0004E46A61BB7403D436C1EA54164462C4358
:1093C00000270D1BE7E6802200231203144C002522
:1093D000A1E53D436F1EBD410027EDB260E70700E8
:1093E0000D000F4CF8E407000D00F5E44E463C007C
:1093F000203EF440A0464C46202C0ED040244E4641
:10940000A41BA7403D436F1EBD4144460027254392
:1094100046E70027CFE70D0073E50027F2E7C046D7
:10942000FF070000FFFF7FFF70B5002830D0C31793
:10943000C4185C40C50F200000F018F9174B184AFB
:109440001B1AD21A1F2A18DD164AD21A944000227B
:1094500024035B05240B5B0D0021100024030A0D7F
:109460001205240B1443104A1B0514401C436400CE
:10947000ED0764082C43210070BD210091400A00D3
:109480000B21081AC4405B052403240B5B0DE3E7A2
:109490000025002300240022DEE7C0461E04000051
:1094A0003304000013040000FFFF0F804200120E7F
:1094B000511C4302C9B270B55D0AC40F012915DD04
:1094C000E02189008C466D071B0B624400212800B7
:1094D0000D0D2D052B431C4D52052B4052081343F7
:1094E0005B00E4075B082343190070BD002A15D117
:1094F000002D1FD0280000F0B9F80A281DDC0B232E
:109500002A001B1ADA4013000200153295400F4A58
:109510001B03121A52051B0B520DD7E7002D06D064
:1095200080221B0B120313436D07094ACEE7084A3A
:109530000023CBE700220023C8E703000B3B9D403C
:109540002B000025E3E7C046FFFF0F8089030000E2
:10955000FF0700004B0070B55E0D0C03751C640A1C
:10956000420F6D052243C90FC4006D0D012D2ADD88
:109570003B4BF318FE2B1ADC002B42DD8001451E0D
:10958000A841D2001043620F0243500704D00F20BD
:109590001040042800D004328020C004104021D0A4
:1095A0000133FF2B03D09201520ADBB201E0FF230B
:1095B00000225202520ADB0513435B00C9075B0815
:1095C0000B43180070BD002E07D01443EFD080204D
:1095D000D20080040243FF23D7E722430023002A5E
:1095E00003D00522D208FF2B03D05202520ADBB26D
:1095F000DFE7002A32D08020C00302435202520A21
:10960000D7E71800173014DB8020000402431E2027
:10961000C01A1F280FDC2500124BF3189D406E1E48
:10962000B5419A402B0013432200C2401A43002345
:10963000ABE70023D5E702256D42EB1A1500DD40AC
:10964000202809D0084BF3189A401443621E944115
:10965000220000232A4398E70022F6E70022A8E729
:1096600080FCFFFF82FCFFFFA2FCFFFF1C21012307
:109670001B04984201D3000C10391B0A984201D3F5
:10968000000A08391B09984201D30009043902A2D3
:10969000105C40187047C04604030202010101013A
:1096A0000000000000000000807F7F7F7F7F7F7FC1
:1096B0007F807F7F7F8080808080807F7F7F7F7FB3
:1096C0007F7F7F807F7F7F807F7F7F807F7F7F80A6
:1096D0008080808080807F7F7F7F7F7F7F80808091
:1096E0008080807F7E7F7F7F7F7F80808080807F83
:1096F0007F7E807F7F7F808080808181807F7F7F71
:109700007F7F7F8080808080807F7F80807F7E7E63
:109710007F807E7E7F807F7E7E807F7D7D7F80805C
:109720007F80807F7F808280807F807F7F7F80813D
:109730007F7F80807F7E7E7E7D7C7F807F7E7F833B
:1097400084838181807E7D7E8081807F807F808018
:109750007F7D7C7D7D7C7B7E807F808385837F7E1B
:109760007F807F80818280808182807E7E7D7D7B04
:109770007C7E807F807F8080817F7E7F807F7E7EF9
:1097800081827F8083837F7E7E807F7D7D807D7AE6
:109790007B7F817F8184837F7E7F7D7B7C808282D3
:1097A0008487867F7E7F7D7A797C7F8083827F80BD
:1097B0007F807F807F7F7D7A7D81828183837F7CB4
:1097C0007B7E7C76787D808081848584807F7E80AE
:1097D000807F817F80807F808182807F7F7E7A7999
:1097E0007A7B7E808183818280807D80817F7F7F84
:1097F00081807D7C80807E7C7F7E7B7B7D7F7F8483
:1098000086868080807D7E7F808281807F7E7D8055
:109810007F807F807E7D7E7C7C7E8182807F828552
:1098200082807F817F7D7D7D808081808181807D40
:109830007D7F7F7D7F8082818080807E7E807F7E35
:109840007C7D7E8081807F80807F7E807F807F8026
:109850007E7E7C7C7B7C8080807D7C7C7D7B7D7F34
:10986000818385828381817F7F7F807F7D807F7FF1
:109870007F7E7E7C7D7C7E7E7F8182817F807F80FB
:1098800080817F807E7F7C7B7D7F7E808283827FE4
:109890008181827F80808082807F7D807E7C797ADA
:1098A0007E7F7D7C7F7E7F7F8082847F81848482B7
:1098B0007F7F7E7E7B797B7C7D7E7F8080818180C7
:1098C0008180848686838382817B757479797979B6
:1098D0007C7E7F7B7D808686878A8C8D86817F7764
:1098E0007172777877747776797A7F868C90939394
:1098F000908B858179757475716E70737272767ED6
:109900008991989C9B96918980726D696969696E4D
:109910007073757B838E939A9EA09A918B867C72CE
:1099200066615F5F5B616F7A7E87949FA29E9F9F57
:109930009F93867A7166615B5A5C5F676F79828DEF
:10994000959DA3A7A9A59E91847666574E4D535E1B
:10995000676F7B828B929AA0A9AEAEAB9F8F79671F
:10996000574C4949536270767C85919CA5AFB5B63A
:10997000ACA08F776355514C4D535E67707A8998D0
:10998000A4ADB5BAB7AC9B856F625D574E4E5050D3
:10999000535B6E8498ACBDC4C2BAAB96806E6867E8
:1099A00060554A4849485265849EB2BCC4C6B8ACAA
:1099B000998574686561554B4C4B4A536A889CACD9
:1099C000BBC4C2B7A49281726A67615B504A4B48BC
:1099D0004E647F9DAFB9C0C2BDAC98877B72695C95
:1099E000544B49494F5A6C829AA6AFB3B8BCB19B4D
:1099F000887D70655953515052585C687E91A2AC75
:109A0000B6BEBEB19E90847D736A5D4D4340444CAA
:109A1000587490A3AFB3BDBEB09B8E86807469644A
:109A20005A524D4949586B8093A7B9C4BEBAA992FE
:109A300081767268575156545351576676859BAC60
:109A4000B9C2C6BBA0887971675F5B5E5C55515235
:109A50005B69829CB2BCC5C5B599807374736F672E
:109A600062625C4E464D648094A2B9C3C2B39E88C4
:109A70007E79776D5E5357514E4952677B91A0B006
:109A8000C0C7BBA79485807D7163595857524F4E0C
:109A90005C758C9BACBBC3BBAB998B86847E6F63C0
:109AA0005751443E3C48627D99B2C1C7C2B2A090B2
:109AB00085807F786C645949373142627F9BB3C39C
:109AC000CCC5B39F8E8B8782786D5E4E362C354722
:109AD000607F9BB4C0C0BBB19B8988938F7D6F664C
:109AE0005435283551667B97ADB9C0BBB3A2969467
:109AF00090867A685A4E463E3F51657A8DA1B2BB38
:109B0000BCB2A69794958C7B6D5F534C463F4856EC
:109B10006F8397ABB7B9B6AB9A9089858679685B46
:109B20004F43393B536D8597A7B5BEB7ACA2938F12
:109B30008B867F6E5E574C413B4A657F94A9B9C3C3
:109B4000C0AA998C867F7A7C776E605448464756C7
:109B5000738EA7B5C2C6B28F797775787B80796826
:109B6000574A41435F839EAEBEC8C3A98B797578BF
:109B70007773726F645749424B5B799BB3C4CEC411
:109B8000AB907973737A76736C6454433B4A678302
:109B90009CAEBFC7BBAA97897D7779766859565422
:109BA0004F4E586B8598A7B4BFC2B398857B7A7621
:109BB0006D635D5352555C6B7C8C9FA8AEACAAA4C0
:109BC00094857C8081725F514C4A556A7F8E9EA439
:109BD000A19F9C9B95877F808582715F4F444155F3
:109BE000728A9AA7ACA8A59F94837A7C7F7E7B76A5
:109BF0006A554B54657C89989FA2A4A1988A7E7768
:109C00007777767870695F595B6F87989E9B9EA582
:109C10009D9085827D6E636968625E62676E7D8DF0
:109C2000999CA0A6ABA79C8B77675F5D61656B6E07
:109C30006F6D6F798B9AA1A7AEA69E8E7E6F615ACB
:109C40005F666664666B6F76899AA7A9A9AEA794CA
:109C500080796D635C585D6161656C767F8EA3AAC7
:109C6000A7A9A9AA967765615C56555D6A6D6E7065
:109C7000778697A5B4B5AEADA08E745D59595C5981
:109C8000565C5F5D697B93A6A8B0B4AC9F9C938142
:109C90006E625A554C48505B68788BA2ABA7A7AE52
:109CA000B9B9AC95795C4742454B56616F7D82915D
:109CB0009D9E9DA2AFB5BAB49A745546413B3D4EA8
:109CC0005F6F7A8B989FA1A0A2AAB0B3A78F6E55A1
:109CD000443F42515E6D767E8B99A3ABAFB1AFAD81
:109CE000AA9676564546443B49617173788EA5AD78
:109CF000B0B5B2B0AAA28D6B50494B4E50596673A5
:109D000073727E9CAFB0B1B6B9AFA28A683E313BE8
:109D1000484C5A7784837F8F9DA2A7ACB5C3C5B04A
:109D200086593D2E313B4D687E8489858898A7AF42
:109D3000B6BCBFB29873553D3132414F64767C85D5
:109D4000909BA5B1B7BBB8B4AA96714F3A323540D3
:109D500059717B7B81929BA7B0B4B0AEB1A5906DD9
:109D6000463032405363718085888F9FAAB2B2AE6D
:109D7000ACA6988463483E414950596C787F8D9FCA
:109D8000AFBAB4AEAFA69886745F47323A46525C1B
:109D900070868F96A1B0B6B4AEAEA59B8E74513DC1
:109DA00038414C5A697F90908E96A1A6A6A3A3A68F
:109DB0009F8B704E353941526275899297989DA458
:109DC000A7A29EA5A6A08B6542353C46526A7F8F0E
:109DD0009293929E9D9396A5B3AC9B87653A2A3B3E
:109DE0004E5E6A7E888C919CA4A3A7A8A5A4A1928C
:109DF000765A433D4346586E777A89A5B3B3A8A2F5
:109E0000A49E938E887E674F424149525E72809035
:109E1000A3AAACA9A29B9796988E795D4640434B26
:109E20006074808891999F9EA0A19C9796958A7650
:109E30005B46414B5C6C797B838B939AA2A49D9A81
:109E40009AA29F89674F4140485C78878280838EC1
:109E5000908F9CA8A5A0A49D87664741414A627E39
:109E60008D897E838C8C8FA1B6B9AEA49C7C503139
:109E70002B3D5268808E867D797D8691A6B8BCB3D5
:109E8000A9A08C653A212C47617989939292888A9E
:109E90008D93A3AFB7B9A9865F3F313040627E860C
:109EA000868B92908C969FA3A6ABA8978067503E16
:109EB0003C4F61696F7C8F99999699A4A29DA2A449
:109EC0009178624F4B4C556A757371788B9699A255
:109ED000A3A19A9A9A91776259595B5F6367686FF9
:109EE0007C818A9DAAAEA6A2A29C877662504A492E
:109EF0005561676D7C8E989FA9B1AA9C918F8D80CA
:109F00006C615F5F5A5A626B6D72859BABB0B2B386
:109F1000AB9A8E8270605451585E5E5C62707E8F28
:109F20009EA9B0B0ACA79A8F83706158575B5E5200
:109F300051667C8A99A6B0AFAB9E93908E88776A63
:109F40005E59514F51565C708CA2ABA8A8A8A79E31
:109F50009690887260564E4D4E5363718194A4B0B2
:109F6000B6AFA8A29A8F837668595356565658634F
:109F7000737F8A9EA9A9ACACA89F9C93785B474A43
:109F80005356565A697B7F8699ABB9BCB9B6AF9E1A
:109F90007F5B413C444C51545666808F979EABB8D2
:109FA000B7B0B4B8AA8C6748383136424F6989A136
:109FB000A4918E969C9CA3BEC9BD9B6A41211B287F
:109FC00035517593A6A194918F939FACB8C7C6AC39
:109FD0007D442521252F496E8E9E9B8F8D93A4A8AD
:109FE000ACBDCCBC916F544133323D4B5F79828123
:109FF0008090ADBFBDBABEBBB2966F4D3A3C3D3B03
:10A000003D4B5F747F94ADC4CCC7B3A6A3A797782C
:10A01000594B463B2C2B415A6F8191A6C2CCC9BBF0
:10A02000B1AEA3896F554A463F3E4B5E707D838A31
:10A030009DB1BEC3BEB7AA96754E34313D46556735
:10A040007F8B88807E8CAACAD9D5C5AA865F301836
:10A05000253B4C58718C90827D8C9CABC4D4D3BF73
:10A06000AD9064342027393E415F7A8588949EAA5A
:10A07000B9C8CFCABEAB885C33242F3D484F5C6E55
:10A080007F878D9FB2C4CDD1D0C1A47C512D263104
:10A090003537436278838D97A6B2BBC7CFC9C2B1AB
:10A0A0008A51281D242A2B406585959A9BA8B2BB0E
:10A0B000C6CECEC5A77E4A241A26333640577988A5
:10A0C000919CACBCCCD3D3CFCAAB75402924211F03
:10A0D0002A44667A8897A0ABBBCACFCBC8C3A87402
:10A0E0003E2A2C312D324B606E7D91AEBECDD8D83C
:10A0F000D0C5B596683C2A2A31323544566E879BC6
:10A10000AFC7D4D2CDC2BDB29A714836352F1B1C11
:10A110002D4A6E8FADC3CDCCCECDC8C2B996612EBF
:10A1200020242C2E3247638097ADB5BECFDBDDD621
:10A13000CAAD7D42140A1627384A5B707D8E9FAEE9
:10A14000C2D3DDDCD3C4AB7939151D2D3539567238
:10A15000797A8393A6BDD0DDDAD1C2A36B33141A0A
:10A16000313F45526C7C848A95AEC6D7DBD6CDBADA
:10A17000996536222A34393740586E8090A3B8CD7D
:10A18000D5CEC7C3BE9F6E3F2C3133292C3E586DB0
:10A19000859EB2C4CECFCAC3BFBDA4723E2D3026A9
:10A1A0002029446175879AABBBC6CFD4D2CFC19664
:10A1B000552315222B303C628187878D929EB5D323
:10A1C000E4DDD0BD8D4F1B0E213037446B8C928B5C
:10A1D00092A2B4C1D1DEE0CEA97D4217101A212788
:10A1E0003C62879DA4A6AFB6BFCED4CFC6AE7B3FA0
:10A1F00013102125273F6984919BA6B2BAC9D7E0E5
:10A20000DCCCA76D301112222A293E64808A93A8E3
:10A21000BDCAD5E0E2D5C09F6E3613121D231D3393
:10A220005F879AA4B2BABABECDD9D5C3A577431A6F
:10A23000121D24223E6F939CA0AFBBB8BECDD7D1D8
:10A24000BE98602B161B25252941698594A7BEC39E
:10A25000C4C8D2D6CBB7925D26111A292D314B74C2
:10A2600094AAC0D0CEC4BBBBC0C3B49058261714A8
:10A270000F0C264C7497B1C3C8C5BAB9BABFC7BBD7
:10A28000925527161C1D1D2D547A9AADBDC2BCBA1D
:10A29000C8D2CBC3AC824E1F121E2A2B3A5E8196C7
:10A2A000A0ADB4B2B1BED0D9CBA6783E160C17265D
:10A2B000384B63889DA3A8B0B7BDC9D4CFBC9B71F0
:10A2C0003B1616293235425C7A93A8BACACBC9CB61
:10A2D000CEC5B6A079492F2F2F221F304B708CA5E9
:10A2E000BDC4C2BFBEC5C4B7A27E543A312E231A24
:10A2F0002C4D7592A8B8C1C3C2BBC2CDC4A87C4EB8
:10A300002B1E1A1A182B5687A1ABA8AAB0B6C1D219
:10A31000E1DCB888542810111929436B8F9B999957
:10A320009FA9B8D1E5E3CEA56F38160C1622375693
:10A3300081A0A39B9AA0A1A4BAD5DCC9A57C481E84
:10A34000090D22385482A4A296949FABB0B9CEDDF9
:10A35000D0A87B51261110162D507C9FA497969E55
:10A36000ABB5C2D6E4D8B482481F0B06091A4B7F9E
:10A370009C9E9796A6B1B8C7DAE8D8B17F512B1743
:10A380000F09183E6D8D8E99B0BEBFBCC5D0CDB241
:10A390008F65442F2C2B2024486B8295AABAC1C507
:10A3A000C8C8C0B5A2826045404138272A44647EAF
:10A3B00099B1C1C2C1C7C8BDAE9776543B302C22FB
:10A3C0001930598094A8C1CEC5BFC0CAC7B29A7906
:10A3D00052331D13161F38668DA4AFBCCACBCACD2D
:10A3E000D0C6A68067492E1F13101836658CA6BAF2
:10A3F000D0D8D5CAC4C1B1957B583B2C241F141AA0
:10A400003C6B8EA4BED5DACCC2CAC8B89A7E614570
:10A410002D2220202A466C90A8BCCECDC6BEBDB64B
:10A42000A9947E5F44331E181D2D456792BDD7D970
:10A43000D0BFAFAEADAD9C7F65533B1D0E1E384AFD
:10A440006395C1DAD9D2C5B2AAADA590745D4F3477
:10A450001005163C5F7A9CC2D5D8C4B4B4BFC3B74C
:10A460009A77593716010511346590A9BED2D5C720
:10A47000BABFCDD1BEA0825A2A3580570A20507D5E
:10A480009CB7CAD0D2DCE4E4D0B08E6C4C2B3680C2
:10A490005814304E7092B2C8D9E9F4F0E2C79A6409
:10A4A0004436253557091C365586B5CDDDECF3EE1F
:10A4B000DBCBB2875C463B2C3A57081737608ABD26
:10A4C000DBE4E4E9E6DEC6A883675A45202D580997
:10A4D000193B6CA1CCDBE0E3E7E3DFC9A779534785
:10A4E0003F1E2E560C1C3A6CABD7E0DBDCE8ECE5EB
:10A4F000CA9F775951474B7F560A234F7CA4C3D03C
:10A50000D9DBE3E9E7CD9B603F4035405406153980
:10A51000628ABACCCBCDDDF2EFE1C8A16C473C2B0F
:10A520003D5306112D597FA6BDCAD1E1F4F5E8C708
:10A53000986C524322305505102D679EC0CBD0DD5C
:10A54000E1E4E9E7CC9B6146313D7F550510275991
:10A5500099C9DCE3EDF2ECDECFB891664D401F2DDA
:10A5600055050F235198DDF9F4F1EDE5CFBBA48437
:10A5700064513C488054060E2965B0DFF0F7FBF1CA
:10A58000DED0BA91664B44324080550A19447FB6FA
:10A59000D7E8F4F3EBE2CEAC7F534C5139407F5710
:10A5A0000A183F79B0DBCA80A8F3E5CC9E63404728
:10A5B0004F3D1A01060D1B3C78B7E0C97FABF8EBA5
:10A5C000C9915D3C3C46351907122234578EC1E3D0
:10A5D000F4D1AAF5E4C08A573D3E402A11070E186F
:10A5E0003772AFD9F0F7FBF3E0CAAB835B4A504D4B
:10A5F0002F0F040A1C427EBBDDEDF2EADDD3C6AEAE
:10A60000875C46483B1A05060D1E4C94CDDDE5EFF0
:10A61000F1E6D7CAAB7743363B3221171F273357B2
:10A6200090B6C3D1C0ABF8ECCEA56C321F29291E61
:10A630001E1D1D32639ABCCDDEF4FBF6EFD7A5607C
:10A64000291F292A1D181E2E4A7DA8C2D5DFE9F12F
:10A65000F2E9CA95603E34301D06060E1A4286C3E2
:10A66000E6EFEFE8E4E1DBC1905A3B332612010646
:10A670000D1F519BCEE6F1F3EBE1DBD0B482523BF0
:10A68000342A1201060F2866A6D5EDF4FAF4D9C4CF
:10A69000B7A1784C3A3B3041540A1A487CA6CAE12B
:10A6A000F0F3EFDCC1A4835E40353E391D0C0C2471
:10A6B0004C73A1C9E1CAABF6E2C59E6C3B3544467A
:10A6C0002E100A11245AA2D0E4ECF6EFD4C9C0A48B
:10A6D000744D46514043520A16438CC5DDDBD2D738
:10A6E000DBD3CABEA7794F3A3B2E3F540917449695
:10A6F000D2E1DADCDFDACABDAE8B543440595738C8
:10A700000E05174A92C1D8DDE2DED0C9BDA5764359
:10A710002E3D53502F0D0A2162A4C6DAE8EAD7BDB8
:10A72000BDC1B07B473139443B2009164486B4C9CA
:10A73000D0D0CFCACCD2CDAB6F37242A34342E241C
:10A740002E5789B2C7CED3D7CFC4B8AB8D5C373CB8
:10A7500053614D291A2B567FA7CDE0DFD4C3B1A694
:10A760009C84593D4561643E140E2F628EBFE5E323
:10A77000CAB4A8ACB1B19E734B4147401E0C2A5DD0
:10A7800083A0BBCDC9BFB8B9C0C0AF84553F3F3C63
:10A79000270D0C285A7FA2C9E5E7D7CAC5B9A88DED
:10A7A0006B4D495655370E0B2E5E80A1CBEAEFDA82
:10A7B000C4B6AA967F604B4D534B24060F3165916A
:10A7C000BBE1EFE7D0C5BBAB997C604E494C381577
:10A7D000051438688FBDE9F1E1D0CBC3B39173584C
:10A7E0004842391C060D2E668DAFD3E1DBCBBFBDD1
:10A7F000B1A79A7B5F4E4537190315406E8FAECCDB
:10A80000D9D8CBC3C2C1AF8963493C321909091CED
:10A810004C8AB6D5E4DFCCB3ACB8C1B792684E452C
:10A82000371C05061C4680B9E1E6D2B9A59AA6BD3B
:10A83000C09D73543F2335531333619ADDF2DEB765
:10A84000A0979CACBAB1906E5D4C270F172F48684B
:10A850008FB9CDCABDAEA6ACB9B591684D423C34F6
:10A8600036415265758EABBFBFB4ACB7C2BDA681D1
:10A87000613E28252E36425170899BB1C1C3B8ADC7
:10A88000B6C9C7A57E634E3C25161D334E779CB0D6
:10A89000B4B8BBB6A6A5B3B59F7F685C4D341E2186
:10A8A0003863899EA0A2A8A9A1A0AAB8B6A0816772
:10A8B000503B261C2B517B9BAFAFABA39EA1A7ABFC
:10A8C000B2AC90725B452F22273E5F87ABBCB59C34
:10A8D00084828EA6C2CCB995694E311B1A2B487260
:10A8E0009CBDBDAD9E948C92A8C1CAAE7F50362D42
:10A8F000272B3E617E92A3A9A69C97A7B7C5C8B691
:10A900008F65432D2525354E697A869DB4B3A6A45F
:10A91000AFBBBEB5A27F5B493925202F4F65758B34
:10A92000AEC5C5BDB5A79BA1A9A1846A5435415048
:10A930000E2A5886B7DAE1D7CBB6A4A3ABA4907D94
:10A9400064481D3251133F7696B3CED5CCC0B9B50D
:10A95000BAB79E8069583C45500929597B93ADC0D0
:10A96000C8C7C7CBC9C6AA82624C3C291004143C94
:10A9700067829FB7C9CCC9CED8D1BA9F7F644B3705
:10A980001F0A071D426285A4BECBD0D4D8D5CEC045
:10A99000976B544A3C1B0205153A729FBDC8CDCD3A
:10A9A000C2B9BBCBC5A88069583A444F061136726C
:10A9B000A4C1C6C7CCCDCAC9C9B7926C5A4C303EE7
:10A9C000531939567195B0C4C4C0C4D0D0C19E7C4F
:10A9D000655A4D351B1121406382A3BCC5C3B7B670
:10A9E000C2C9C2A87E5A47361E060824578CB0C377
:10A9F000C9C9BCA89A9CAFB5A385735F444B4E0EE2
:10AA0000316695B2BCB7B6B3AFABB6BCAB92745DB2
:10AA100045270D0E2A5A86A1A3A4B4C4BEB0AFB276
:10AA2000B29B7E6E5F50361D1C395F7D929595A35B
:10AA3000BCCECABCAFA183645153543F2D2E466E89
:10AA40008B97969CB0C8CFC2B2A1856A5A5B6059F9
:10AA500046373748668A9A969CB8CEC9B7ADA79351
:10AA6000796463654E2D2131517D999E9A99A5B5E2
:10AA7000B6A59D9A8778757A6F4F383B465F7F936E
:10AA8000918084A3C2C4B4A4917F73777F73593F2C
:10AA9000323D658C9B8B808EACB5AC9C8E867C7C6D
:10AAA00086826A523B2E3E6E9DA794838597A1A015
:10AAB0009FA19F9B958C7A57372735547D9B947D1A
:10AAC0007487A4B4B0A18C7E7D78777465534C599B
:10AAD00076878F8A7F81A1C0C8B090817A707275A5
:10AAE000684C3B40526E898D7A7388A9BFC9C1A753
:10AAF000897474797A74624E43506E84806364837F
:10AB0000ACC6BEA8896E68798D9E8D7462544E6005
:10AB1000746F565A8BC0D3C3A07D625E718B9289CD
:10AB20007969666D7C7C65474B74ACCDD0BC9D7FEC
:10AB300074757C7E70635956657F7C5D404C7FB137
:10AB4000C8C9BCA7938B86807A7466514A596D6ECA
:10AB5000574D5E83A6BBB7A69DA6B0AD9E886F522B
:10AB60004143525E6765637493AAB0A39EA2A19706
:10AB70008A7B6658546075817E684C486E9DC1C85A
:10AB8000BCA593867D6E62585A656E797E6E584A72
:10AB90005983B7D4D1B59E9088785E5764747D7A16
:10ABA000736857464E719FBCC5B49984828F90825A
:10ABB000797B8177624F483F405A89B5CBBFA990D6
:10ABC00081879FA287675962675F595F58536A9868
:10ABD000C1C9B598837B8B9A96856A585A65686512
:10ABE0005A50506A9BBFCEC4A48F848284837968F4
:10ABF00060676B685136304A75AADAEDD6AE91843B
:10AC00007F858C8774676D644525141E437BADD3A7
:10AC1000E3D4BAA9A2948B8476655C60665C3C261A
:10AC2000274E83ACCCDCD4BFAB9C958871615A5C59
:10AC30005C524C423C4E79A8C1BEAFA39B9C9FA2E4
:10AC4000957C5F50595D524847516285B3D2D6C05A
:10AC5000A693898C94876F5A6067563E2A23375D86
:10AC60008BBED5D9D0BCADA6A9A1887064645A4565
:10AC700024131B3D6A91AFC4C3B8B1B3C1C5AF8D36
:10AC8000705C4A331E191F406A95B8C3BCB2AFB599
:10AC9000B6B6AC8D665157614D342622396397C1E3
:10ACA000D0C9BCB7BAB6AA9677574F585F593C225D
:10ACB00021396BA5D2EAE3CAB39F958E7F6E656595
:10ACC000685E3C180E22558EBEDAE3E0DBCBB2990B
:10ACD000857259454A5A5C41282239608CAFC4CBF1
:10ACE000D5DDD8BE9C7657454354636358413A52EC
:10ACF00084B2C1C8CDCFC5B2956E4E43495768687E
:10AD00005D40263773B4DCE4DCC8B2A8A189705B6F
:10AD10004E494748484235355187C4E3DFC7BAB684
:10AD2000AE9C8F7E644E474D493D322D386BAAD67E
:10AD3000DDCEC6C6C0B3A2835B3227323F505A4C29
:10AD40003D4F8AC2D8D5CECBC9C6AD885B3B29243E
:10AD500033536559363062A8DDF5EFD4BFB5AE9AEE
:10AD60007A604A3A3331404F46323970BCBBB0DF6B
:10AD7000B8A1A09B928B7F6C4D3329262C3535537F
:10AD800093D9C7A5C49F9DA9AAA1977C58371F2412
:10AD90003639384368ABDDEDDBB39AA2AEB9B19377
:10ADA00070523D34281C1B224680B3D9D9BFA6A1BE
:10ADB000BBD5D9C5965F3B2D21140D122F598BC3DE
:10ADC000DFD3AF939ECBF0EABF80553D20110E0F2D
:10ADD0001A2E558DC3D9CABBB4C1E3F4DC995543CF
:10ADE00041280F0715252D4786BCD6DDD0D0E8FBBE
:10ADF000F0C97F5446290E020511202C446F96BFDE
:10AE0000D7E2BB80B3F1B76E4F37444C102E413BB5
:10AE10003A48668AB5DBC18080B1E2A5692D394C1C
:10AE2000091A302D24294179C3BB807F807FA7B3C5
:10AE30005B1902050E1729302B2B3252AFC57F80CC
:10AE4000807FB3D8812C07050E14222A2B2B304388
:10AE500091B4807F8080B3E3983D0A060D141920D9
:10AE6000252C313D7FA87F808080B5E3A25D1D0445
:10AE70000A111A1F262B30376E98807F807F80AA98
:10AE8000C6765B4A060E161C22282E3666937F80F5
:10AE90007F8080AFD485323F4A0A111A20252C3298
:10AEA000608E7F80807F80B1D88A482509050E1486
:10AEB0001922272E59867F80807F80AFD68945262C
:10AEC000444B0A121920252E6190807F807FB5EFB8
:10AED000BD755C4F554C0910161D242C74A77F803E
:10AEE0007F80B3EAB26856542901060D1519223342
:10AEF0008BB8807F80B6F9E4A151514D4F4A080DBF
:10AF0000161C265D89807F807FB4F4DD9A5C6059D1
:10AF10005B7F4A080D162A77A2807F80B4F4EDD6B5
:10AF2000BB745B441F3A804B0A112B7AA4ACE3B389
:10AF3000B3F4E5B2898462341B0B080B0C13307A2E
:10AF4000C9E1E7BEB6F8DC9D868D5D1C133A503F23
:10AF5000313E76B8CFC1D1EFF3E5B67A65502941DD
:10AF600059384B445790A2A5C8B8C8D4C6A88D700C
:10AF70004F37322D2D3B5D9AB4C2E2DDAC85899FFF
:10AF80008A5540413B1D08327CA5B7CAE5F0DEB0CA
:10AF90007A68829373432C2820090C3B8ED3EFF9F7
:10AFA000F4EBC38072938D5120182628110A205C7F
:10AFB000A9E1C4B6F8EEC38E8E9F823A3B80480664
:10AFC0000D183A8BA5807FB6F9EECD9B9284494D42
:10AFD0007F49040912192F7298807F80B5F9EAB76A
:10AFE000744A253D501112121924478F9D80807F8D
:10AFF000B6F8E3BA9B685580571D111218244C818E
:10B00000C6C28080B7F8E7CDB57C627F8048060D68
:10B01000162A64AAA480807FB3DBAEA39A524A5456
:10B020001D110C131C376CA3A280807FB5E7C3B23F
:10B030008A3617352C0A0A0F15204BA3B5807F805E
:10B04000B4F5E2B7735D7F500F0A0D151D22407FE6
:10B050009B7F807F80B5E9A744404C0A0C111A2AD7
:10B060005A8796ADA480807FB5F4E6A74309080609
:10B07000060C1120447BA3D9C3807FB5F4EDD28D9B
:10B080004B363D2641470514375D74ADB37F7FB520
:10B09000F5EDCE7D36445863804910396C82AEE2BE
:10B0A000C1B5F4EDE6DEBD644C51144246041F60A8
:10B0B00093B0D9F2FCF3ECE3D6CA9D4F4C7F80806D
:10B0C000481C6DB1BBCBE2EEEDE6E1D7C5913D1575
:10B0D0001A18447F491A66A4A0AADCF9F4EDE4DF4B
:10B0E000BD5A427F807F4A0914368CA88080B5F60D
:10B0F000ECCEC3D2B75F4D80808047060F3681CD3E
:10B10000BB80B8F7DFB2A3B08B3D42807F4A0A1103
:10B11000214E8ECEC27F80B4F5DB9C5A2D458048EF
:10B120000A111A45ADBFB6C480B5F5ECE5D49A4B0B
:10B130004E807F80480A0F257CA97F80B7F9F0E90F
:10B14000DCAA4D497F8080490B111A2A7DA9807F96
:10B1500080B5F5EEE7C4694D7F8046050F131C4AA4
:10B160007D80807FB8F8F1E9DFAC7C7F8080470686
:10B170000E15246392807F80B5F5EEE0A9524D7FD5
:10B180008046050E151E497B7F807FB8F8F2ECCF14
:10B19000805F808045060B12193489AA807F80B5B4
:10B1A000F5EEE5BC722E418080480A1317369FC227
:10B1B0007F80B8F8F1E8D08C373F7F80480A1118BB
:10B1C0002478A77F807FB6F5EFE9CB725380807F2C
:10B1D00048091219286F9D7F807FB8F8F1D79540F4
:10B1E000468046060C121928608C7F807FB8F8F3E1
:10B1F000E6C28C504D7F80480A0F1638A4BF807F6E
:10B20000B9F8F1E9CA82411A3C8045060E16236955
:10B2100097807F80B6F5EED78D31427F80470B1245
:10B220001A214D7D80808080B7F4DC9B5D3C537F8C
:10B2300048080E161C2875A2807F80B8F9E19E4947
:10B24000507F470A12171E232946A6C37F807F809E
:10B25000B7EEAE768044060D141922273681A980F8
:10B260007F807FBAF6D170527F47070E151E232AC2
:10B27000527C807F807FB9F2CEA371634603080DB4
:10B28000161E242F779E807F807FB7EBCB9E575072
:10B290008046060E161C23437180808080B9F2C25E
:10B2A0007D505E7F480913181D242E76A07F807F75
:10B2B00080B9F4D28E4A5180460A0F161D2444727A
:10B2C000807F7F80B8F9F0DD966A807F46060E1594
:10B2D0001D2774A07F807FB9F8F1E4B14E46807FCE
:10B2E000470912171E3293BA807F80B9F9EAC47AEF
:10B2F000647F45030A11181D2446777F807F80B93B
:10B30000F9E29B3B4280460A12171E233999BC8002
:10B310007F807FB8EEB651487F470A11161E233052
:10B32000769F807F807FB8F5EFC4563F7F45060C3F
:10B33000111A203088B0807F80B9FBF5EBB7827F8F
:10B34000807F490C111A1F3899B97F7F80BAF9F1B3
:10B35000E9BA84807F80480D1119215A8680807F48
:10B36000BAF8F1E8C9765E7F8045050F131A33827B
:10B37000A17F807FBBF8F1E0B2682C152115020691
:10B380000E1846A7B27F80B9F9F0E9C97B260824D8
:10B39000405D4507113082C9B080B7F7F0EBE3BBE1
:10B3A000584747242C4C470C17499BA4807FB9F77A
:10B3B000F1E8DDAD534D44043F44060D3082DCBF5F
:10B3C00080BBF8F1E8DFC691502D2E214480430860
:10B3D0002B7CD0BCBAF9F1EADBAF836F655A451B11
:10B3E0003E8043104C9BD4B8B9F6F1E8D5A87B6BEE
:10B3F0007982645E80807F554D8DC6F1F9F3EBD57F
:10B40000B08F787493AC87717F804433768EB7EABF
:10B41000F0EBD8B49A8C6C6893AA7E6980805756FA
:10B4200091B3DCEEE9D7A87D6F695F68858E6427EC
:10B43000437F697DC3E3EFE8DFB36E525C5E51503A
:10B440005E583D2325497AADD7F0F0E9DEB96C2F7F
:10B450002138586552301C2C5785AAC7E3F2EFE912
:10B46000D9B072391B1A31453F28152669ADD2E88B
:10B47000F6F4ECE5CEA4754F3C301D454416364E2F
:10B4800072B0DDF4F8F1EADFB97F583E2F29231AB4
:10B4900018253D5980A6CFEFFBF5EDE2C2834E366D
:10B4A00029103F420A2C5F85AAD1B3BBF9F0E9DA33
:10B4B000B279553B163F804206133E83C4B17FBA32
:10B4C000F6F1E9CF996D614857808042060D2E7DD7
:10B4D000D8BE80BCF8F1E8D4A4765D384F807F43B5
:10B4E000060E2C7BD0BA80BBF9F0E9D2A57F5F2E87
:10B4F0004480804408103B96A6807FBAF5ECE5CFE7
:10B50000AC86552142808043051449AFB57FBDF814
:10B51000F1EADFBC9575404A80807F450E347BB9E7
:10B52000A780BBF9F0E9D9AF7E56304B807F450A42
:10B530001E508EC5B17FBCF9F0E9D7AD7B44527F78
:10B540008080440C3173A6CEB67FBAF4ECE6D9AC59
:10B550006C3313418080450C346EA0DABEBBF8F228
:10B56000EDE3C7945D301040804205164078A4DCBE
:10B57000BFBBF9F3EBE3C68940110B12464305212B
:10B580005D87A4D5BABBF9F0E4CFAC773349410C61
:10B590001610184177A3C1E2B9BBF4E7CBB29A6D9C
:10B5A0003712438041092F6EA2BFDEB8BBF3E1CC56
:10B5B000BC9D764C2B11438049244F81AED2ECF8D0
:10B5C000F5E9CBAB9D8B6B3F21100B0B18325C86E2
:10B5D000B2DCF6F9F2E5C09B836C4C290F050A1822
:10B5E00036608AA9C3DFF6F8F1E0BC9073523219D5
:10B5F0000F0F1C2D476F96B2CCE2F2F5EAD2AC8366
:10B600005F3F28170F142440628297ADD1EEF7F107
:10B61000E1BE90684833210D01123762829BACBFB6
:10B62000D3EAF1EDD8AE8057361E110808153D71EA
:10B630009AB0BBC4DCF0F1E5C9A5784A271612120E
:10B640001322477CA2B8C5D4E1ECEDDFC49A683C74
:10B650001D09061122365681A9C4CFDCECF1E4CDD8
:10B66000A77E4F2A110A101F32507194AEC0D1E14B
:10B67000ECECDFC79D6F401A444616283F5A7B9674
:10B68000ABBED3E2E9DFCEB79970441E0707163789
:10B690005A738496B0C6D7DFDED5C2A07D57381F57
:10B6A0001214294767808D9BAEC3D2DBDAD1B994DF
:10B6B0006D4D352617152246718E9DA7BED7DDD656
:10B6C000CCC0A6805F49311A0C1634577C96A3A8CB
:10B6D000B9D5DFD8C6B69C7C5D43342720203361C2
:10B6E00094A9A5A0ABC4D6D6C7AC8A684E3F352E68
:10B6F000272B406A95AEB2AEB3BCC4C2AF977E648E
:10B70000513E3B4144434C688EA8B4B7BDBFBCB367
:10B71000A88E6F54464041424954627A92A8B3BB06
:10B72000C1C2BAAC947A614F43403E434D5F7686C6
:10B7300098A6AEB9BFBCB5A8927C624C3E383A46DA
:10B7400052627488A1B0B7BABFBDB7A78E7A654FF1
:10B750003A3034455A6D7C8394A5B4BCC0BEB7A4BE
:10B760008B715F5144313148687B7C7B8295A5B5F4
:10B77000BEC0B9A4886F635A4C3E3B5575847D7238
:10B7800074869AAAB6BEB79F85727170614B435694
:10B7900073807B7277869AA5ABABA6968174757B16
:10B7A000725E50627B807065708899A2A7A79F8A9D
:10B7B00079757679736C6A747E7A716D79869092F8
:10B7C00096938D857C7A7978726C717C817D7278A4
:10B7D000858B8A8B8D8A8074767D7F7A7277828B57
:10B7E0008477717C888F8E8F8D81706B727B7C7576
:10B7F0006F757F857F77788593928D8C897D6D6A53
:10B8000075817E74717D84837A777B878F9496901F
:10B81000887C716D727C7C767680827C6F727F8C86
:10B820008E8D8C8A887F7472767B79767C81807726
:10B830006C7183919694908E857C76777877757B02
:10B840008483786A646F80939C9B968D857E7777DE
:10B85000797877787C797062616E82929697979208
:10B860008C837F807F7D767573716B656675838E43
:10B87000949697939088817C7C80807D726C6562C1
:10B880006772808D969796979288827F7B7C7C7773
:10B89000716761636D7C848A909396908B85827CBE
:10B8A0007B7D7E7A6E65666E797F868E9394918CB1
:10B8B0008580807F807F80776D656A727F858A8CC6
:10B8C0008D8C8D89847F807F80807E796F6A6C7695
:10B8D0008184858C8F8F898480817E7C7877757355
:10B8E000706C717C888D8A868185888781807F8154
:10B8F0007F7B726E6C707580888D8F8E87837F8062
:10B900007A7B8083827A716C70747B8085888E915B
:10B9100090877B76767E82837F7B7270727D828455
:10B92000818589908D857C77787D848581796F701C
:10B9300078848A8A8684838686807B797B808384E8
:10B940007F746B6E7681898A867F818487807C7A1A
:10B950007D8082827B757475787F878A867F7F8001
:10B96000837F7B787B8080807A75747B7F82828501
:10B970008481808081807B797D7F807F7F7D7F81D6
:10B98000858683827F7E7D8080807D7D7E818080B4
:10B990007D808283818281807E7974797D7E7D7EC7
:10B9A00083817C75787F8485868986837F797779A2
:10B9B0007E7F807F827F7B767680888D8D88837F77
:10B9C0007D7877797D7B7A7B807E7773747C8187C5
:10B9D0008B89848483807F807F807D7F7F7F787563
:10B9E000767C808686837F7D7E7E7A7B7C7F7F7E71
:10B9F000807F807D7C7F848988868382807C7B7940
:10BA00007B7E80838080807F807F868A8B84807B22
:10BA100079757472787D80808080808180868B8D3E
:10BA2000877F79797A7C7A7B7C7B797C8082817F45
:10BA3000848A8E89817B797A7B7C7B7C7978747827
:10BA40007E848480868E938E847A787B7F7C7A78DD
:10BA5000797875777A7F7F81888F9089807D7E80E5
:10BA60007F7E7C7D7A787575767D81878B92908BD1
:10BA700082807F7F7B7A76737173787B7F81868CFF
:10BA800094938E84807E7F7E7D7D777474747478C9
:10BA90007C80858B92918A8480807E7D7B7A75768E
:10BAA00078797A7A7F818387898985817F807F8091
:10BAB0007C797676777678767A8189908F88858298
:10BAC000827F7D7B7D7D7D7C7C7B78777980898F93
:10BAD00089817C7E807F807F7F7D7B7A7A7E7E7F7E
:10BAE0007F828689837E7C7F7D7D7E7F827F7A795F
:10BAF0007C808181858889857F7E7E7F7B7B7C7F42
:10BB000080807E7B7C7E8080868988807C7A7D7D3B
:10BB10007C7A7D7F81817F7F7C7D7F868B8A867F1B
:10BB20007A797D7D797674787D818081807E80854B
:10BB30008D8D887F7A797C7B7876787A7E7F848514
:10BB4000857F7F868A89817D7979777475787D7D17
:10BB50007C7F8285838284848987837F807C7774DD
:10BB600075787A7F80818183858686858582827FCC
:10BB7000807C777472767C807F8080808587898ADC
:10BB800087837D7D7E7E7977777A7B7E80838181D6
:10BB90008184868682807E7D7D7979787777787ECC
:10BBA0008185858484868584808181807D79747691
:10BBB000787877777C8083828180817F8181817EA4
:10BBC0007C7A7C7D807E7D7C7F808686868386866F
:10BBD00083817F7E7B77767D7F807E7A7C7F808489
:10BBE0008587868281807F7C797A7A7E807F807D5E
:10BBF0007F81828381848687817F7C7B7879797A53
:10BC00007C7A7A7B8080807F848784838081807E39
:10BC10007A7A7C7E7A777C7F817F8083878887832E
:10BC2000817F7B7A79787C7C7B7A7E807F807F8243
:10BC3000868987858383807E797A7B7B77767B7F15
:10BC4000807F808286888784838281807F807F7BDB
:10BC50007475787B7B7F81888D8A857F81838180E5
:10BC60007F807E7A7474777A7C7B7F858B878382F2
:10BC70008180807F807F7D7877777B7C7C7C7F87ED
:10BC8000898783838281817F7B797A7C7A7B7C80C0
:10BC9000807E7F82828483848688827E7C7C7A7B9D
:10BCA0007B7C7A7B7C80818584837F828583807E98
:10BCB0007F7D7C7B7E807F7E7E8081828080818490
:10BCC00083807E7C7E7D7C7B7A7C7D7E808284828C
:10BCD0008183858684807D8081817C7A797A7C7D70
:10BCE0007F7F808080808384857F7D7D7E7E7A7A61
:10BCF0007C7F7D7E7D7F7F807E8085858481828341
:10BD000084807E7B7D807F7E7C7F7F7F7E7E807F48
:10BD10007F808084837E7A797D8080807F7C7E7E38
:10BD200080807E7B787D8287857F7D7E8081838217
:10BD3000807E7C7A7D7F7F7B7A7E82837F7C7C8025
:10BD400081858684807F7C7A7C7F7D7A777C818305
:10BD5000807D7E808383828282817E7A7B7D7D7BF3
:10BD60007E7F807F7C7D80818383838381807E7DD5
:10BD70007C7A7B7D8080807B7A7C7F8082848484D7
:10BD800083817F7E7C7A7C7F8384807C7C807F80C3
:10BD90007F808080807F807F7D7B7D8182817D79B7
:10BDA0007C7F807F8081807F808080807E7D7F839C
:10BDB00084817D7B7B7D807F807F807F7F80808092
:10BDC0007F807F8283807C7B7B7E7F7F8080808082
:10BDD0007E7E7F807F80808382807F7E7E7F7F7F6C
:10BDE000807F807F7E7E8080808082817F807F8058
:10BDF0007F807F7F7E7F7F807D7D7E7F8081818150
:10BE0000807F807F807E7E7E7D7E7F7F7E7D7E7F49
:10BE1000818282817F7E8081817F7E7E7E7D7E7E2B
:10BE20007F7E7E7F808282807F7F818282807E7D16
:10BE30007D7E7F7F7F7F7F80818282818080818104
:10BE4000807F7F7F807F7E7D7D7D7E7F8080808004
:10BE50008082828280807F7F7F7E7E7F7F7E7F80E8
:10BE600080807F7F80828281807F7F7F7F7F7E7ED8
:10BE70007E7E7E7F807F7F8081828281807F7F80C7
:10BE80007F7F7E7E7E7D7E7F7F7F7F7F81818181C0
:10BE90007F7F7F7F807F7F7E7E7E7F7F807F8080B1
:10BEA000818181807F7F7F7F807F7F7F7F7F7F7F9A
:10BEB000807F808080808080807F80807F7F7F7F88
:10BEC0007F7F7F7F7F7F8080808080807F80808079
:10BED000807F807F7F7F7F7F7F807F808080807F6B
:10BEE0007F807F80808080807F7F807E807F7F7F5B
:10BEF0007F7F7F807F7F7F7F7F7F807F7F807F804E
:10BF00007F7F7F7F7F7F7F7F7F7F7F7F7F7F7F7F41
:10BF1000807E807F807E807E807E807E807E807F2F
:10BF20007F807E807F807F7F7F7F7F7F7F7F807E1F
:10BF3000807E7E7F7F807F7F7E7E7E7F807F7F7E14
:10BF40007F7F7F7F7F7F7F7E807E807E807E807F01
:10BF50007F807F7F7F7F7F7E7F7F807E7F7D807EF3
:10BF6000807E807F7F7B807E7F7D7E7F7F7F7F80E6
:10BF70008182807F7E787A7A787A76758080807FF9
:10BF8000807E807C808180747B8088837B788078D1
:10BF900074787F7E79818288827A78797874707CEF
:10BFA0007F7F7C7F858C80857E777A788188807999
:10BFB0007877817F7F807173797C8B8784817A7CAD
:10BFC000868280766B776C8084867F807F8E817E90
:10BFD0007778766D658380857E8C95826E67757FB8
:10BFE0007764747A7F869DAB976C67627D73645EBD
:10BFF000746A8B99B3A487837A7571605E615B7094
:10C0000097B0AA8E8D937F73544D48506191BAC5F5
:10C01000BDA7AA8E8559351217284E90CEF2EBCACD
:10C02000ACB7AA6B1B01061026A3E8FEB67482DE2D
:10C03000CE8D1B0B130165F6FDC14232B9F2CC590E
:10C0400004080E0CC5F8C2430455F9FDD6420A1681
:10C05000397DF09C400526C9FFF37017066B96D416
:10C060009D510B0843E2F4DC1D0926D3D8AD2919F4
:10C070001E31B9EEE962071BAFFECE401233443ADF
:10C08000F6DFE6280820DFE59804116D3D98EAE523
:10C090009E571A9BE2D440122D7702B0E2FEA649C9
:10C0A00000C7E4C82716596238B5D9F898244FE676
:10C0B000F39A1D1B5B5263BBFDE2650075EAFE7FD0
:10C0C0000907608CBCD7E6B52D22D5F0E92E011EFC
:10C0D000BBD6D28F736B1F83E6FDA4240049EFE02B
:10C0E000C33B2B4D5CCBDDDE2210069FF8F494138E
:10C0F0003765B8D4F5B3112A2ECCF1E0481141A62A
:10C10000EDF4FF8C0F0D41D5EBC4180E54D2FAFBA1
:10C11000EF64080C67FBF686021181FEF4E7C9584C
:10C12000140058F2E772070E95FDF2C8975D120DE4
:10C1300065F8E3510813BAF3F3A4766817118AFB84
:10C14000D93E0023C5DEE972808B151D90EBD32B01
:10C150000A1EEDCDFC559E64081EB9E5A000025FE5
:10C16000FDD6F60BB145052CB7E498122068F7C44C
:10C17000CB3EE63A0F18B1EC9A1D1854E6DBF529D0
:10C18000A2000F14B5E392262761F0D4BA0F6525FB
:10C190003017B2DB7F260B57DDCECE253E31260988
:10C1A000B6D561050047E9DCFA2D2A3E4F1FE5C4EC
:10C1B0004A01087EFDD6D90C2C66853BB6C32903FF
:10C1C0000699DEDBC32C3381A32D838B110F1BBC9F
:10C1D000DBDEC21F4193D8475966241520A7DCDD5A
:10C1E000C2203FBCFC57393F3014039DCCE3D13E05
:10C1F00030C7E44C0B132C111EB2E7EFFB5C30F19F
:10C20000DD6E0005080121C2E8ECEF632CD2E28963
:10C21000190B020A2BD6F0F3EC7002C3D7AE2E0D29
:10C22000070956FEF9F4EC870BCDDCB722130F1784
:10C230004FDFFBDDF2B015ADEBBF4A01210B38DC5F
:10C24000E4C9EBBB0D97FBD2670D2C074DD0E7B3CC
:10C25000EBD33E87EFC97E06190051D6FCB5E3FD4E
:10C26000686BD5CC850D00004DD0F3BBE0F88D3B5D
:10C270009AB1B135030D4DC2F4D4D0F8A82659A512
:10C28000D76413152EB0E0E5BEF2C64B0FB2CDACAD
:10C290000C200092D5FAA9DAF9622A9BDEAB001FC6
:10C2A0000289C3E591C9E4871983E6C6260E0653C1
:10C2B000B6EEBEDBEF890A66D7FB41170133ACCD82
:10C2C000E5DEFC8F3325C6DC5F03032391C3FCDB73
:10C2D000EBA25529CBD79B00161091A1E7D6DFB270
:10C2E000731F8EC7C431051B527AD8E3E0C382079F
:10C2F0005BAAF270020B2366D0F7EAC89A31389530
:10C30000E9AB010B0A42B9FDE6CEB4501572CFBDC0
:10C310000100012B9CFAE1DDC06D1646D9D84D0015
:10C32000050E91FEF3EEC4800C2FC0EE8511000DBA
:10C330006CFFFAF5D777350CAAEECC39120541E13E
:10C34000FDFAD06C4C03A5E3E65608021AB2F4F3EA
:10C35000E17F51155CFAF5A3070D068BF2ECF57D34
:10C36000560034CDFECB2E070461F3DFE48347177C
:10C3700007A4FEF3640F1936D3E9E0A74821058B23
:10C38000FBFE9C14170BAFE5EACF60160F4AFDF6D3
:10C39000CB05130B6CEEE8E98B1B2230CAFCE94E8F
:10C3A000051345F1EBF9A619272A88FAF88704291D
:10C3B0001FBFF8F1C9181E3A52EEF5CC24130383BF
:10C3C000E9F6DA4E0B473BD6F7EB390F0F3FEEF2AB
:10C3D000FD80143637A0FCEE91011417D3ECFAB2AD
:10C3E0002D1A3358E5DBC423190B86FDFDDB550AF6
:10C3F0002151CADEEC630B0938DCEFF694021948D0
:10C40000BFE0E5A610120EA5EFFDC43D00569FE16A
:10C41000F0D8030E0C63F6F5FC69005581CEF5EA01
:10C4200070001829E0ECF9AB1B4098ADF7F4A913A4
:10C430000F139FFAF3D1072E69AAF5FCFC4C0403F5
:10C4400042E4FDE766007CADD8F6F17B050F0EB83F
:10C45000F1FD8D105EBBDFF8F4C40008075EE2FE5C
:10C46000DB3F35DBB8D8F6EC6C041C17B3FEF06D7F
:10C470001492C2CAF7FCB31C160A61F7F9B3004A5A
:10C48000B39FE0FEFC51191229BDF5D63F04B2A1BD
:10C49000B4FEF9B1142F0174F4FB8A0A829993FE59
:10C4A000F8DB3E0E121FD0F6CD2B3D8491CDF2F479
:10C4B0006E002710C1F2E43F1358A0BDE2F6BA2582
:10C4C0001B1565EBF9932623969AC3ECF0512010C7
:10C4D00029BDF4C65F02579C8FF4EEB3051D03849B
:10C4E000F2FB971B1D8A9BF3F4BC25070A37DCF38C
:10C4F000E356035AA6D3F1EE5D011C1EB9F3F39384
:10C500001434AAAFE5F9B529070F74E7FDB4391261
:10C51000908AB6F8EC52140D29C7FDD67B0B4593D3
:10C520007AF7E2BC0A14038EE8FCBD2C228183C397
:10C53000FFD6520C0913D7F5F86008618B9FF9E715
:10C540007A002110B4FBF87E08367E7DDEFAC8281A
:10C550001C007FF4F8BB30276B5885DEF86F0C2D7C
:10C560006EEDFAA81A043AA8F4F8DF4A030739D99D
:10C57000FAE356093970BBF1FC97102E1499E7E7DE
:10C5800078011055CFFDFDD83E02014DE8FEBE26D4
:10C59000073180E7FCF48807120788E2FDB3190E23
:10C5A000619EE9FDD518150C42C0E5E26328577A73
:10C5B000C3F9EE7E020D01A1DFF5A0252C7799ECE1
:10C5C000F4B6181E097ADFF9BF3E144D86D4F9F788
:10C5D0006802202EB0D6DA7B0C3D7AB6FDFCA212A2
:10C5E0000E0B91DAE7AC2D1D5B8FEAFEE21F0C0803
:10C5F00054D2E9DB5D145474C6FEF48F020903AB18
:10C60000DEEE9B222272A2F4FAB216150A79ECEB46
:10C61000D247116487D1FCF660060D3AC7E6D76EA3
:10C6200003497EB5F8F8AA151B0979DFECA3381584
:10C630007089E9F9DE37060358C9D0E261215979DA
:10C64000B5FFF583031C070176BFE4CB462F768A3E
:10C65000CFFCDE5206192FC4C4DF66434F67A0FB30
:10C66000FDB21A050975C7E4A642366C88DEFFEDF7
:10C6700036241130AAC4D76C286B8EC3FEF1830612
:10C680000515A1C7E4833C53838FE8F9C21B270833
:10C690007CADDBB9322A8088CEF6E6520B202FBF64
:10C6A000D9D1681B4E8EB8F1FF961112087CC7D302
:10C6B000BD4D4D7F78C1FBEB5C03193CBDB8C9692A
:10C6C0003A6E8A8CEEEFA1171717748BB48C5C7BD3
:10C6D000B8D88F70251C1088D1E0735A458FD2E4EA
:10C6E000B58147090248D2FAAC4C5C55B8D6E79DF3
:10C6F0008820140E8EE7E1685E5A98CDF0BF9858F6
:10C700000D041DCAF8C15D705BC1D5EA8E850D05AB
:10C710000277E3FC836A5E87C9E9AE8F5F03062E6A
:10C72000ABECBD626C6AAFD5D4869D280A0154C4B7
:10C73000ED7875717FDAEC9F9C6E07101A93F0CC40
:10C740007F936CBAD8B087A83C080345BEF7A78F83
:10C750007A75B8CE8EB78A15001281F1C08A826CC4
:10C76000B1CD8E89BC4304073FC8E473796086D796
:10C77000C47DB08B2005006DE3AD84745EBDE37BAA
:10C7800080B251050621AAD48B9C7C92D9B468B69C
:10C79000832A070A60F3C090887AABD67797C66C75
:10C7A0000C0118B1EDADA37D8EDC8F61B6A84807F2
:10C7B0000C4BE4CF9F847CA8BE6189C2821E00100E
:10C7C0009ADBB0998281C48358BEC159090138B837
:10C7D000C6A88E7E9ABB558FCCA41302038AE7CBE2
:10C7E0008C8773B67361C0D36C000231AED4A37B67
:10C7F0008AA0B765A0D0A21900117BD6D08B838008
:10C80000B03D0514668FA2C394938D9392A5787959
:10C810001128369183CCA99E799781B67F801B1F02
:10C82000327993AAB9AA858188A8A3723F0B376190
:10C830009593BAAEA66C9193B26F53144351818D08
:10C84000A5B3BD79809BA882472F385B659589BACF
:10C85000BF9467A2A1A14B393B505B7C8DA3C5A0BF
:10C860006884B5976D2B52505E619290C4A3786333
:10C87000B99B8635574D5F519B96B6A77D56B0AA9A
:10C88000865045545C5890AAA49B8261A7C78358E0
:10C890003F4C635C79BAA38A816194CD91615D4913
:10C8A000575765AFBD816F5F8CC19F596B554D5A0E
:10C8B000609DD18E524C88C4AC6F66623F576991BF
:10C8C000DAB04E3E6FBCAA897A743A415D99CDD2F6
:10C8D000583252B3A693928B3C274B9FD2DC6C18F4
:10C8E0003DA3AD93A39944222FA2DCDA88122483BE
:10C8F000B3A5ACAB541B2D8FE9CD9F21116697B525
:10C90000B4C06720167AD8D89F5307467CB4BBC7FB
:10C910007D2B1D6BBFDEA16E1D3251ABD0CA8D4485
:10C920000C65B2E3B17832193A8AD3D39A661C49BE
:10C9300093D1CF8C54111F67CEDC9C7C404086B2D3
:10C94000C7A960231052B4F1A3845D4463B0BBBA9D
:10C950006F2E024F92E7B48C7F644798A9BF824440
:10C96000093E7ABEBB9E8B824276ABC18C4D13389A
:10C970007396B3A391965453A0BE9560232F6887F6
:10C9800096B193A97E497DB48C7B46304D7F79B5B5
:10C99000A4A496666BB1857A5C4645836897A7A385
:10C9A000AD816D937B6F7E6255755867A8AEB99463
:10C9B0006B72766889756665594093B5C5A77E5ACE
:10C9C0006766908C8163453570BBD4BA80544E65E0
:10C9D0009B959C67382C58B1E4CC8B4E3F5E99A94F
:10C9E000AC662D1B56A8ECC892474C5F9BADBD7141
:10C9F00030154999DECB9355456980B0BE793E1C10
:10CA0000409CC2BD9F62517376B1C3753D2146AD56
:10CA1000BC9F8C696787859FAB6F483E4F98A17C10
:10CA2000817C81868F90936B515C6D8F8B5C678A64
:10CA3000A7939782726D5D71888273544886B8A4FB
:10CA4000A6815A596989AF8856373585D4CBB169E3
:10CA500048487EAAC982431C297FCEE3BE57303F97
:10CA600081CDD68A2D0A2785C3F9C35822407FE39A
:10CA7000D98F29012384B7F5C15D1B3F85E7DD8D83
:10CA80002F012783C3E7BB60204193E8D991360784
:10CA9000287BC5C8AF6837489AD0CD89401D30790A
:10CAA000C4A98F76565E9CC0B7874D333F80BB8A42
:10CAB0006A747B7F9EA89B7D634C5C889B6A556FE4
:10CAC0009DA99A8D846D6E6C7D9879483C6EAEDA26
:10CAD0009D7667667491A19B57252E73B8E39F627C
:10CAE0004F5D7EADC4A641092779CEE7AD523855DA
:10CAF0007FC5E6A32A031B7CD8DFA95F2C5382D80D
:10CB0000F1A426001B82D0D2A16E3C4888DCEAA0AA
:10CB100031031C85BBB8927D4E4F9AD4D798401BE9
:10CB2000377B9E978781705799C6BD865F3A5A7B3F
:10CB30007E767C848A8395AB94746A6773735C5940
:10CB40006F8A98B6A9897267789A94693C316B8626
:10CB5000AFD9B85D565481C9B15A2F185A8EC6F74D
:10CB6000CB52385287EBC6541B153998D1F5CA59A8
:10CB700028518CE9CC5C0F131D96D4F2BB5F214D7C
:10CB80009CE6CB691512238CDFD9B4703A44A1C559
:10CB9000BA76330B397EDABCA17F6558A7A3998199
:10CBA000531E4A7CB0AD8A967E838D8C7490694EFC
:10CBB00055808091829F9EAF7D60587F82776E7393
:10CBC0005B6485A0C6CF7F3A4F6BA19C8E644840C2
:10CBD00084A1DCD27F18395DA6C0A253313B7FB659
:10CBE000EFDA7B2D1E679FDDA7550D3D63C1DED6B5
:10CBF00072480E6C9EDCC061154564BED9B4735397
:10CC00002762A3B2B569314574ADD1A4865C55667F
:10CC1000A598986C4A4A738FA88F7A71717A8D9211
:10CC2000788A746D7F87838372748E89656E597E6E
:10CC300093867C8072817795AAA369575A7CA194C8
:10CC4000766962646D8FB89F7543607DB2BA8A71F0
:10CC5000645B6C95B0976B3C4F7597B495736B6143
:10CC600075A2B9A079525077859D966D63526B91EC
:10CC7000A3997F655C768F92AB8975666C80878897
:10CC8000846E5A5D687FA4A38784727B87879C919A
:10CC90007557516092A19289675873789EA58962F1
:10CCA000506790ACB3966D455B718D9C805A46641D
:10CCB0007EACC9B07B56518793A1815C4460679478
:10CCC000B3AB715A517F959886746473728FB0A11B
:10CCD0007F60556F81717C7179698290B1A394797D
:10CCE0007677765D697C80706F807E928E92888088
:10CCF00066636E9598817A7B6F8188908F69504BBF
:10CD00005F8FA394908078769EA6AA6B48315E7F51
:10CD1000A68786606A6B9DAFB2745E4E6A91A894D6
:10CD20008568566C7EA18B6E4F555E90A5A593814C
:10CD3000668B92A87C68585A607A7F89847A6D8263
:10CD400096907F8084807C777E8A8C746F6C806DF7
:10CD50005E6D848D84807A8C9D91998D8163506302
:10CD6000838E7C6D5E6F869096957874627A96A0BD
:10CD7000908066627B7E8B7B595A626F959B9E8901
:10CD80007C728B9DA4815C586965867D84826F6E00
:10CD90007C9099846F708684838C888F7C73647791
:10CDA0007B6D676B7F847F858D9A9B8F856F7C6E93
:10CDB0006D707673706C7C89999183676E7B8791B7
:10CDC000868080717E82898B7B534C6B7E928A7DBC
:10CDD0008487849093A18968495C77867E6E7C887D
:10CDE0007D7F858B947768668E938F7486847E6E44
:10CDF00072707F706C5B7C928C8791998C87737456
:10CE0000807C6A5F5580868A928E81806B6F7F9767
:10CE10008B77667591939081747066547085867F68
:10CE20006A659EA5A38E8374765D62747876695870
:10CE30008BA5958E74767E7B6A857E8D78707CA3BB
:10CE4000877E68676E75676C7885918B90A19D7DF4
:10CE50007C6E786A6E525F738E8C91818C827E8537
:10CE6000847C7F67607F8F9E8672697F697F7A6F1F
:10CE70006D765784A5BAA08263807682766E5864F8
:10CE800051668EA79E81717C8C8B8779706E6F64E2
:10CE9000849192766F60807D77777375847F859EAD
:10CEA0009588826C73836471686A6B82698F8E9EC9
:10CEB000918A758B737E7A7B758161647A8790869F
:10CEC0006E6B77728A88908681597A8B9C917553A4
:10CED00066617781847A7F616E90A6AD90645C72A2
:10CEE000748B837263634D7B95AB95765774839C8B
:10CEF000968368725D68919D957352507D859B887D
:10CF00007571766C9CA1A588654D797886826D6275
:10CF10006B63829EA29F78607381878B7C6E686A48
:10CF20006B8588947669667B79838A80798079803D
:10CF30008D9086736A636B6E847D7A777A798B8F36
:10CF40009C8C7F62696D89867F706F65717E969516
:10CF500085685471869D9585746F62769299846B0D
:10CF6000495E7F8F94927579647A96A28E77565631
:10CF70007A8B8D8A75686168929A8F806E5F7C8DDE
:10CF80008D947F6565647E8A837878626C828593F0
:10CF9000937172747D867D838378656F748A8D77D3
:10CFA00072756F7C7D8E9193746F6D808A867274BA
:10CFB000665F748A929F7E6B6D808D9E89776352C7
:10CFC0006E888D9983615D697F9B947F68557090B1
:10CFD0009A9F986F585C6D90977F614F6083979D83
:10CFE000A68A685A718C9D8C655658798B8E97915C
:10CFF0006E55637F9C9B7B6B62758C95969D74527E
:10D00000546A889483705F6584999EA59064586380
:10D01000808B917865517288958F966C656877875B
:10D020009B8D7E6171848A7D8C7C64605F738F9739
:10D03000887072848E868D937A6856657E9887771D
:10D040006672757E839F9474605E7DA29F876E5F1B
:10D0500069717E8D9A73624F7495AD9A8260637028
:10D060008A929A7962536483999C7E62576C889401
:10D070009A916E6A6E7B949A8667505C7C878793E0
:10D080007C7178718BA4937C5B5D7A83858E7F79CC
:10D0900077696F938E86676371818791928C7B6EBF
:10D0A0006A8089826E616072808D949F7F756E75D3
:10D0B000888F7E6E596B77848C9C84706E667690B8
:10D0C000977B65657A828B9D907A715D5D7D93819A
:10D0D0006C64738290989A887E685D739587755F9B
:10D0E0006476898A8F8E8370626D8E8F8871657386
:10D0F0008882838E8777595F78908E806B7785855D
:10D100007F8E8F8267606A7F8B7C71727F7B7D856B
:10D1100099917A6965738F8C7D77746A7077959130
:10D120007F6B64668D958E837C6B6D73909B876C33
:10D13000615A76928E8676716E7589A092816B6245
:10D140006C889288746A64687A95948A77696B812E
:10D15000989684706664728D918C7B66656E8A96F3
:10D1600089786E68718695938C7163667F8F8C76F3
:10D170006D5C6F7C9693957F6C6C7D8C917D7165F9
:10D18000687082909084736B7381958676736C73EC
:10D19000818C8E8D776D6E75888877746B737F86C2
:10D1A0009190847676707F817775726979798991AB
:10D1B000877F77757883837C757175797E91848696
:10D1C00073736D8085827279777C7D958B8C7B748F
:10D1D00068758281717873747B85908E8A796E70A0
:10D1E00083817C74766D78788E868B79746E868078
:10D1F0007F7977737F738E8C837A74717B7D7A7E6F
:10D2000072767B7F859785837C7A757F797672715C
:10D2100076807D94867D818279807F76777278872B
:10D22000828286717E837B797F6E77737A898B7E2B
:10D23000847A7F867C767272727479888A777E822D
:10D24000828D877A6D7674787A8784796A807F8612
:10D2500089836A727674838D8A7F6E7784808885ED
:10D260006C6D76718087868974718E808786746E06
:10D270007C727A807F7F7271858482837B797C7DEA
:10D280007B7F8080797579817F807981737E7E75DF
:10D2900080857D84717E80807B83707B7B6C7782D0
:10D2A0007D85797685807E8A817A80736A7B8583A5
:10D2B0007C6E7F837F80877C827C6C768A8482729E
:10D2C0007283807D8480797A6D728F8680766E8499
:10D2D0008C7F81847A77716C7F857E7A6C7C8B8879
:10D2E0007F85807874737D85817871708386807D79
:10D2F0008A737576727F8B777C7781858176867B62
:10D3000075796E73897C807C7F89847986827E7B47
:10D310006F6B7C80807C738382817E8E857A6E6F5A
:10D32000718A8A806D7A7C85808685776E6C6C8642
:10D330008D8579797B8B86808574736B64778C8718
:10D340007C717B8893847F7E746C69758887826C1E
:10D35000788491867B7C756E6E77878887757488F4
:10D360009089787A7A716B7277878A7F75888C8FCB
:10D370007F7577746D70717F88847B818C858175F2
:10D38000757C7C7576778587817B8581847A6D72E3
:10D3900077717973838E927D807F828070707873CD
:10D3A0007471778B9188747C83847876797D7D76AF
:10D3B00074818A8D6C7681827A76737A807D7480AE
:10D3C00090907A6E7F79807775727E7C76768C8984
:10D3D00084737A81858179767D83766F7E81857C81
:10D3E0006E8284847C787989817C778081816D7B71
:10D3F000837F7D767483827D707884897B75868651
:10D400007E79767F867C646C7C8388768286837F57
:10D410007F8087806468777E857F76817C7E83804D
:10D4200085836A687C7F8D8E777F807C86847D791A
:10D430006D64707B8E9A81798183898D807271672A
:10D440006D73858F83707E82858E7B7777746E7B1C
:10D45000828F867A7B8086867E72737571768285EE
:10D460008A8581818389847475757570777A898ED0
:10D4700081828384837B7A82807C72737F8C8382B7
:10D48000837B827E7D81827B6E6D81938D857F77AC
:10D490007D7E767F857D6E64778A968C877C8180A1
:10D4A00083858E7D735F6980958A857D7D83818785
:10D4B0008D82786C627F9A95867C77818086848461
:10D4C000766E60788D9B87828086858882817A6C73
:10D4D000636C84948B7C86858982848183766B6B74
:10D4E0007D8C937884858482807F827E736A768542
:10D4F0009088829182807E7F7A8479696E7F8C9118
:10D500008590838386817B8781736A757E918B8802
:10D51000867E847E7888917A6D6B7A919482877EFC
:10D52000827B74838E8B71636F8C93898389817DF9
:10D530007C838C8F7B606A7D8C90858B7F797F83E9
:10D54000879887636A75839085888A777F838299B5
:10D550008E6A6B6D7A928E838B7B818486928F78B4
:10D560006768708990868182828587928C886D68D1
:10D570006C808B897F82838A8D8E838878636F75B8
:10D5800083897C868F8B8D8786897F656B6F7F848F
:10D590008183918C928484898770696A7382808484
:10D5A000939690867D8782816C65697B808A939A49
:10D5B000938C7B838189765E64787E828E99948F4A
:10D5C000837C858D7E61647479838E939291857A54
:10D5D00086887F69617077858E9392908B7883853A
:10D5E0007675636776818C8F8C9390838381747A50
:10D5F0007464787E7F838D93938B7C75757C816F4B
:10D60000767A7D7E9091978F7F6D777C8578727624
:10D6100076778891979D846D7A848180726E747319
:10D620007E8A9A9786707183848B796E72747A87FA
:10D6300096948477708087897E6C6D7474819494DD
:10D640008982767E8B847D6E6A726F7A898C858CF6
:10D65000827E8588847B6E756F747D848692897CDA
:10D6600080827F807576736F797C8C9498827978CC
:10D6700079817974746B68738A989C927D797C80C7
:10D68000807378696167808FA0968075787C827DD1
:10D690007C72646A788C9C9B846F75787F84786FC9
:10D6A000636974899B9A8C7A7377818A77696466D7
:10D6B000707F91959183707A848A7C706B676F76A6
:10D6C000878E908E747381857F6F6D6E73757E8D7E
:10D6D00090937F767A7D7A756C7273707280919375
:10D6E0009278787C837F767775686871838C9D8368
:10D6F0007275818281777867676C7F8AA395736E74
:10D7000079817E7A7568676F748BA19F7F6F738153
:10D71000857C736D606966809C9A897476828D8140
:10D72000726D6B69667A9298917C727B867F736F5B
:10D73000716767738D979C8A74757F7E717475624B
:10D740005C6C7E979D99847A797F777676665D6A40
:10D75000718E9A9C8E786F777A7C7D6F6469748401
:10D760009E9A967B6C707C7D776B6A666E7F989DC7
:10D770009F8C716B7C7D776E6B646B798D989B90C1
:10D78000776973807A77726D6E79809199907A6CEF
:10D7900071748078757671737A899C9585766C6ED4
:10D7A00078767378706F777E91998880736A7A7CC7
:10D7B0007C7F7A686E7A87938D7F736878828285A2
:10D7C0007A7368747F8F9089776A6A7D85857D75A5
:10D7D000666C7E8A918F7A706C7C91857C7B6864A4
:10D7E00073818A8F7D746F78938A7F78716B6D7780
:10D7F0008585847673798B858276766A717282816B
:10D8000089797A808783827475726B68757E858A60
:10D810007F8884847E7D757770636B787B8A8C8546
:10D820008780787A787D7B6961727B8E9887837B2D
:10D83000737A7D7D806A5C6A7B8EA393867E727428
:10D84000807C7F705960758A9E9D857F70727D8116
:10D850007F78595B728D98A089776E6B7582847C16
:10D8600068586B8697A6937A706C6C81887B6E6221
:10D87000667E8EA39B8070716E7F877D6E6B6874F1
:10D88000879A9C87706A707C888573746C748B9798
:10D89000968B7366757A7D83767676707F92918D9E
:10D8A0007F6C757E777F7D797D6F718588858574C6
:10D8B000717B777C868080796E7E857F867A6E7BB1
:10D8C0007C738087887F74757B838F8375707D768A
:10D8D0007C858A7F7669757E8B8A80707A7F7D856C
:10D8E0008F827A6A687B868482747582817E908E4C
:10D8F0007B7164708185837F74808978878B7D726A
:10D900006C6B7E878787787D8E7B7B84806F72636C
:10D91000738089887F7A8B877682867C776A657840
:10D920008589817B7D8B7F7981817A6F6871829017
:10D930008B818087807075837A726C67798A948A0C
:10D9400082848A736D84827973696F81918B7F7F02
:10D9500086806E798580746E6C7E91908081817BEB
:10D960006F6D8188786F697691998981827E7763FE
:10D970007585806E6B71839290807F7E806F7088DA
:10D9800086726B7779899382777B74766E7E8D7DD4
:10D990006B7B78829A8D787E7775747383837575C7
:10D9A00079779393827F78757C757E877F727770A5
:10D9B0008398887B79737C797689877671747D9476
:10D9C000917D7477737675808D7A6D737B8C988278
:10D9D000747A74747C8189806A6C787B9688767896
:10D9E0007A767F84898170697B818B8D7C6D787478
:10D9F0007F87807F7B6D7A8A858C896F727D7E853B
:10DA00007D7B80736F8781878F767180838180793A
:10DA100083796F797F78897D707B837B7F7D84803C
:10DA20007875828081817379837A737D807F7F703E
:10DA30007F8580847F78827D767C817F8074747F0F
:10DA40007E7E857E7A7B78788687817B6E7D807E00
:10DA5000858276777B777F87827C757685828387E0
:10DA600078757F7E7F837C7C77757D807F837E76F3
:10DA70007F82817F807D76747F83817E7C787B82CC
:10DA8000827B7D83787A7B7F827D7C817B858376B8
:10DA90007480787C797E7F7D798585838377727CBD
:10DAA000807D7B787B797E828783837C747C818395
:10DAB0007B7777777C848D807F74707684888071A3
:10DAC000767A7E8A85857F7772797D877E6E737E92
:10DAD0007F8F86817F7874807C858770737F828951
:10DAE00084787D79757E787F8479707E84838D7D5E
:10DAF0007A7C757A7B777F7D737B89828180787B66
:10DB000080797D7E78817D7885807E8379797E7944
:10DB10007980767D857C80867E818077787A797C35
:10DB20007C7A8F827582847C857979807C7B7D7715
:10DB30008789707A887D847E6D7F807A7E7D7F89FB
:10DB4000787483817E7C6E73837C79817F817F751D
:10DB50007F8B7F7D747083807A807E7C82797689EA
:10DB600084787F727D837C7E8379807C74828D76DD
:10DB70007A787A80857E7F7B7E827D7C8A7E7A7FC2
:10DB8000767E867B777A7C83857B798278857B76C7
:10DB9000818173797E84827A6E84868380737982B0
:10DBA000787A7F83867B6C7F8F8480716E7D7F76B1
:10DBB0007D82877B7278928D7F766C78847D77808A
:10DBC0008277757C919380756A758880787F7F797C
:10DBD0007B82879481746973828A7A7C7F7B7D865D
:10DBE0008486827470767C867E76797C8389868151
:10DBF000837674727A7F8374787F8C8881767F7C59
:10DC00007977777F8579777F8B8A7F72737E7F7C48
:10DC100074797F807A828E8D80707482847C747037
:10DC20007A7E7F838D90806B717E85807C70787C1E
:10DC30008682868D816C717C85847A71707E8589FF
:10DC4000838C8274707A80827E77727B828B8084F0
:10DC5000807D74787882818076777F85837E807EF0
:10DC600079717580828680757C83838280808070E4
:10DC70006C7782868777747F80847F8183776A76EA
:10DC80007F8A8F7F6F7A7D81827F837969727D89B8
:10DC9000928474747F8384807E7B6E6B7888928E8E
:10DCA0007B6B7B8287817C7C766E75868D8F7F6BAC
:10DCB00075838383787E796C71828B9186746D7D98
:10DCC00081807C797C75757D848B8F8072777F7C79
:10DCD0007F7B807B77787E86898777727A7D857E69
:10DCE000807E79787E84888D827372797D807A8156
:10DCF0007F7A7980868A8D766E787D8180807F7646
:10DD0000767A8486907B6E767B8284827F7E767242
:10DD100080858B836D717980837F7D807E7779812B
:10DD2000898B7A707A7F83827A807C747580848F05
:10DD300081737C8580807B7F7E75727D8085867710
:10DD40007A877B7D7C7F8278717A7F84887F7983F4
:10DD500080737B807A7C70738081868680808274F9
:10DD600078817E7A73717C817E8885808475727EED
:10DD70007E7A7D76787B7C878C838178717E7A7AD7
:10DD80007E7A7B7D7886918A837B7172777A807EBA
:10DD90007A747A8290918080766D707E83837A70B7
:10DDA00073818B95857D766C6E818684786E7280AA
:10DDB00088938D7F756D6A7B8684777072808A9177
:10DDC0008E83767475738581776F787C8A8D8E8566
:10DDD000797A7976847F7971767E8B8E88827B7D65
:10DDE000827978827979797E859085827F84848032
:10DDF0006E757B787B7E8486827E85868787726956
:10DE000076787B808784807D868989887965757A34
:10DE10007D8088837F7D8589888C7F6B6A7C828307
:10DE20008884787F868B888C7F75687781828281F1
:10DE30007D838388838987806C6F818283858081DD
:10DE40008A8583838684746A7982828485848179D1
:10DE5000767B81837C72747A81838484847B7676FA
:10DE6000808382776F7581818784837C76767F84D7
:10DE7000847F72707C808687867E787479828481C4
:10DE8000756F7580828685847D76767F86817A70CF
:10DE9000707E838587838079777E84827C756F79B5
:10DEA00081838584827D75767F82807D7474808194
:10DEB0008384858278777F7F817C7273797E80848A
:10DEC00084837E77757D81827B73777A8083868277
:10DED000817A72788083807975777F7F8683867C6C
:10DEE00072737D83837D74707B7F86878681776E76
:10DEF000798286817772767A7F8587837C70758157
:10DF000084847D737777808389858070717A83823A
:10DF10007F746F777B83868A847B71798083827933
:10DF2000707279818588887E736F7A81848075723A
:10DF3000767B82898784786F767E84817A6E757E1F
:10DF400082858A897E71707A80807E7373777F8202
:10DF50008A8B81776F767E83817973777A81888CDB
:10DF6000847A726F7880817F7775797F858A867FE2
:10DF7000766D6F7D81827B75797C818687847D73E8
:10DF80006E7981857E7976777F81868681746B72E2
:10DF90007F86837D75797C7F838585796E707D84AE
:10DFA00085827779797F8287877D6E6E768285829A
:10DFB000787776797E8587837670757D87857E779D
:10DFC00076787F8186837F72707783848379787691
:10DFD0007B80848583796F727D83857B7677767F7E
:10DFE0008185857E7674768083817A79767D7E825E
:10DFF00088817972747D82817E7877797E83878843
:10E000007F73717480807F7A79787A7F868A837B48
:10E010006F747E83807C7A7A787E8488857B726D4B
:10E02000788183807A7A777E8088877F746F6E7E2E
:10E030007F837D7C797D8184878477706F77818110
:10E04000807E797A7E8086877E7270747F82817B03
:10E050007D7B807F8285807672707A827F7F7E7CF6
:10E060007B7F808484777471787F817F7F7F7B7DE5
:10E070007F82827F7475757D80807F7F7E7C7F80CC
:10E0800082807A7574787D8180817E7B797D7F84C2
:10E090007D777477777F80807F80787C7E81807CBD
:10E0A0007775757B7F7F8081797B7F80817F7777B4
:10E0B000747C80827E817B7A7B80878279737274A4
:10E0C0007C7F807E80787A7F83857E7673747B8286
:10E0D00080807F79797F808583787573767F818171
:10E0E0007E7D787C8082847B7375767B807F808068
:10E0F0007B7C8083847E767377777C80807F7F7B58
:10E100007D7F83847B737575787E7E81807F7A7F47
:10E1100080847F757476767B7F8181807A7E82862B
:10E120008279727576777D8080807D7B8082857D27
:10E13000757274787D838281807B7B818282777324
:10E14000727678808181807E7B7F82837D7371751A
:10E15000797F808182827D7B818181767273777DF8
:10E160007F8284827F798081827A747377797D80DF
:10E170008585827A7B81837F757174787D828685BF
:10E180008178777F85847E73717579808787837ABC
:10E19000767A838580746F737A7B8687847E777ABC
:10E1A0007F86847A706E797C8388828077787F8599
:10E1B000847F746E787C8184847F7C797F82847F85
:10E1C000766F747B7F83837F7E7B7D7F847F7C7192
:10E1D000737A7F808282807F7F7E81837F76727771
:10E1E0007F80808080817F7D7980807A77767B7F59
:10E1F0007F818382817B7A7F82807874767D7E8046
:10E200008385827B7B7B82827D73767A7F80838429
:10E21000817B7A797E847F7871787E807F84837E2B
:10E220007E767D82837873767C7F808082817E7922
:10E23000787F857E7776787E7E8080857F7C7A8009
:10E2400082827B75767C807F82837F7F787A8183F0
:10E250007D7A75787A7F818283827D7B7D83817DE3
:10E260007676797D7F8183817E7E7C81857F7875DE
:10E27000767D827F848181807B7F82807777737BCC
:10E280007E82818381807F7D80827C7673777E80B1
:10E2900080828180807B7F80807975747A807F81A5
:10E2A000808180807A807F807576767D7E81838391
:10E2B0007F807C807F7E797676797E7F8083828185
:10E2C0007D7E807E7E7477777C80808482817F7C77
:10E2D0007D8080797576787E808384837E807F8060
:10E2E0007F7D7577767B7F8285837F80807F7F7C53
:10E2F00077777678817F848281817F7C7F7F7B7551
:10E3000077767D8182838382827E7D7C7B76777641
:10E310007A7F818383827F807E7B7C797776797F29
:10E320007F828682827F7E7A7C787A797A7C7F820D
:10E330008385817F807979797B7A7B797F818384FA
:10E3400083827E7D797A7B7B787A7A8080848481EF
:10E35000807F7979797D7C787A7F808283827F80E3
:10E360007A797B7C7C7B787C7F808482807F807ADA
:10E37000797C7E7B797B7E818082817F7F7E797EC6
:10E380007F7C7B787A807F8381827E80797B7B7BB8
:10E390007A7A7A7D8080818180807E7A7E7F7B7AA6
:10E3A000787A807F8480837E807B7B7B7B787977A3
:10E3B0007D80828282827F7F7B7C7B7979787A8084
:10E3C0007F818283817F7E797B7978787A7F808272
:10E3D000828480827F7A797A7A7A7B7E7F82838355
:10E3E0008182807B787A797B7C7C7F818383838147
:10E3F000807C79787A7B7C7D7E8182828382817E3B
:10E4000078767A7B7D7E7C7F82828382827E7A7838
:10E410007A7C807D7E7D8181828381807C79787B1E
:10E420007D807E7E8081828282807D7A797C7E7F03
:10E430007F7D7E80818281807F7D7B7A7D807E7EF4
:10E440007F7F80808180807D7C7C7D7D7F7F7F7FE2
:10E4500080808080807E7D7C7D7D807F807E8080CE
:10E46000807F807F7F7D7D7D7E7F7F7E7F808080BF
:10E4700080807F7E7D7D7E7F7F807F807F7F807FAD
:10E48000807F7E7D7D7F7F7F7F7F7F807F807F809D
:10E490007F7E7E7E7F7F7F807F807F8080807F7E8B
:10E4A0007E7E7F7F7F7F8080808080807F7F7F7E79
:10E4B0007F7F7F7F7F7F7F808080807F7F7F7F7F68
:10E4C0007F7F7F7F807F80807F7F7F7F7F7F7F8058
:10E4D000808082807F7F80817F7E7F807F80808040
:10E4E000807D7C7D7F807F808080807E7D847F7D3D
:10E4F0007C8082827F807F807E7B82807F7F807F26
:10E50000807E807F827B7D81807F7F7F7F807E7D1C
:10E5100083817B807E807E7E8084817E7982837E03
:10E52000807E7F827F8082817D7C7C7F8380807DF6
:10E5300080807D7D817E7F7D7B817F7F817F7F7EEF
:10E540007B827F807F80828382817F817E7D807DD0
:10E55000807F8280807C797E7C7981807C7D8381D4
:10E56000807E7E8183777E8C85827F7E7F7D8081A9
:10E570007F807D857D7C7F7E7E808184807C7E7CAB
:10E580007E827D7F807E807C7D8084807E88838487
:10E59000817D82828081877979847A7B7980817F8D
:10E5A0007D807F817E7D7C7E7F807F837F75808480
:10E5B0008080827A807C7B8080808D788A8981854A
:10E5C000817B7A807A7A8D83867E87847F746B7371
:10E5D000737B8B7A847C7F7A776D67716E778A81A3
:10E5E000858093857A837A7E80868787908D9C7ECE
:10E5F0008B83828B838387807F738581886F7E7313
:10E60000707875797D57946373835467AD884C8FA8
:10E61000C5417C7877CB5A279CCA7B5E7C59C47AEB
:10E6200008C5988C964A60B98F45A544A7A319BC24
:10E630009D3F305E97CEDB4D4EE1426BB4786C94DB
:10E640006B53D16257F41F80752468B9815A8F4586
:10E65000C1E420D788808E809BBA6A105F9172BE19
:10E660004D83A04D196EB661817A04E37453B99855
:10E67000476F7E2CB0A001C77DA86C529AD0A57FB1
:10E68000988A9FBB34A9A87A5184C9A8914231DEE7
:10E69000199E713D87874284D0456AFD1B9C784C4A
:10E6A00090D9B7705638629C41C76189AC5241B26B
:10E6B000BE58AFA44DEA402B997A5F84677AD60F93
:10E6C00042E85C9DAB79999D353AC88179A646951B
:10E6D000762445B1AF72AD606E9741D7CE9DC4A28E
:10E6E0005F94A23DD8E13F9E5E42B0AA72B5AE2DC6
:10E6F000EF950AAFB2C4BD552A8AA43FCAC1C6E38A
:10E700003032524164B9D6C8D3112DD94999B68354
:10E71000B1AA2444E1628ED161A9601552B1A680EC
:10E72000B6888C510A5DBADCC883433D46159BF21E
:10E7300077C97A6D734561DCEFC5D34932A2326B7C
:10E74000D6BC949F621C928B71ECA78960223BAA75
:10E75000E8E5ED874F450C7199A4D3B33E343F10E3
:10E76000AED49CDF811D2F382F89D28DC98011171F
:10E770004D5B8FA87F78870F77BA90E2987B8C4D9E
:10E780000E66D58EDD8F649A2E6291ABDCD7724512
:10E79000C1515AE896C5BE584F804A3DECBC89B677
:10E7A000415B6869A3E1DAA7690A7ABF73B6C1ACB5
:10E7B00084462667D8A5B5D24B783E2D9ADECCC8C4
:10E7C000A7426E5A0B9BB693A1682A6B822281E501
:10E7D00070554115558480A0CCA46C224E8AA5A208
:10E7E000BDA87D623D54F7BC85CD654D674580E58C
:10E7F000BB909E2F839A308DE6A28082555C86273F
:10E8000083F5B56654386B8C77A6EAA548032EAF1E
:10E810009E8FC1B25E392630C1E39EE294485951C1
:10E820006CD0CD74764A30674B72C09A524D3D29F8
:10E8300081844FD6C45832284A86978EBAA23112A4
:10E840003F9CC89E90AF893E5E4493F67870AD6B56
:10E850003E494986EA8E5A79535C6172C1E2893A2F
:10E8600058498D8C62C3D45C1125538AB46BB8CCE3
:10E8700056191B6CBDA7759CAF30481C52E88B5FC6
:10E880008E7C3830466BF6C263605D5C4F72B4E3D9
:10E89000B94D3F2C58926DA0C08036324874CA885A
:10E8A00094E067464368B1C299A1B950394045BB6D
:10E8B000AF82888C61425E91CDBA727C7167617360
:10E8C000A2BF8948664A3C7F5E87C28A4D5F68590D
:10E8D0008F889BD9814E4F5779968E92AB5D284792
:10E8E00061B1BB94989E6C4B718FCDB77189735A8F
:10E8F000646774AFA33E6F77417C7E91C9B463595E
:10E90000715282AA99C7954937466F9F9F94C576E1
:10E91000306864A7D0A692A26F45776EA5D6746FB3
:10E920007A4F476372A4D1745C965468908AB3C5D9
:10E9300071437059689174AB9B4444606694A276AD
:10E94000C5A63E667477B1A473958F254A6A72B3E3
:10E9500096678773426C908CEB9F568F6D578B91A7
:10E9600094BB812876555D988095A8694D72797B16
:10E97000C67596BD4F547A6D85A57B66A6353C8ECF
:10E9800068AFB281858A5E63A381C3BA4E78634A59
:10E99000728E8CA0A03F567B48989C99B390576488
:10E9A0007A5BA39B64B65E3967696FA6996BA272A6
:10E9B000308A819BBA987E866C5280898DB4686556
:10E9C0007A5D66919095B36454976387A7919A9204
:10E9D000524E7A5F80A370907F445A7F7A8FAD7ECB
:10E9E000869E476C918196926E7176406E9480B24D
:10E9F0008A6785725E8FA491BC85508473669396F6
:10EA0000858A663D6E76679B927F90605282897C94
:10EA1000B186738F504F8B84889978657849629856
:10EA20009AA19F76747E687BB0979796525F7959CA
:10EA3000779B8780864668876798A68D96795773F7
:10EA4000856D9C93727F6349738983929572776E0B
:10EA50005C8AA59AA389707167599591839C6353C9
:10EA60006F5E6D9DA18A9964527F7788AD9D89798B
:10EA700056477A7283AD8078744F618D8F94B27FE0
:10EA80007A7F557C94929A8968666349819686A5B7
:10EA900082607072688BB090938D45657668909DAA
:10EAA000877D6E416E7E74AF977F85605986988DA5
:10EAB000B58A68724E5B87919797796170556DA59D
:10EAC00092989C6F697D6E74AB8F8092575A716972
:10EAD0007B958C7F7C586880789CA08B85735B6964
:10EAE000867C8E9D6A716755768E8C959269776F5C
:10EAF000569E9793A17E606A695E939B7C8E6C5B49
:10EB00006A7580959C8C807263807C8D9D8B8076ED
:10EB10005E597E7B7AAB7275745C73919299A07C1E
:10EB20006F7C5886948C908365616A667CA8858B1F
:10EB30008068707D80929E888073517D7078968306
:10EB40007375615486847BAA8B7A7F6E708B9088F4
:10EB500093866871626A8A8984887665766978A9FD
:10EB60008D908E71737970849B7D7F785571736EF3
:10EB70008A907E7B7A647D937C959D7D777669779C
:10EB80008B79849067736465868A8A978B75816AAE
:10EB9000729D8C8A8D756C6F697090867A836C68B3
:10EBA0007B78839C948088766A8F77849B7F76704D
:10EBB0006067807786977C786D6A808E9098967A69
:10EBC000796C66888C808479666871668A9E7C928E
:10EBD000806F807D80979A7F866E5E7B6E7A8D8354
:10EBE000767069688085889E8E7E7971798A89873A
:10EBF000957B6D735A748A7F858B726D80678CA844
:10EC0000878C847173777784957D776F6470777B59
:10EC10008D94857B7A6A7F8B82A3947B7767677FED
:10EC20008778957C60765F74928C8A90846F7A7511
:10EC30007A9D8F7F7E72666B747B918A767D696F19
:10EC40007E7D91A08B7D8064758B74919278716AC2
:10EC50005F73837E90967374747089958E8F906DB8
:10EC600067766B8B8F7C8073616772739A947E8FEB
:10EC70007472807B859C8C777865607F79839682BF
:10EC80006F7271708D9488A9846E776E7B8F8A8382
:10EC90008D6A5B7063828F8387816C6C797D9DA4A4
:10ECA00086867B636C757C9199736D7554718380D6
:10ECB0009C9677727A68859385A0856968646A7F77
:10ECC000888190775F676C7F94948E918068777667
:10ECD00080A3837E80645D727783A57E7086616E7B
:10ECE00082869BA1866F73656F8383918C70606150
:10ECF00069788F899493676C7379949A8B8F855810
:10ED00006A72729A8B7A7E6F626E8189A4967A801B
:10ED1000766E7C858D9489676568587C808C967D3D
:10ED2000696F737A978B90A0706C737282908380F6
:10ED300081645C717489968A82816F687F8791A6ED
:10ED40007E7875626B7B828D8E686C716082889034
:10ED50009C8C737578748D8F8A947863676B7687D3
:10ED60008C7F867956757F8A9F91827F73647A82C1
:10ED70008C9C7B776D5E64778593957E76786D7AD3
:10ED80008B9399907869726F788E868C8163626DAF
:10ED90007686998B9188616D7D869694877F725F68
:10EDA0006777868E837A776B697989939F8F6F7D7A
:10EDB0006F6B848B8D8F7C5E6A696B888A90897299
:10EDC00068737E8A9793908269606F7A868C887D5B
:10EDD00076625E7B8598998580786B738B8C9F9823
:10EDE0006D726A6174838B90826966707384959C7E
:10EDF0009481706C797F8C9686806B5B6976818E4E
:10EE00008F82826C5C7F87979C8A817968667B8C15
:10EE10009391786B6C666D8595978F7A687B767D1C
:10EE20009699938269626F72808E8389735D6A7925
:10EE30008291978888776471868E928C8074695DE0
:10EE40006E898C928372756F6C8399999C846A73B6
:10EE50006F76878F8F826A5F6A707D8F9192846DE3
:10EE60006A7A878E9894817E605E7A82878D8174BB
:10EE70007060698D919A917E78726B7B8F96978284
:10EE80006A68676B7A8E90847864667C7D909E92C7
:10EE90008874626D7F8493957E7B5E5871818C91BE
:10EEA0008D8078696681939B9384786C646A829480
:10EEB0008B876D5F696A75919C90876C67787A8B98
:10EEC000989587726064757F88918A7B6B636D8586
:10EED00094989689776C63788C908F847066626062
:10EEE0007C958C947D6B70737A8E9E988B7267681C
:10EEF000747D8A938872635C6C80859C9684766846
:10EF00006A8190939A8B746C596A828C8F87766D24
:10EF10006A667A989C9586786F6F747F98998275E7
:10EF20005F5F6F738696917F6F617184859D9A8D07
:10EF30007B666073848A8F8877675C5F7B9096922C
:10EF400088776C6C7190A4968B7866686B748F97D9
:10EF5000887C6464707789999B8B76656D7A8491DF
:10EF6000998F7B6459637F888994836C69647B96ED
:10EF70009B958F7A6D696685959288756561666FD8
:10EF80008A9B9A84726C6F7B89989E9279665D7178
:10EF90007D83978F796B5E5F7E8F90A08E7A71678D
:10EFA000748F9A968B796A5B5F7690968B7C71688A
:10EFB0006A758BA59F88796B6B767D8E9D8B756648
:10EFC000546C78829596877667667C8F979C97803D
:10EFD0006A64687E91928680675B63708D9C948979
:10EFE0007B696C7281A39B88796661697385979050
:10EFF0007C685E677A8797A094796A686E8C939133
:10F00000927D625B60748C928E89716B63708F9F4E
:10F010009B8E7F6C69687292998D7B6A5F64738442
:10F0200095A487726C667685929B977D695E5F7EFC
:10F03000859090806F6160758E9A9B8E7D6E626EFA
:10F04000869A9A8C7B6C5A636F869F917E756864F2
:10F05000778396AB937D6C63707E899592816B57B5
:10F0600061798691958F7C696473889D9A91846A91
:10F070005E64748D9689817559646F83A09F8C7FBF
:10F080006D64717F919F967F675E616E8291958BB3
:10F09000705E62758C939C99846C65667E9995917F
:10F0A000876C5E5D6D8599978A7B68616F859AA490
:10F0B000937E6F635F7689979B80675F616E8193B4
:10F0C000A097796D616F86919B9A85655759718B71
:10F0D00095928978605A6E869FA89285755E6B7D41
:10F0E00093A2977B6C5B576E7F9BA08D7865637452
:10F0F0008596AB9F846A5C657B899495896B555B2B
:10F100006B839D9892846B5D6C8197A993846F59F2
:10F110005D6C879C9885715C5B6B809EA89B827000
:10F12000676D7C8F9B9F87645A5B69849494957903
:10F13000596370859DA29B8A715F6379929A9683C9
:10F140006D5C57647F9A9F917D6C62678098A8A0E0
:10F150008169615D6A868F9C8A685A5F6C83969F1D
:10F160009B89695D6E81919A9886705D566C8593D6
:10F17000988A7A685D677E9AA99B827663637989AB
:10F180009B9D82695D5A627D979F957D66627180C5
:10F1900093A4A18B72595F7486939387745C5668AD
:10F1A0007F979D928871646A7D91A69D8374605754
:10F1B0006580959A8A715E63667A9BA79F886E6563
:10F1C0006D7989979A8C6B595B6781919492846869
:10F1D0005C697F9CA29B8C77615B6D889C9D896F2D
:10F1E0005F565E7A96A29C826865657797A6A1892C
:10F1F0006E5D5A697D8F9E93725E5C687F96A09D5E
:10F2000090785B617D8D9E99877560506080929F3C
:10F210008F7D6B5D647C98A8A58B73646271819807
:10F220009C886D5B56657B92A09E856C626C7E901F
:10F23000A29F8F7A53566B8093978B7C64555E7D2B
:10F240009EA6988A786765738DA5A18A705C5B61BC
:10F25000788F9C947C625F697795A4A594746166AD
:10F26000728498968B7C5A52637C919A96857263CD
:10F27000647B9CA49F8C76645D658097998D726297
:10F280005C5D7791A2A28E6E666A73909EA1927564
:10F290005B59667B8B9A967D6957637F949E9F929C
:10F2A0007B675A748C999A8A7763565A778FA39C96
:10F2B000807167627691A4A4927662626D7A919D64
:10F2C0008D765E57647D899AA18C7864677E909A6A
:10F2D0009D8F7F624F637F92988B7B695B5C73939A
:10F2E000A7A48E786D686E849A9D8D775C5C637040
:10F2F000899896836B5D697D8FA1A5997B64606F0A
:10F300008291938E7E62545B778D989388796C633B
:10F310006F91A2A092776B6464748F99917E655E01
:10F320006574899DA490756568778A959F977C63BD
:10F330005763798894977F6F5D5B79939EA0927EE7
:10F340006D5F6581989B8B77635C5E718AA09D86FB
:10F35000766A6B778A9EA79679635D6F788B9792B2
:10F360007E65585F7889999E8E7F6A61748A999AC2
:10F370008F80695959708D978E817163626E87A8ED
:10F38000A5937D6A676D7C939C917B5D59636F84C7
:10F39000959A8D766164768B99A19A80685F667E76
:10F3A0008F908D82685A5B6E8E9C9B8D796C6A6F94
:10F3B000869FA2947B6661627084969381685D6289
:10F3C00075869AA3967F6A6371889098967E695A2B
:10F3D0005D72899192877A665F728E9DA09381712A
:10F3E000676179929D8E7B685F5F6C7F9B9E8B7758
:10F3F00068667783939F987F6A5B667C849192822C
:10F400006D5D5E7288999A95836E627085999A8F08
:10F410007F6C5E5D67859A918474676972829DAA2C
:10F4200098806A67707C88949180675A6070849035
:10F43000948F7A686572899A9A94846D60607589F0
:10F44000928B806F625F65869C9A8E80706D7380F0
:10F4500097A3977E6B62626E808D94876F646376EC
:10F4600085949D988471646C818F9092826F5E5CAC
:10F470006E869393897C6F636E849DA2928172667F
:10F4800064748498957B6B5D606E80909F917D6BBA
:10F49000647682909998856D60627484888F867690
:10F4A00062626F85989C908A73686C7E91988F8059
:10F4B00071625E6B7B939689786A69738294A39C70
:10F4C000866F656B79838F91866D5B5C6A8590949E
:10F4D00092806E667083999C92897563616E839247
:10F4E0008F7E73665E667E97A2967F736E717B8950
:10F4F000999E866B63616D7C86918E7B6766708852
:10F500009599988A7765677989909080725F5B6931
:10F51000808F948C7E74696E7F93A49884726765E3
:10F52000747E8B96856D61636C7D8D9B9988746A02
:10F5300073828E95928977625D6B7F8C8D867D6BF1
:10F54000666D80959F93867D6E6D748998937F70AC
:10F55000626169768C978D7B706E737F8D989C8FBE
:10F5600075646A74818A8C8878625E6C7D92928FF1
:10F57000887A6D717F9099938577675F697A8C91AE
:10F5800084766E6B697B8F9D9B87776E727B858E91
:10F59000938B6E5C5F6A7B878E8C80716A728492BB
:10F5A00098978E7D6C6571828C8E7F756C5D6378AB
:10F5B0008E9893807472717E8C9D9E8A7567686F39
:10F5C0007B838C89766867707D8B94968D7D696E60
:10F5D000808A948E867B6860697C8B91857F776C4E
:10F5E0006B7C919F9A8779716F73818F9285726717
:10F5F000656A7585969584727077808B9798917CF3
:10F60000616171808688837B6C60677B8F97908750
:10F610007E726F798C979483746C616976858F8A1A
:10F62000776E6F72798A989C8F7B6E6F7B848B8CE0
:10F6300089755D5E697A828C8D87796E6B7E8F9A13
:10F64000948D8271656A7C8C8D8271706B6976880D
:10F650009797897A79757A8795998B79696871779F
:10F66000818C8A806D646F7E8992948F83736B78AE
:10F67000868E8C827C6E60637385918B7F796F6CD4
:10F6800076899A9A8E7B70737379888F887967648C
:10F690006D798590968A7B6D717F8B92968F806E47
:10F6A000636B7A8685817F7368677A8B93918A7F93
:10F6B0007B7477818E91887C6F6A6B6C7F8D8C7E7A
:10F6C0007270757C89949A9880716F777F8589872D
:10F6D000806D616378838B8D887F786E778D94934E
:10F6E0008B7F766B6672828C84766D6C6D71809385
:10F6F0009B8D7E75767C848D958D7C69646B777E21
:10F7000085868277686F808B92969086796E707FFF
:10F71000898B81797066636E7F8D8A847D7674783B
:10F72000859398907F747174757E89878070686CFA
:10F73000787F8A908E8875737D838A8D8F857467B4
:10F74000667282848181796F6E768897948B827FCE
:10F7500079757D888D897D6D696F6F7B888F8579DF
:10F7600072777F878C979685776E727E8284837F8F
:10F7700071656575848B8A86857E74768492958B97
:10F7800080766F6A6D7C888A7F717072797F8C98C1
:10F790008F8379767A7F828A8E806E6667747D82A7
:10F7A00084847E726C7B8992928C868075707A8656
:10F7B0008A837A746E6D6F7B8B8E867F787A7D807C
:10F7C00087949284766D717578808680766D6E7779
:10F7D00081878E908B7C7377848B8A8481796D6727
:10F7E000697C85827F7C7674747D8C9A9082817B23
:10F7F00078767D88877E716D6D6F76808B8D7F7753
:10F80000788084888D908C7F6F6B75807F81807805
:10F810006F686B818D8F8C89827D787B85938C80DE
:10F8200077736E70777E84817A75767B8087919608
:10F830008C7F78797E8080887F7A6D68707B7F800E
:10F8400081847D777A838F908A89847972727B84B0
:10F85000847F77716E6E77838E8C88807F7F7F86C2
:10F860008D8F85796D6D71767B81857D736F7480E9
:10F8700087898F8D8578727B8488837D79736768AB
:10F8800072808382817F7C797F8993918A807A7A62
:10F8900075797F8580766D6E73757E888D8A7F7BA6
:10F8A0007C82868A8A8981776970797B7C7E7B7687
:10F8B000716C778B8E908A83817C7A808A8C7F763C
:10F8C000746D6E6F788388807A787D80808794925B
:10F8D000857A787A807F82827F6F666A777F848676
:10F8E00087847E7A7A89908D87827B706E717E8420
:10F8F0007F79767474777D89938E827F817D7F8214
:10F900008A897D746E7074757A80837E74777F8740
:10F91000888C908A7F77767D82807E7D7A736C7109
:10F920007E86868180827C7B828B928D847A7B75B9
:10F9300073757D837D716E71787B828B8C877D7C06
:10F940008087868485847B6F6C727B7E7E807F7CE3
:10F9500075777F8C8F8986827E78787F83817974B2
:10F96000717271717D8586817C7D8080848A8E88AC
:10F970007F78777A7C7A7F827E706F747B828587CE
:10F9800089847D7B8088888482807A7271767E8289
:10F990007E7B7A78797C838B8E8882817E7B7F7F69
:10F9A000858178737373787B7F83837D7A7D81848F
:10F9B000888A88847F787A7F807F7E7A787572776C
:10F9C000808484838280807F81878A857F7D797827
:10F9D000767A80817D79797C7D80848889857F7E37
:10F9E0007F81808280807B7474797E7F7F80807E3F
:10F9F0007B7D8288888382807C7A7C8081807C7A0F
:10FA00007A78797C828583807E7F808083858581FA
:10FA10007D7A7A7C7D7E80817D79797D8182838407
:10FA200083817E7D80838180807E7B797A7E8080E9
:10FA3000807E7E7E7D80828483817F7F7E7E7E80CD
:10FA4000807F7D7B7B7D7E7F8082817F7E7F8182C8
:10FA5000828181807E7D7E7F807F7F7F7E7D7D7FB6
:10FA600080818180807F7F7F808181807F7E7E7E9C
:10FA70007E7F80807F7F7F7F8080808080807F7F8F
:10FA80007F7F8080807F7FA503060A05FF641A3E82
:10FA900000FF090100FFFFFFC0FF00FFFFFFFFFFA6
:10FAA000FF0000830E0000FF010204080000102088
:10FAB000000000408000042D49100E0800000000E6
:10FAC000000000000000000000FF020406090C0F07
:10FAD00013171C21272D363D454F59636E7A8692A8
:10FAE000A0B0C2D6FAFFFF0A0000000010FF001409
:10FAF00014141414141414400A00FFFFFFFFFFFF36
:10FB0000FFFFFFFFFFFFFFFFFFFF000404040404EB
:10FB100004040402020202020202020000000000C9
:10FB200000102040000000000A2020000401020014
:10FB300070B01070000000000101014000000000E2
:10FB40000000000000000000000000000000644011
:10FB50000000014C442D472D33340054616D732057
:10FB6000456C656B74726F6E696B0000000000007D
:10FB7000FFFF00030200000000010800000400FF76
:10FB8000FFFFFFFFFFFFFF500251010608520791E0
:10FB9000B1BFA10305540412145513181A56199233
:10FBA000B257A215175816C1C959C5D9E15ADD93E4
:10FBB000B35BA3CDD55CD1090B5D0A0F115E109428
:10FBC000B45FA40C0E600D363861373C3E623D9543
:10FBD000B563A5393B643A484A65494E00664F967D
:10FBE000B667A64B4D684CC2CA69C6DAE26ADE97B0
:10FBF000B76BA7CED66CD23F416D4045476E469855
:10FC0000B86FA842447043E5E771E6EBED72EC99FA
:10FC1000B973A9E8EA74E9F7F975F8FDFF76FE9A79
:10FC2000BA77AAFAFC78FBC3CB79C7DBE37ADF9B10
:10FC3000BBC0ABCFD77CD3EEF07DEFF4F67EF59C66
:10FC4000BC7FACF1F380F21B1D811C212382229D1D
:10FC5000BD83AD1E20841F2D2F852E333586349E07
:10FC6000BE87AE30328831C4CC89C8DCE48AE09FDC
:10FC7000538BAFD0D88CD424268D252A2C8E2BA044
:10FC80007B8FB0272990285F7369636865725F3E38
:10FC90000000340206000030052016000000002F8E
:10FCA0007369636865725F00010000000200000074
:10FCB00002000000040000004D3B000085410000F0
:10FCC000A13F0000F93E0000ED3D0000713D000045
:10FCD0003D4200005942000095420000C142000030
:10FCE000894300008543000051430000ACAAA9A548
:10FCF000A3A69C9A999593968E8D8BB1B2B4B87445
:10FD0000726C6A696563665C5A595553564E4D4B21
:10FD10004771E8E4E2D1C9C5D8D4D2CAC6CC7817B5
:10FD20001B1D1E2E363A272B2D353933427300000A
:10FD30006672000024730000FC720000247300004F
:10FD4000F072000024730000FC7200006672000074
:10FD500066720000F0720000FC720000A8730000E0
:10FD6000A8730000A87300002A73000066720000E8
:10FD70006672000010730000FA7200001073000039
:10FD8000F072000010730000FA720000667200004A
:10FD900066720000F0720000FA720000A8730000A2
:10FDA000A8730000A8730000B4730000A0760000E0
:10FDB000FE750000FE750000FC75000092760000E4
:10FDC0009276000088760000FC75000092760000B4
:10FDD0008876000092760000FC750000987600009E
:10FDE000987600009876000022770000508400008A
:10FDF0001E8300002484000014830000248400007B
:10FE00002E84000024840000148300001E83000060
:10FE10001E8300002E840000148300000A8300006B
:10FE20000A8300000A830000808600007C8A0000AC
:10FE30003C8900003C8900003A890000548A000097
:10FE4000548A0000468A00003A890000548A000063
:10FE5000468A0000548A00003A8900005C8A00004B
:0CFE60005C8A00005C8A00005C8C0000E2
:10FE6C00001BB700600061006200630024002500E5
:10FE7C002600F00000000000001BB70000805101BC
:0CFE8C001027000000805101008051018F
:00000001FF
